:020000040000FA
:10100000C0870020017F0000CBD50100ED7E0000ED
:10101000ED7E0000ED7E0000ED7E0000000000008F
:1010200000000000000000000000000091800000AF
:10103000ED7E0000000000003D800000ED7E00001D
:101040003D82000097FB01003D8200003D820000D0
:101050003D8200003D8200003D8200003D82000094
:101060004DFB01003D8200003D82000081FB01003C
:101070003D8200003D8200003D8200003D82000074
:101080003D8200003D8200003D8200003D82000064
:101090003D8200003D8200003D8200003D82000054
:1010A0003D8200003D8200003D8200003D82000044
:1010B0003D8200003D8200003D8200003D82000034
:1010C0003D8200003D8200003D8200003D82000024
:1010D0003D8200003D8200003D8200003D82000014
:1010E0003D8200003D8200003D8200003D82000004
:1010F0003D8200003D8200003D8200003D820000F4
:1011000001F0FF01102A2BDB10F0070F08D010F8B8
:10111000013B013A8B422DD010F0070F42B3F6D1BC
:10112000F0B441EA012141EA014122F007047FF0D5
:1011300000070023F0E80256083C85EA010586EA2C
:10114000010685FA47F5A3FA87F586FA47F6A5FA68
:1011500087F68EB9EED1F0BC01F0FF0102F0070274
:1011600032B110F8013B013A83EA010313B1F8D11F
:101170000020704701387047002D06BF3546033800
:10118000073815F0010F07D1013015F4807F02BF39
:10119000013015F4C03F0130F0BC0138704700BF8A
:1011A0002DE9F14F03F11C0402EB840C4FEA930B81
:1011B0008A68CB680868496800F046F93CE9F000A5
:1011C0006040694072407B400BF1060E4EE083EABE
:1011D000134480EA134582EA134746BA96EA344438
:1011E000604000F00F1684EA063420F00F1684EAFF
:1011F000161054BA94EA0106724002F00F1486EAFF
:10120000043622F00F1486EA14124CBA6540694085
:1012100001F00F1485EA043521F00F1485EA14114A
:101220005CBA67407B4003F00F1487EA043723F071
:101230000F1487EA141344BA44404DBA4D4056BACD
:1012400056405FBA5F4087EA174886EA174B84EA40
:1012500017464FEA38488BEA1B4485EA1B4788EA61
:101260001B4580EA3440694072407B4000F0703496
:1012700000F0803500F00F3040EA440040EAD5002D
:1012800080EA900404F0332480EA8400604001F096
:10129000703401F0803501F00F3141EA440141EA38
:1012A000D50181EA910404F0332481EA840161408C
:1012B00002F0703402F0803502F00F3242EA44024C
:1012C00042EAD50282EA920404F0332482EA8402DC
:1012D000624003F0703403F0803503F00F3343EACB
:1012E000440343EAD50383EA930404F0332483EAF6
:1012F00084036340C943DB4381EA000483EA044674
:1013000086EA020183EA014382EA334583EA144311
:101310005C4084EA00077FEA040A8AEA024A8AEA11
:10132000010B87EA11488AEA374A80EA060181EA16
:101330001A418AEA030A04EA0A00454088EA0407D7
:1013400007EA0B0041408AEA0B0608EA060084EA35
:1013500034428AEA3A4602EA060358404540414090
:1013600087EA37438BEA3B4003EA000985EA09052F
:1013700082EA0309464006EA0906714085EA01004F
:1013800005EA3546464006EA314181EA304181EAC4
:10139000364606EA304686EA354634400F4086EA4D
:1013A000010508EA050886EA3640024088EA020894
:1013B00081EA314213405C4080EA020309EA0309F2
:1013C00087EA0907674088EA040806EA0A0601EA8C
:1013D0000B018AEA0B0425408AEA3A442040454042
:1013E0008BEA3B4B02EA0B02564084EA0B04234093
:1013F00059406E40694087EA364080EA384080EACA
:10140000060380EA104481EA134585EA344585EAFB
:1014100017427D4082EA354180EA05403CE9F00010
:101420006040694072407B40BEF1010E3FF6CFAE96
:1014300020BC00F05FF828606960AA60EB60BDE83E
:10144000F08F00BF00F000BA80EA101404F0F0142E
:1014500080EA0410604081EA111404F0F01481EA7B
:101460000411614082EA121404F0F01482EA0412BA
:10147000624083EA131404F0F01483EA0413634017
:1014800080EA102404F47F4480EA0420604081EA6A
:10149000112404F47F4481EA0421614082EA122489
:1014A00004F47F4482EA0422624083EA132404F4B1
:1014B0007F4483EA0423634081EA500404F05534F6
:1014C00080EA4400614083EA520404F0553482EA21
:1014D0004402634082EA900404F0333480EA8400DA
:1014E000624083EA910404F0333481EA840163406A
:1014F000704700BF82EA900404F0333480EA84002D
:10150000624083EA910404F0333481EA8401634049
:1015100081EA500404F0553480EA4400614083EAD3
:10152000520404F0553482EA4402634080EA1024F5
:1015300004F47F4480EA0420604081EA112404F42A
:101540007F4481EA0421614082EA122404F47F444A
:1015500082EA0422624083EA132404F47F4483EA8B
:101560000423634080EA101404F0F01480EA0410AD
:10157000604081EA111404F0F01481EA0411614022
:1015800082EA121404F0F01482EA0412624083EA40
:10159000131404F0F01483EA04136340704700BF8F
:1015A0002DE9F14F94464FEA930B8A68CB6808689F
:1015B0004968FFF749FF0BF1060E33E083EA134455
:1015C00080EA134582EA134746BA96EA34446040FB
:1015D00000F00F1684EA063420F00F1684EA161085
:1015E00054BA94EA0106724002F00F1486EA0436F7
:1015F00022F00F1486EA14124CBA6540694001F0DB
:101600000F1485EA043521F00F1485EA14115CBA31
:1016100067407B4003F00F1487EA043723F00F1470
:1016200087EA1413BCE8F0006040694072407B40D8
:1016300000F0E03400F0103500F00F3040EA5400C4
:1016400040EAC50080EA900404F0332480EA840074
:10165000604001F0E03401F0103501F00F3141EA53
:10166000540141EAC50181EA910404F0332481EA7E
:101670008401614002F0E03402F0103502F00F32D4
:1016800042EA540242EAC50282EA920404F0332498
:1016900082EA8402624003F0E03403F0103503F084
:1016A0000F3343EA540343EAC50383EA930404F087
:1016B000332483EA8403634081EA324787EA13458F
:1016C00081EA354690EA060484EA034B82EA1B422B
:1016D00080EA044484EA054483EA144A85EA14440F
:1016E0008BEA044B84EA374481EA0B4181EA1641D4
:1016F00004EA0A00454082EA04082BEA0800414057
:101700008AEA0B0602EA060084EA34438AEA3A4689
:1017100003EA060778404540414088EA38478BEAAB
:101720003B4007EA000985EA090583EA07094640C4
:1017300006EA0906714085EA010005EA3546464099
:1017400006EA314181EA304181EA364606EA30460E
:1017500086EA3546344008EA010886EA01052A404F
:1017600086EA364003405A4081EA31431F407C40BC
:1017700080EA030709EA070988EA0908544088EA69
:10178000020806EA0A0601EA0B018AEA0B02154082
:101790008AEA3A42104045408BEA3B4003405E40B3
:1017A0004240174079404D404E40E443F64386EABC
:1017B00018435D4085EA054083EA134386EA034106
:1017C00083EA384284EA114383EA04435FEA3343FD
:1017D000BEF1010E3FF6F2AE1ED4BCE8F000604050
:1017E000694072407B4020BCFFF784FE286069603E
:1017F000AA60EB60BDE8F08F2DE9E0414FF2F00206
:1018000080EA1031114080EA0130484041088208E6
:10181000C3084FF0000E4FE700F0113001F0113116
:1018200002F0113203F0113340EA410040EA820035
:1018300040EAC3004FF2F00280EA1031114080EA22
:1018400001304840BDE8E0812DE9F04F02F11C0570
:101850000646074600EB850851F8040B043A46F8A3
:10186000040BF9D14FF0010CFFF7C6FF5FEA3020FF
:1018700080EA0C001ECF41404A4053405C401EC6E7
:101880002000464517D04FEA4C0C1CF4807F18BF4F
:10189000ACF1E50C2C2DE7D03C2D06D1FFF7ACFFC9
:1018A00006CF41404A4006C6100006CF41404A409C
:1018B00006C61000D8E736E90F00FFF7C5FD043D66
:1018C00086E80F00F7D1BDE8F08F00BF30B44FF0CD
:1018D000000310F8014B11F8015B013A84EA05049A
:1018E00043EA0403F5D1A3F101034FEAD37030BCFE
:1018F000704700BF4FF0000310F8012B013943EA95
:101900000203F9D1A3F101034FEAD370704700BF7E
:1019100030B411F8014B12F8015B6C4000F8014B38
:10192000013BF6D130BC7047014B1B685B68184720
:1019300000000020014B1B689B6818470000002036
:10194000014B1B681B69184700000020014B1B68F6
:101950005B69184700000020014B1B689B69184712
:1019600000000020014B1B68DB69184700000020C5
:10197000014B1B681B6A184700000020014B1B68C5
:101980009B6A184700000020014B1B681B6B18471F
:1019900000000020014B1B68DB6B18470000002093
:1019A00010B4034C2468E468A44610BC604700BF30
:1019B00000000020014B1878704700BF900E0020F7
:1019C000042810B511D883B104280CBF1024282492
:1019D000A1420AD2064C54F8200018B141568A425E
:1019E000A8BF0A461A70002010BD6FF01500FBE773
:1019F0008009002030B50346114890F91C209A4216
:101A000019DD90F924209A4217DA9A1A846AA05CA8
:101A10000C4A15569D420DD00E32002918BF0130D8
:101A20009442C0B206D129B1013BDBB2012B01D8EF
:101A30000130C0B230BD0D20FCE70020FAE700BF46
:101A4000800900201852020008B5054B93F91C309C
:101A5000984203DAFFF7CEFF024B1B56184608BD2B
:101A6000800900201852020010B51C4C94F82C304C
:101A700073B9012384F82C3002F0E2FF48B1184B0F
:101A8000A362D823236284F824300823A361237738
:101A900010BD02F0EBFF0028F1D102F0F1FF0028A9
:101AA000EDD102F0AFFF38B10E4BA362D823236211
:101AB00084F824300423E9E702F0AEFF0028F3D1D4
:101AC00002F0B4FF0028EFD102F0C4FF0028EBD1F0
:101AD0004FF4DF71742002F035FE00BF8009002052
:101AE00053520200265202004FF0804201235360FD
:101AF0000023C2F80031014A13707047AD0900207D
:101B0000014B01221A707047AD0900204FF080434D
:101B1000D3F8003123B9034B187800F00100704767
:101B20000120FAE7AD09002070B50A4D01260446F0
:101B30002E70FFF7EBFF30B94FF080436E706C6092
:101B4000C3F8046370BD002CFCD0A04700236B6079
:101B5000F8E700BFB0090020024B00221A705A704B
:101B60005A607047B009002010B5034C208100F086
:101B70007DFD608110BD00BFB0090020014B588978
:101B8000704700BFB009002010B5EFF3108472B6A3
:101B9000064A937B0133DBB29373937B012B01D114
:101BA00003F061FB04B962B610BD00BFB0090020AC
:101BB00038B5FFF7E9FFFFF7A9FF094C4FF0804563
:101BC00040B103F07AFB01232B610423E37300236C
:101BD000237438BD0323E3730123C5F80433F6E708
:101BE000B009002010B5EFF3108472B6094A937B58
:101BF00023B940F2DD116D2002F0A4FD937B013B7F
:101C0000DBB29373937B0BB9FFF76EFF04B962B637
:101C100010BD00BFB0090020024BD87B003818BFB0
:101C200001207047B009002073B51B4D6B7C63B970
:101C3000E86900F0030003F030FB30B1EFF31083EC
:101C400072B6EA7B1AB103B962B602B070BD012266
:101C5000EA7303B962B64FF080430822C3F8082341
:101C60004FF42073ADF80630BDF80640A4B2631EF1
:101C70009BB2ADF80630002CF6D14FF080460748F5
:101C8000C6F80C4103F091FC85F82140FFF790FF66
:101C90000823C6F80433D8E7B0090020D009002093
:101CA0002DE9F041384C94F82230002B69D04FF0E8
:101CB0008043D3F80071D3F8046157B10122C3F80F
:101CC000082363782BB16368002565700BB19847D2
:101CD00065604EB14FF080430022C3F80421022218
:101CE000C3F80823FFF7A0FF4FF080462748D6F837
:101CF0000C8194F82150EDB203F05BFC20B140F26E
:101D00007E216D2002F01EFD47B1E37B032B05D140
:101D10000423E37303F0D1FA01233361B8F1000F18
:101D200016D04FF080430022C3F80C21E37B042B34
:101D300002D04FF42771E4E702F0ACFEC0B14FF0DF
:101D400080430022C3F8342C0223E373FFF74AFFD9
:101D50004DB1002384F82130E37B022B01D1FFF742
:101D600027FFFFF73FFFBDE8F041084803F030BC14
:101D700002F070FE0028E2D102F082FE0028DED1DF
:101D8000E2E7BDE8F08100BFB0090020D0090020E3
:101D900010B5054CE06900F0030003F07EFA00285E
:101DA000F8D0002010BD00BFB0090020F8B50546EE
:101DB00050B10278042A07D8437842B9013B1F2B5F
:101DC00002D88378212B07D96FF0150097E0002BFC
:101DD000FAD18378002BF7D1854B0127C3F88070A7
:101DE000BFF34F8FBFF36F8F4FF08046C3F8807102
:101DF000804C4FF0FF33C6F808330023C6F800319B
:101E0000C6F80431C6F80C31A373AB88A38103F084
:101E10002FFA08B12770A773D6F80C24D6F80C3423
:101E2000D20303D5DF0701D5FFF76AFE4FF4AF6099
:101E3000FFF79AFE2B78A97863740022E261A174FF
:101E40002274042B2CD8DFE803F00503192729009E
:101E50000123E36103F013FA002851D003F016FACE
:101E6000E36903F0030398424AD1AB79EBB9FFF77A
:101E70008FFF00281EDA40F2064113E0FFF784FED0
:101E80004FF08043D3F80C14D3F80C24CE03F9D5CB
:101E9000D007F7D50223DCE7574BDAE7574BD8E7F3
:101EA0004FF47E716D2002F04DFC4FF08043022212
:101EB000C3F80423A37C6BB12B785BB9FFF726FE34
:101EC000054602F0F5FC6FF00043002D00F08D8018
:101ED000C4E905034FF08043D3F80C24D3F80C3445
:101EE000D20303D5DB0701D5FFF70AFE404A0123E1
:101EF0000020E07384F82230C2F880311360F8BD0E
:101F00004FF080430122DA600022C3F80421E26925
:101F1000C3F8182502F076FD10B34FF080534FF050
:101F20008042D3F84432C3F34233C2F83C3502F066
:101F300069FD10B34FF080430122C3F84C254FF0E8
:101F4000804301229A600222C3F80423AA79002A5E
:101F5000B0D1D3F8042391071CD440F2AB31A1E7F0
:101F600002F05AFD0028D8D102F060FD0028D4D13B
:101F700002F070FD0028D0D1D9E702F04DFD002815
:101F8000D8D102F053FD0028D4D102F063FD00281F
:101F9000D0D1D4E71A4A1669116941F010011161D4
:101FA000D3F8043106F010060BB903F01EFB4FF016
:101FB0008047D7F8043133B1FFF7EAFE002805DA8D
:101FC00040F2C5316EE703F00EFBF2E726B90C4A8A
:101FD000136923F0100313614FF080430222C3F80A
:101FE00008230022C3F8042164E7C4E9053071E73F
:101FF00000E100E0B0090020010002000100030040
:1020000000ED00E010B50D4C04F1200003F0D1FA12
:1020100048B9E37B022B01D1FFF7CAFDBDE81040B0
:10202000074803F0D5BA074A012384F82130BDE8F8
:102030001040C2F80031FFF7A7BD00BFB009002073
:10204000D009002000E100E0094B1A7810B50446E1
:102050001AB13C216F2002F075FB5A7832B9012287
:102060005A70FFF791FD2046FFF75EFD002010BD7E
:10207000D409002038B5084C25781DB152216F20B5
:1020800002F060FB637823B1FFF766FD6570FFF730
:10209000A9FD002038BD00BFD4090020014B5B68BA
:1020A000184700BFD4090020014B9B68184700BFA8
:1020B000D4090020014BDB68184700BFD409002079
:1020C000034B1A780AB9FFF759BD988D704700BFC6
:1020D000D4090020024B1B780BB9FFF7A5BD704750
:1020E000D4090020014B5B69184700BFD4090020C8
:1020F00010B5144C2378A3B1236A9847002806DB57
:1021000094F82A3023B1012384F82E30002010BD2A
:10211000FFF7E8FF0028F6DA4FF48B716F2002F02A
:1021200011FB094B6361094BA361094BE361094B47
:102130006360094BA360094BE360FFF737FE00289B
:10214000E1D0E4E7D4090020911D00000520000043
:10215000191C0000891B0000E51B0000E152000073
:10216000064B10B51C7824B140F275116F2002F0B7
:10217000E9FAFFF7F9FC204610BD00BFD4090020A2
:10218000034610B3007888B91A79012A1ED85A7903
:10219000012A1BD89A680E49643A8A4216D8D86830
:1021A0000C4B98422CBF00200120704701280CD115
:1021B0001A79012A09D85A79012A06D8DA68044915
:1021C000643A8A4201D89868EAE70020704700BF65
:1021D0003C8601000040420F10B5054C236813B146
:1021E000984700232360BDE8104001F06FBB00BF9B
:1021F000040A002038B5044620B940F2A9116A202B
:1022000002F0A0FA90F82850072900F2EC80DFE8ED
:1022100001F004464676808AA39190F82630033B6D
:10222000012B02D94FF4DA71E9E7052390F8241065
:1022300080F82630002380F8293061BB714B0122E1
:10224000C3F84015C3F84011C3F84415C3F844114E
:10225000C3F84815C3F84811C3F84C15C3F84C111E
:10226000DA6003F059F82378012B0FD101F0D8FC84
:10227000C4E90601236A0021284698470146204602
:1022800003F061F8022840F0B18038BDD4E904239E
:10229000C4E90623EEE7BDE83840FFF79DBF90F89C
:1022A0002630DA1E012A02D940F2D511A7E790F8AC
:1022B00024202AB121462846BDE8384003F012B850
:1022C000042B0CBF02230123012980F82630036A66
:1022D0000AD10521284698470028D6D00378002B3C
:1022E000D3D04FF4F5718AE7062128469847002895
:1022F000CBD00378002BC8D040F2EF117FE790F8E5
:102300002630052B02D04FF4FB7178E7036A0221D7
:10231000B2E790F82630052B02D04FF4FE716EE73D
:10232000036A0121A8E790F82630052BB3D040F2CC
:10233000022164E790F82630052B02D040F20721F5
:102340005DE7036A0A21284698470146204602F0C5
:10235000FAFF40F20A2152E790F82630052B07D009
:1023600090F825200AB1032B02D040F20E2146E757
:1023700094F82420002A9DD194F8293093B10223A7
:1023800084F8263084F82920236A082128469847B3
:1023900000283FF47AAF0378002B3FF476AF40F289
:1023A0001A212CE794F8252062B194F8270084F8CC
:1023B0002530214601F03AFC00287FF466AF40F258
:1023C0001F211CE7022384F826300721236A2846B0
:1023D000984700283FF459AF0378002B3FF455AFDE
:1023E00040F226210BE740F22B2108E720B101281B
:1023F00005D1236A04213FE7236A03213CE74FF418
:102400000F71FCE6008000402DE9F843884607463E
:1024100080B300F037F84FF0000905465FFA89F6FF
:10242000AE420AD2304600F033F890F8264009F167
:102430000109002CF2D1FF2E03D16FF00B00BDE893
:10244000F883304600F024F80546848480F826405E
:1024500080F8286001460A4801F094FB202885F89E
:1024600027000AD001232F6285F82630204688F8FD
:102470000060E4E76FF01500E1E76FF02200DEE7AF
:10248000F5210000014B1879704700BF080A0020B1
:10249000054B1A79824283BF1B6800EB400003EBB7
:1024A00000100020704700BF080A002010B510F08F
:1024B00003040A460BD107490A71086030B102EBE8
:1024C00042021201214602F035FB204610BD6FF09A
:1024D0000D00FBE7080A002043F60952C0F3080389
:1024E00002FB03F3400A03F5807302FB00F000EBEC
:1024F0005320704743F6095CC0F3080210B50CFB8B
:1025000002F2C0F34E24030E43EA01230CFB04F055
:10251000090E02F580724FEA411C00EB52205A016D
:10252000B2EB030E4CEAD36C6CEB01044FEA841C53
:102530004FEA8E12B2EB0E024CEA9E6C6CEB040C6E
:102540004FEACC0C4CEA527CD200D31841EB0C0180
:10255000DA03C903801841EA534141F1000110BD7B
:10256000430B48F2376C0CFB03F34FEA134C00B5F6
:10257000104B43F6095E0EFB1C0000FB03F35B0DE2
:102580000EFB03FE03EB4C230EF5745C0CF1080C00
:10259000B0EB5C2F08D80EF5807EA0EB5E20C0B2B9
:1025A0000B6010705DF804FB013300200B601070AD
:1025B0005DF804FB6F0C0100F8B5274DA94246D821
:1025C000264E274F450F45EAC105A6FB0514C0F36B
:1025D0004F31A40B01EB054107FB1411A6FB015180
:1025E000890B41EA04411F4C04FB110448F2376C8B
:1025F000600B0CFB00F04FEA104C43F6095E1A48E2
:102600000EFB1C4505FB00F0400D0EFB00FE00EB31
:102610004C200EF5745C0CF1080CB5EB5C2F12D855
:102620000EF5807EA5EB5E2E5FFA8EFE069D85F888
:1026300000E00D0628184FEA112141F10001186051
:1026400059601460F8BD01304FF0000EEEE796219E
:102650009B2002F077F800BFFF7F841E83DE1B43C0
:10266000000024F40080841E6F0C0100420B48F22D
:10267000376303FB02F2120C43F6095C074B0CFBB9
:10268000120101FB0333013B5B0D0CFB03FC500209
:10269000B1EB5C2F88BF0130184470476F0C01000C
:1026A00010B5094A92F80033202B03D13E210220B5
:1026B00002F048F818214B43D018BDE81040D35819
:1026C00040680321184700BF100A00200C4B0D4939
:1026D0001B78012B14BF4FF4E0224FF4C022C1F845
:1026E000482318BF0023C1F80823074A99000A4469
:1026F0000021012B42F8041B00D170470123F8E7A9
:10270000500D002000B0004040B1004070B5EFF324
:10271000108472B6094A0A4B0025D2F80415D2F883
:1027200004612EB1596801315960C2F80451F4E7CF
:102730005B6804B962B6C0E9001370BD00B0004028
:10274000500D0020094BD3F80435C01A20F07F4308
:1027500023F001033BB120F07F40B0F5000F8CBFA8
:102760000220002070470120704700BF00B00040E9
:1027700008B5124BD3F8042522F00302C3F8042550
:10278000D3F8082542F00302C3F80825102292FA74
:10279000A2F2B2FA82F2092A04DD094840F2A73116
:1027A00001F0C6FFC3F810250122DA60054B4FF493
:1027B0008072C3F880211A6008BD00BF008000400D
:1027C0006765020000E100E0114B4FF40062C3F8BE
:1027D0008020BFF34F8FBFF36F8FC3F880210D4B65
:1027E00001225A609A60D3F80425002AFBD10A49D5
:1027F000C3F808134FF4E021C3F84813C3F840218D
:10280000C3F84421C3F84821C3F80421704700BF2E
:1028100000E100E000B00040020007000D4B4FF463
:102820008072C3F88020BFF34F8FBFF36F8FC3F860
:102830008021094B01214FF0FF325960C3F8082372
:102840000022C3F84025C3F840211961034B1A72D6
:10285000704700BF00E100E000800040500D002004
:102860002448FF2310B54FF0FF32002443724FF08D
:10287000FF33C0E9042304704460FFF7CFFFFFF784
:10288000A3FF1D4A1D4BC2F800424FF400611960BE
:1028900080691B4930B901230B60194B0222C3F830
:1028A000042310BD174B184CC3F8A845C3F8AC055A
:1028B000C3F85C194FF40021C3F804150521C2F8D0
:1028C000401501211160D2F840110029FBD04FF4CE
:1028D0000021C3F8081501215160D1600021C2F820
:1028E0004011C2F84015C3F8A815C3F8AC15C3F8D9
:1028F000AC15D2E7500D00200080004000E100E060
:1029000000B0004000F0014040810040014BD3E99D
:1029100004017047500D0020014BD3F804057047A7
:1029200000B0004013B56846FFF7F0FEDDE9000493
:10293000FFF7D2FD024B0021E4FB030102B010BD02
:102940000080841EB1F1FF3F08BFB0F1FF3F2DE9C9
:10295000F041404C05460E4638D13F4DD5F8003188
:102960007BB33E4E3E4BC6F808354FF00008FFF7EC
:10297000ADFE84F80980FFF751FFFFF7F9FE394BF0
:10298000C5F80081384FC6F8A8354FF40023C6F8C3
:10299000AC75C6F8043502F0FAFDD5F800312BB15C
:1029A0000123C5F800817B60FB60F4E7013041F151
:1029B00000010223C4E904012370FF236370BDE812
:1029C000F08102F0E4FDC51C41F10006D4E9047376
:1029D000B34208BFAF42F2D0204B214AC3F80825CA
:1029E000FFF774FE1C4A4FF4803125F07F48002326
:1029F000C2F808134046C2F84813C2F84031FFF746
:102A0000A1FE20B14FF43F716C2001F09BFEC2F893
:102A10004085C2F844132378012B06D127F07F4765
:102A20003846FFF78FFE0128FAD000236372FFF7C4
:102A3000F5FEFFF79DFE094A01234FF00041237088
:102A4000C2F8041504226270034AC4E90456C2F8AD
:102A50004833B4E7500D002000B0004000F00140C2
:102A60000000088000B100400080004037B540B150
:102A7000041FE4B2022C13D940F295316C2001F00E
:102A800061FE214B4FF48032C3F80823C3F84005A0
:102A9000C3F84001D3F840310093009B03B030BD30
:102AA0001A4D2B7893B16A7882420FD1184A19498E
:102AB000C2F80815012B01D1FFF7B0FE00232B70DF
:102AC0004FF0FF324FF0FF33C5E90423124A4FF4B1
:102AD0008033A340C2F80833C2F8483304F5A87322
:102AE00052F82300FFF72EFE012818BF0B4B22B22D
:102AF0004FEA84041CBF00211951084B53F82230BF
:102B00000193019BCAE700BF00800040500D0020E8
:102B100000F001400000088000B0004040B10040DB
:102B200070B52C4B30B1041FE4B2022C2AD94FF4FB
:102B300054710BE0D3E90401B1F1FF3F08BFB0F1DC
:102B4000FF3F06D11B7A23B94FF44A716C2001F084
:102B5000F9FD12B94FF44B71F8E71F4B4FF4803178
:102B60000120C3F80413C3F840255864D3F8441572
:102B700000248A42C3F8444503D82046FFF776FF75
:102B8000204670BD197829B15B78834202D14FF499
:102B90005371DBE7114B124E22F07F41A200134428
:102BA0004FF48035A5400022C6F808530846C6F801
:102BB00048531A60FFF7C6FD48B904F5A874012010
:102BC00046F82410C6F80453C6F84453D9E7104613
:102BD000D7E700BF500D00200080004040B100400A
:102BE00000B0004008B5FFF771FD054B4FF0FF3214
:102BF000C3F808230022C3F84025C3F8402108BDCC
:102C00000080004008B50122084B10B1C3F84423EE
:102C100008BDC3F84823FFF701FE054B4FF0FF3115
:102C200018704FF0FF30C3E90401F1E700B0004035
:102C3000500D0020F8B5164D164E00244FF4803785
:102C4000D5F8043307FA04F21A4212D056F82430A9
:102C50007BB1002346F8243004F5A87355F823000F
:102C6000FFF770FD28B1201DC5F80823C0B201F0A0
:102C70003FFA0134032CE3D1054BD3F8042132B1E0
:102C80000022C3F80421044A536801335360F8BD9D
:102C900000B0004040B10040500D002010B51C4C69
:102CA000637AFF2B2DD0237883B10122022B22726D
:102CB00021D1184B4FF40022C3F8082500232370BC
:102CC0004FF0FF324FF0FF33C4E90423124BD3F827
:102CD0000423D2031BD5D3F84021C2B14FF4803274
:102CE0000020C3F80823C3F84001FF236372BDE846
:102CF000104001F0FDB9022360782370FFF7B6FEA3
:102D0000E4E7054BD3F804330BB10720EFE710BD20
:102D1000500D002000F00140008000402DE9F04FF0
:102D200095B01C460492CDE90201FFF7EFFD182390
:102D300001910646C049082004EB440213FB040439
:102D4000631801EBC202083265581F7BD3F8048078
:102D500093F80D9005970FCA0EAC25F07F4A84E8D2
:102D60000F005046FFF7B8FBB44B7C1C984204445C
:102D700000F298819C4200F39380002C55DBFFF712
:102D800099F9B9F1010F834608D0AD4FD7E9022375
:102D9000B3F1FF3F08BFB2F1FF3F4BD0FFF790F90F
:102DA000019B0690B3F1FF3F08BFB6F1FF3F03D090
:102DB000B54278EB030378D2029B0322EB1A9342CD
:102DC00069DBBBF1000F00F0F88000230793029B42
:102DD000B5EB030B039B68EB0307FFF771F90930B1
:102DE000C217834577EB020380F0EB80049B012B35
:102DF00000F0F180079B002B5AD1019BB3F1FF3FFC
:102E000008BFB6F1FF3F53D0721B63EB0803042ADF
:102E100073F1000180F23881012A73F100033ADA7C
:102E2000DDF81CB026F07F4A52E004F1F45404F5BA
:102E30009024A4E70028B1D1FFF742F9019B069046
:102E4000B3F1FF3F08BFB6F1FF3F00F0B380B542DA
:102E500078EB0303C0F0AE803B7C002B069B14BFD5
:102E600000221A463346EB1A9A4214DC01230793D8
:102E7000D7E90232B2F1FF3F08BFB3F1FF3FA6D05E
:102E80000699EB1A68EB02028B4272F100039ED2A4
:102E9000B9F1010F9BD00024204615B0BDE8F08F9A
:102EA00004F1614404F5F70469E73346002285E73D
:102EB00028464146FFF746FD4FF0000BB8F1FF3FB3
:102EC00008BFB5F1FF3F00F0F2802E46CDF8048038
:102ED0005046FFF701FB5B4B221A9A420ED3001BB0
:102EE0009842C0F08C80554B9A4200F2C2809842C2
:102EF00040F2E780C0F1614202F5F702D3170020EB
:102F0000FFF70EFE04460028C5D04D4FB9F1010F62
:102F1000D7E9022375D0BBF1000F40F09780B3F1E1
:102F2000FF3F08BFB2F1FF3F00F0B5800120FFF77F
:102F300069FE3B7C002B40F0A1806A1E68F1000313
:102F40000620FFF7EDFD002851D0B9694FF080420F
:102F500000230B60C2F8083500238DF84830089331
:102F60004FF0FF324FF0FF33CDE90A23DDF814A014
:102F70008DF84590CDF83C808DF844A00E9508AFB3
:102F80000FCFDFF8C4904E460FC60FCF0FC697E89D
:102F90000F0086E80F0028464146FFF7ABFA53467C
:102FA00001331B1841F100012046C9E9043115B075
:102FB000BDE8F08F029BC21C55E7214FCDF81CB035
:102FC00056E7B9F1010B2846414618BF4FF0010BF7
:102FD000FFF7B8FC72E7019BB3F1FF3F08BFB6F102
:102FE000FF3F73D026F07F4A4FF0000B70E7BA69BD
:102FF0004FF080410123C1F808351360ACE742422D
:103000007CE7B3F1FF3F08BFB2F1FF3F24D1BBF132
:10301000000F8ED0069BF21A019B4FF0050063F162
:103020000003FFF77DFD002846D03B7C002B84D1B8
:1030300001233B7481E700BF100A0020FF7F841E3C
:10304000700D00200040420F180D0020B3F1FF3F2B
:1030500008BFB2F1FF3FDDD0FFF726F84FF0FF3297
:103060004FF0FF33C7E90223BBF1000F3FF461AF1C
:10307000D0E702F1F45202F590223FE70520FFF776
:10308000F5FC00233B7458E728464146DDF81CB0A8
:10309000FFF758FC12E7FFF701F802F078FAC7E9EA
:1030A000020143E740F21E41702001F04BFB40F269
:1030B0002A71702001F046FB40F22121702001F0BE
:1030C00041FB40F2EB71702001F03CFB40F28E615D
:1030D000702001F037FB00BF2DE9F04F8D4F7C7C55
:1030E00004EB44033B4483B05D78202D48D08A4BE9
:1030F000E6B26400002B00F08980884BDFF8209254
:10310000002B5FD005EB461207EB420A4FEA461848
:103110009AF81C30013BDBB2052B34D8814A12F8F7
:1031200003B0BBF1080F2ED0AFF30080EFF3108394
:1031300072B634443C449AF81D206270A278AA42C8
:1031400004BF2022A27013B9AFF3008062B6A84476
:1031500005EB450509EBC50207EB4808506859F82F
:1031600035300122594688F81C2098477C7C04EBB6
:1031700044033B44E6B25D78202D4FEA4404C1D1BC
:1031800003B0BDE8F08F40F25961702001F0DAFA27
:1031900062B6A84405EB450509EBC50207EB4808F4
:1031A000506859F835300122594688F81C20984754
:1031B0007C7C04EB44033B44E6B25D78202D4FEA6F
:1031C0004404DDD005EB461207EB420A4FEA4618ED
:1031D0009AF81C30013BDBB2052BD4D8514A12F8C7
:1031E00003B0BBF1080FCED0AFF30080EFF3108334
:1031F00072B634443C449AF81D206270A27895421D
:1032000004BF2022A270002BC3D1C1E7434BDFF8DB
:1032100014B1DFF80CA14FF02009002B4FD005EBC3
:10322000461207EB42024FEA4618137F013BDBB21E
:10323000052BA8D81BF803100829A4D0EFF310839E
:1032400072B634443C44527F6270A278954208BF03
:1032500084F80290002B52D0A84407EB480805EBF5
:1032600045050AEBC5025AF835305068012288F846
:103270001C2098477C7C04EB44033B44E6B25D7819
:10328000202D4FEA4404CAD17AE762B6A84405EB80
:1032900045050AEBC50207EB480850685AF8353077
:1032A000012288F81C2098477C7C04EB44033B44B3
:1032B000E6B25D78202D4FEA44043FF461AF05EBA0
:1032C000461207EB42024FEA4618137F013BDBB27E
:1032D000052B3FF658AF1BF8031008293FF453AFF6
:1032E000EFF3108372B634443C44527F6270A2788C
:1032F000954208BF84F80290002BC7D1C5E7019121
:10330000AFF3008062B6A844019905EB450507EBD1
:103310004808A6E7700D0020000000000000000033
:10332000100A0020845202002DE9F04F85B0DFF82A
:103330000C81019301EB41034FF0200C18F803407E
:1033400003916445924682F800C073D04B01DFF8C8
:10335000F09006469B4610E0727B012A02D0427D27
:10336000012A57D00BEB040308EB43038AF8004013
:103370005B7F202BA4465DD01C4604EB440009EB88
:10338000C000D0E9032387683568716813EB070E26
:1033900042F10002754571EB02024FEA4403DBD2B1
:1033A0001D46019B83F800C0039B4FEA431B28196D
:1033B00009EBC0003768B368D0F808A07268C1682C
:1033C000DB1942F100029A4571EB020310D3437DF1
:1033D000012B02D0737B012B03D0012005B0BDE887
:1033E000F08FFEF76DFEAAEB070701308742F4DA93
:1033F000019A254409EBC5051470A97DB27B0BEB3E
:103400000403914208EB430310D95C7F202CE4D0E5
:103410006500CCE70293FEF753FEED1B01308542B9
:10342000A0DA029B9AF800C01D46BAE7002005B05A
:10343000BDE8F08F019B1C70CFE700BF700D00202E
:10344000100A00202DE9F04F83B00C4615461E46A9
:103450009DF83070FFF70AF922686368451946F154
:103460000006954276EB030342D3DFF88C8005E03B
:103470005D4576EB09033BD3C4E900B90DF10703C1
:103480000DF1060239462046FFF74EFF88BB9DF836
:10349000073003EB430308EBC303D3E902A01A6927
:1034A0001AF1030B40F1000012EB0B0B627B40F1B1
:1034B0000009012ADCD05B7D012BD9D1FEF700FE8B
:1034C000ABEB0A0301308342D2DA9DF8073003EBFD
:1034D000430308EBC303D3E902B9FEF7F1FD013062
:1034E00010EB0B0B49EBE0795D4576EB0903C3D29A
:1034F000002003B0BDE8F08F100A00202DE9F0474E
:1035000015461C4612782F7A95F809C088B000231A
:10351000E360C4E90033A7739DF8408084F80DC0D0
:103520000646A360E2730F46002A3AD1FEF7E2FF97
:10353000D5E9042C3C4BC31841F1000E9A427CEBB8
:103540000E030AD3013E47F1FF37C4E900674FF489
:103550007A73A36008B0BDE8F087263041F100011E
:1035600082427CEB0103EDD3501E04F10C036CF19D
:103570000001009304AA06ABFFF71EF8049B6868DD
:1035800002330DF10F0205A91844FEF7E9FFDDE94A
:10359000053207999B1A23F07F43C4E90021A360F9
:1035A000D8E7224804F10C0206A9FEF7D9FF204B08
:1035B0001B78202B24D01F498B69D1E907210833C0
:1035C00042F1000A13EB01094AF1000A6B68207B03
:1035D0001844023005AA04F10801C4E9009AFEF774
:1035E000BFFF2869CDF8008032463B462146FFF7F1
:1035F00029FF0028AED1C4E9006708B0BDE8F08714
:10360000637B16F1080947F1000A012BDED0FEF7B3
:1036100051FD0028DAD1FEF753FD10EB090399465E
:103620004AF1000AD2E700BF0040420FFF7F841E2C
:10363000100D0020180D00202DE9F04700EB40038D
:10364000344DDFF8D480EC5C06464700FFF764F9A0
:103650004FF0200C4FEA461E04EB440108EBC10179
:103660000EEB0403D1F808A00A69AAEB000929F0BF
:103670007F49B9F5000F05EB43030DD812EB0A02A1
:10368000121A22F07F42B2F5000F05D8BCF1200FCC
:103690000AD12046BDE8F0875B7F202BA4461C465C
:1036A000DAD1BCF1200FF4D00CEB4613BA1905EBBC
:1036B000430315F802805B7FAB54710144464FF021
:1036C000040E0B1905EB430322469445204683F86C
:1036D0001CE05C7FF5D1BB192B440A4493F802E04F
:1036E000BEF1200F5FFA8EFC18BF8C443E4418BF19
:1036F00005EB4C0C05EB4202354408BF83F8018012
:103700004FF0200318BF8CF81D80A8705377204617
:10371000BDE8F087700D0020100A00202DE9F0416F
:1037200001EB41034A4DEE5C202E82B00C468046F0
:103730004FEA410740D1474B0BB1AFF3008001F096
:1037400026FFAB7C0191202B0AD0434BD3E906E244
:1037500010F1020C41F10003E64572EB030330D394
:10376000202E0AD042463346FFF7D8FA00283DD033
:103770000220AE7402B0BDE8F081D5E90223B3F1B6
:10378000FF3F08BFB2F1FF3F1FD12B7C43BB04209A
:10379000FFF76CF9FFF726FA0020FFF733FAA96963
:1037A0004FF080422020A874002301200B60C2F853
:1037B000083502B0BDE8F0810846FFF73DFF8642BC
:1037C000B9D0002002B0BDE8F081FEF76DFC4FF0EB
:1037D000FF334FF0FF32C5E902232B7C002BD6D0FC
:1037E0000520FFF743F900232B74D0E73A1906EBC5
:1037F000441305EB430315F802C05B7FAB54610132
:103800006246042013468A1805EB42029E42107756
:10381000527FF7D13A192A443C449678F0B2202ED0
:1038200018BF4018194418BF05EB400005EB4101D3
:10383000254418BF80F81DC0AB704FF000004FF05A
:10384000200308BF82F801C04B7702B0BDE8F081C9
:10385000700D002000000000180D002038B5164A39
:10386000164D4FF0FF304FF0FF310023C2E9020147
:10387000C5E90201202142F22000A970136082F8FC
:103880002830A9741C4628806B742B7405F11C0227
:1038900002F814300134202CFAD1094801F046F81E
:1038A000084B094A1C70107001F000F9A861FEF77E
:1038B000D7FF0123EB7438BD180D0020700D0020D8
:1038C000D9300000100D0020480D00202DE9F04FE8
:1038D00083B001F05CFEA44F06460C46FFF782F968
:1038E0004FF0FF334FF0FF32C7E9022397F828303B
:1038F000BBB9BB693A6AF9699C48023341F10001DE
:103900009B1802F5DF62A0FB02024FEA922241F10E
:1039100000019B1841F100019E4274EB010380F00D
:103920000E814FF0FF304FF0FF31FFF70BF8904A58
:1039300092F800B0BBF1200F00F011818D4D2023D3
:103940001370AB746B7C00223A6003EB43025FFAA6
:1039500083F915F802805B00B8F1200F00930BD0BB
:10396000DFF814A208EB48030AEBC3034FEA48024E
:10397000D97D012900F0B780009BDFF800A203EB9E
:1039800009062E444FEA49183478202C04D04846C2
:10399000FFF752FE8442F7D1BAF1000F01D0AFF326
:1039A000008001F0F4FDAB7C202B09D0D7E9062381
:1039B00010F1020E41F1000C724573EB0C03E3D3DE
:1039C000202C19D023460122FFF7A8F9002860D047
:1039D00008EB0B0305EB4303AC741A7F022A36D0C5
:1039E000FF23AB71009B4B441D446B78202B40F0B0
:1039F0008C8003B0BDE8F08FD5E90223B3F1FF3F1F
:103A000008BFB2F1FF3F07D0FEF74EFB4FF0FF3289
:103A10004FF0FF33C5E902232B7C002B5DD104203E
:103A2000FFF724F8FFF7DEF80020FFF7EBF8A969AD
:103A30004FF0804200232020A8740B60C2F80835A4
:103A400008EB0B0305EB43031A7F022AC8D14A4A4D
:103A50000BEB4B0102EBC102527D022A6CD0009AA3
:103A60004A442A440621197791782029CBB260D0A4
:103A7000434405EB430383F81DB0009B4B442B44A8
:103A8000D84405EB480883F802B0202388F81D309D
:103A9000A6E708EB040305EB430330785B7F337044
:103AA000024604211346424405EB42029C42117730
:103AB000527FF7D1B178B370CAB220291CBF4244FB
:103AC00005EB4202434405EB430318BF50774FF028
:103AD000200208BF70705A7756E70520FEF7C6FF30
:103AE00000232B749BE75B7D012B15D1033644F13A
:103AF000000402EB08030AEBC303D3E90202B0425D
:103B0000A24128BFC3E9026436E71D4B187803B011
:103B1000BDE8F04F00F026BF0192FEF7CBFA019A04
:103B20000028E3D1FEF7CCFA8619019A44F100048B
:103B3000DFE782F801B0A0E701221A7750E70C4BCB
:103B40000D4A1B78182101FB03F3D01807214068A8
:103B5000D358984740F2A621702000F0F3FD40F2C0
:103B6000B121702000F0EEFD180D00209300DC92D2
:103B7000100D0020700D0020100A00200000000031
:103B8000480D002038B505460C46FEF7ABFA002874
:103B900022DB14494B7C01F11C0C5FFA83FE0CEB19
:103BA000831C002302E00133202B13D01CF81320C8
:103BB000D8B2002AF7D10C4A03EB4E1E03EB4303A5
:103BC00001EB4E0142F8335002EBC30301220A77A6
:103BD0005C6038BD184638BD40F20731702000F0F7
:103BE000B1FD00BF700D0020100A00201F2808D86A
:103BF0000A494B7C00EB431301EB43031A7F012A74
:103C000001D0002070474B7C00EB431301EB4303D2
:103C10004FF0000C104683F81CC07047700D002058
:103C2000014BD3E904017047180D00202DE9F04F36
:103C3000AC4A53688FB0C3F3080383460491002B4A
:103C400040F0628108230393049B1B78012B00F250
:103C50003D82A54E26B1002140F23D50AFF30080D9
:103C60000023A24C05934FF0010926B1002140F238
:103C70004A50AFF30080B9F1000F04D19C4B0BB157
:103C8000AFF3008062B6657CEDB24FF00003A37124
:103C9000039B002B40F09880A84626B1002140F2FB
:103CA0005E50AFF3008001F072FC049A00950AABFD
:103CB0008246FFF723FC26B1002140F26650AFF3A5
:103CC00000800BEB481904EB49094FEA481799F8B3
:103CD0001C30013B012B75D80A992AF07F4AA1EBD1
:103CE0000A0222F07F4323F00103002B40F0BD8045
:103CF00008EB4802224407EB0B03907804EB4303E4
:103D00000421202819774FEA4803C1B200F09681B8
:103D1000394404EB410181F81DB0434423445F441E
:103D200004EB470783F802B020237B770023059339
:103D3000012726B1002140F26B50AFF300806D4B9C
:103D40000BB1AFF30080EFF31088C14672B6A379D0
:103D5000002B8AD1684B0BEB4B0C03EBCC0C0AAB62
:103D60000FCB0CF1080C8CE80F008FB1039B002BDC
:103D700000F0EA80059B23B1604B1B78202B00F0FC
:103D80006081637CDB4303F001036374FF23A37151
:103D9000B8F1000F04D1564B0BB1AFF3008062B6FF
:103DA00026B1002140F2A250AFF30080002F4AD18B
:103DB00026B1002140F2AE50AFF3008038460FB07C
:103DC000BDE8F08F0027B4E74D4B05F1010A0AF07A
:103DD000010A03EB851E03EB8A1CBEE80F00ACE86A
:103DE0000F00BEE80F00ACE80F00BEE80F00ACE823
:103DF0000F009EE80F002DB28CE80F00D0460FFA9E
:103E00008AF726B1002140F2DB30AFF3008005EBEA
:103E1000450507EB47076319625B9B78E25327442C
:103E2000BB7056B1002140F2DF30AFF3008026B105
:103E3000002140F25450AFF30080A379002B7FF4AF
:103E400014AF554629E7637C03EB43031C446378B6
:103E5000202BADD026B1002140F2A950AFF3008055
:103E6000284B187800F07EFDA2E722F07F42B2F5E1
:103E7000000F3FF63DAF0C9B5B18A3EB0A0323F04A
:103E80007F43B3F5000F3FF633AF0DF127030DF17C
:103E9000260229460AA8FFF747FA059000285AD1BA
:103EA00008EB480222440423907889F81C304FEA3A
:103EB00048032028C1B2434418BFC91923445F44B2
:103EC00004EB470718BF04EB410183F802B04FF041
:103ED000200314BF81F81DB082F801B07B77012761
:103EE00027E700BF00ED00E000000000700D00209B
:103EF0000000000000000000100A0020100D00204B
:103F00008C0D0020480D0020103B59B20029C0F252
:103F10008D8001F1604101F5614191F800335B0949
:103F20000393002B7FF490AE704B1B78202B00F096
:103F3000D280049B1B780393002B3FF48AAE40F29F
:103F40003651702000F0FEFBFF23A371B8F1000F83
:103F50007FF426AF1FE79DF826C09DF827E0F445C3
:103F600018D1BCF1200F00F09E8007EB0C0304EB8E
:103F700043035B7F89F81D30BC4404EB4C0C0022EA
:103F80008CF81DB05F4404EB4703059F05920322A4
:103F90001A77CEE6BEF1200F00F0A28007EB0E03E9
:103FA00004EB4303BCF1200F597F00F0878007EB3F
:103FB0000C0204EB42024FEA4803507F069051770F
:103FC0004FF0050A3A1804EB420201468E4581463D
:103FD00082F81CA0507FF5D103EB08022244079120
:103FE00092F802A0BAF1200F5FFA8AFE63D0BE44B5
:103FF00004EB4E0E069A8EF81D2003EB08022244B5
:10400000079982F80290394407EB0B024FF0200E1B
:1040100004EB410104EB4202F44581F81DE05077C6
:10402000AAD14344059A04F803B0ABE703F00F03A9
:10403000043B13441B7E5B09039372E782F801B0D3
:104040006BE629460220FFF769FB00287FF499AE52
:10405000637C03EB430020440BEB431204EB42026E
:1040600085780421DFB211775A015B00202DE9B277
:104070003B4418BF891823445A4418BF04EB41013C
:1040800004EB420283F802B04FF0200318BF81F81E
:104090001DB0059F08BF80F801B05377B8F1000F3D
:1040A0007FF47EAE77E608EB4803E35C89F81D30C9
:1040B0004FEA4803B5E7069951709EE708EB4802BE
:1040C0004FEA4803A05C0690A15479E740F23A51C8
:1040D000702000F037FB40F23351702000F032FBCB
:1040E00040F2CB11702000F02DFB00BF100D00201E
:1040F00070B586B007280DD8DFE800F0310C0C0C45
:104100000C1D040E604B4FF080419A690123C1F8E9
:104110000835136006B070BD5C4B5D4A1B7803EB3D
:10412000430302EBC30052F833304068042106B069
:10413000BDE870401847544C237C002B49D0D4E98B
:104140000223B3F1FF3F08BFB2F1FF3F00F08580CB
:104150000120FEF757FD0023237406B070BD4A4CC2
:10416000D4E90223B3F1FF3F08BFB2F1FF3F56D0BD
:10417000464E0120FEF746FD3378202B56D0454DA4
:1041800095F82520012A3BD0FDF794FF034600282F
:1041900035D194F89C200132D2B2312A84F89C2087
:1041A0006CD84FF47A7230786946CDE90032CDE9A7
:1041B0000233CDE90433FFF739FD002859D095F8D3
:1041C0002840012385F82830FFF780FB85F8284038
:1041D000A0E72E4B2E4A1B782E4903EB43034FF0EA
:1041E000FF344FF0FF35C1E9024502EBC30152F83D
:1041F00033304868052106B0BDE870401847337871
:10420000234A03EB430302EBC30052F83330406808
:10421000002184F89C1006B0BDE870401847FDF7F7
:104220003DFF01F0B4F9C4E90201A1E7637C03EBAF
:104230004301DAB2635C202B16D003EB421204EB8D
:104240004202507F6054FF21A171124D3370022150
:104250001177002285F8282092E7FDF71FFF01F073
:1042600096F9C4E9020173E740F24221702000F0A0
:1042700069FA4FF4C561702000F064FA40F22461DD
:10428000702000F05FFA00BF700D0020100D0020BC
:10429000100A0020180D002010B51B4B1B78202B96
:1042A00086B026D0194CD4E90223B3F1FF3F08BFF2
:1042B000B2F1FF3F22D1D4E904310DF10B02C01855
:1042C00041F1000104AB009203AAFEF775F99DF8D5
:1042D0000B20DDE904130F2A94BF0022012252189B
:1042E00043F100030520C4E90223FEF719FC06B0E0
:1042F00010BD40F2BF71702000F024FA4FF4F86155
:10430000702000F01FFA00BF100D0020180D0020D3
:1043100038B5254B93F800E0BEF1200F3FD0234D78
:104320006B7C95F811C003EB43035FFA8CFCEB5CEC
:10433000202B25D01E4C4FEA4C1C05E0634405EBB6
:1043400043035B7F202B1BD003EB430204EBC20231
:10435000917D8142F2D80EEB4E0E04EBCE04D4E9EF
:104360000213206940189168D26843F10003C41C0D
:1043700043F10003A14272EB030304D2002038BDD5
:104380004FF0FF3038BD0B4B081A03381C68FEF79E
:10439000A3F804F132038342F0D8001B38BD40F289
:1043A000FB71702000F0CEF9100D0020700D002080
:1043B000100A0020180D00202DE9F04F8C4B1D78BD
:1043C00087B0202D019000F00D81DFF82892DFF8F2
:1043D000288299F8113003EB43030646D8F8000011
:1043E00019F80340D8F8183003930DF11302D8F8E8
:1043F000203002938B46304405A9FEF7B1F87F4B7D
:10440000A6F132029A426AD8DFF8F4A1059BD8F8E7
:104410001C6005EB45050AEBC505A8681B18286953
:10442000D8F818501818401B20F07F43B3F5000F40
:1044300055D899F81120C8F82000202C88F826B00B
:10444000D2B200F0C2805201DC462021934604EB38
:10445000440240190AEBC20246F1000ED2E902639F
:10446000864273EB0E034FEA440746D3537D012B7C
:1044700003D098F82530012B35D005200091FEF7A8
:10448000F5FA009999F811004FF0FF324FF0FF3321
:104490002029C8E90223C0B240F0958000EB40001B
:1044A000202419F80030524A99F81110127802EBC2
:1044B000411209EB42025377D8F80030019A1344B5
:1044C000C8F80030FF2389F80630202C35D04D4B3A
:1044D000187800F047FA002007B0BDE8F08F0120FF
:1044E00007B0BDE8F08F0091FDF7EAFD751B0130C4
:1044F00085420099C1DA98F826C027440AEBC7071D
:10450000BB7D63450DD90BEB040309EB43035B7FD4
:10451000202B16D02146D8E90656D8F820001C4694
:1045200095E7DDE90231D8F818205B189B1A0220C4
:10453000C8F8203007B0BDE8F08F002007B0BDE814
:10454000F08F0520FEF792FA4FF0FF324FF0FF3365
:1045500099F81100C8E90223C0B204EB401309EB3B
:10456000430346005A7F00EB4003410119F803A0C2
:1045700009F803204FF0050C5346CF1809EB470705
:104580001A4694421D4687F81CC07B7FF5D1371828
:104590004F440A4497F802E0BEF1200F5FFA8EFC08
:1045A00018BF8C44304418BF09EB4C0C09EB420295
:1045B00048444FF0200114BF8CF81DA087F801A0DB
:1045C000857051776FE70C46C7E70520FEF74EFA76
:1045D00099F811004FF0FF324FF0FF33C8E9022382
:1045E000C0B25BE740F62401702000F0ABF800BFDA
:1045F000100D0020700D0020180D0020CE3F420F3E
:10460000100A0020480D0020BFF34F8F0549064BCC
:10461000CA6802F4E0621343CB60BFF34F8F00BF60
:10462000FDE700BF00ED00E00400FA05094B0122A0
:104630005A604FF0FF32C3F80823074B4FF4804213
:10464000C3F88020BFF34F8FBFF36F8FC3F8802173
:10465000704700BF00E0004000E100E0094B01228C
:104660005A604FF0FF32C3F80823074B4FF48052D3
:10467000C3F88020BFF34F8FBFF36F8FC3F8802143
:10468000704700BF00C0004000E100E0084B00227E
:10469000C3F8FC2F0122C3F8FC2F064B0222C3F8FB
:1046A0008020BFF34F8FBFF36F8FC3F88021704717
:1046B0000010004000E100E0F8B51B4E33780546DD
:1046C0000C46174663BB00F091F9FDF7CDF917488A
:1046D0007760002D18BF28463472FFF7D7FFFFF729
:1046E000BDFFFFF7A3FFFDF703FD0546B0B9FFF7D8
:1046F000B5F8FDF7EFFC00F09BFE002C0CDB04F09E
:104700001F026409A40004F1604404F5614401231C
:104710009340C4F880312360012333702846F8BDEC
:104720004FF0FF35FAE700BF100E00208A5202005A
:1047300008B572B6024B5B6803B19847FFF764FF98
:10474000100E00201FB572B6134B5D688DB9FFF7D0
:104750005BFFB2FBF6F2DCB20133002AF9D104F1BF
:1047600010036B4403F80C2C0A2234B901A8A847A3
:10477000EDE7024600230A26EDE7631E04AEDCB235
:1047800056FA83F3B0FBF2F602FB1600303003F862
:104790000C0C3046E9E700BF100E0020074B93F9E0
:1047A0000830002B09DB5A09012103F01F0301FA2D
:1047B00003F34032024941F822307047100E0020C6
:1047C00000E100E0014B1878704700BF100E002098
:1047D0002DE9F84FDFF8C4A0314C324DDFF8C89016
:1047E000074601269AF800805FFA88F8FF238AF8C6
:1047F0000030B8F1000F01D08AF80130EFF31082D9
:1048000072B600236660C4F80031C4F80431C4F8FD
:10481000047526603AB962B605E0D4F8043133B9BC
:104820002B69DB0620D4D4F80031002BF5D0D4F866
:104830000431002BE2D1B8F1000F13D19AF8013006
:10484000DBB28AF8018003214FF48042C4F80813D8
:10485000C4F80481C4F80081C9F880218AF8008076
:10486000002BBFD1BDE8F88F4FF48043C9F88031E9
:10487000EFF3108B72B60323C4F80433D4F800317D
:1048800013B9D4F804311BB1BBF1000FCBD1C2E78F
:1048900000F0A9FEBBF1000FC5D1BCE71C0E002043
:1048A00000E0004000ED00E000E100E0FFF790BF15
:1048B0001B4B4FF4805270B5C3F88020BFF34F8F6D
:1048C000BFF36F8F174D184C0021C5F80011C3F8C6
:1048D00080212669236943F0100323610123C5F871
:1048E000043306F010062B60D5F80031A3B11EB9D1
:1048F000236923F0100323610A4B0122D3F8080532
:104900005A60C3F808230022C3F80021044B4FF477
:104910008052C3F8802170BD00F065FEE4E700BF5F
:1049200000E100E000C0004000ED00E038B50C49B7
:10493000024605200138C0B2FF2803D14821692072
:10494000FFF700FF01EBC0031D7905F0FF04002D08
:10495000F0D141F8302001225C719C711A7138BD90
:10496000200E0020042808B503D958216920FFF73C
:10497000E9FE094B03EBC0000379012B01D059215B
:10498000F4E7437982790133DBB29A4218BF43716D
:10499000BDE80840FFF702BF200E002070B5124CA2
:1049A00006250026013D15F0FF0500D170BD94F8E5
:1049B000281004EBC1031A79012A09D158799A7990
:1049C000904205D05A79D2B29A7154F83130984752
:1049D00094F828300133DBB2042B94BF84F82830DC
:1049E00084F82860DEE700BF200E00204FF08052E0
:1049F000034BD2F830111960D2F834215A60704755
:104A00004C0E0020034B1868A0F10F035842584188
:104A1000704700BF4C0E0020034B1868A0F10A033A
:104A200058425841704700BF4C0E0020034B186895
:104A3000A0F10E0358425841704700BF4C0E0020B1
:104A4000034B1868A0F1100358425841704700BF4B
:104A50004C0E0020044B1868062803D0431C584213
:104A600058417047012070474C0E0020034B1868D6
:104A7000A0F10D0358425841704700BF4C0E002072
:104A8000034B1868A0F1080358425841704700BF13
:104A90004C0E002008B5FFF7BFFF20B1024B58684D
:104AA000B0FA80F0400908BD4C0E002008B5FFF7B1
:104AB000A9FF70B9FFF7B0FF58B9FFF7B7FF40B9CA
:104AC000FFF7C8FF044A054B002808BF13461846E5
:104AD00008BD024BFBE700BF00E701400C050040AA
:104AE00008B5FFF7B7FF08B3EFF3108072B6104AAE
:104AF0001369116941F010011161A2F5406203F0E0
:104B00001003D2F80011D2F804210A4300D040BFAC
:104B100020BF00BF00BF00BF00BF23B9044A136914
:104B200023F01003136100B962B608BD20BFFCE793
:104B300000ED00E02DE9F04184075FFA81FE5FD0CF
:104B4000002A59D0034601E0002A55D003F801EBB2
:104B5000990702F1FF32F7D14EEA0E24032A44EA04
:104B600004443ED9151FAE08172D06F10106C3F304
:104B7000800147D99846002940D048F8044B771A5D
:104B800003EB810C79080CEBC101CCE900440CF17A
:104B9000080C6145F9D127F0010C08EB8C01674541
:104BA000CCEB8C7805EB880517D02F1F032F0C60FA
:104BB00013D9A5F10807032F4C600ED9A5F10C07F6
:104BC000032F8C6009D9A5F11007032FCC6004D9FD
:104BD000143D032D0C6188BF4C6102F0030203EB0E
:104BE00086034AB1013A83F800E005D0012A83F830
:104BF00001E018BF83F802E0BDE8F0811546BEE78A
:104C00000346A9E719461546CFE700BF014B1B68CD
:104C10001B68184744000020014B1B685B6818475D
:104C200044000020014B1B689B681847440000208B
:104C3000014B1B681B6918474400002038B504204D
:104C4000204CFFF765FB2568854228BF05460421F7
:104C50002846FFF7B1FB30B10138C0B2012820D996
:104C600040F2431108E02368E068AB420DD1FFF742
:104C700013FB20B940F223116B20FFF763FDE268BC
:104C8000236822611344E36038BD05446089E56010
:104C90000123281A2375FFF7FFFA68B940F22D1196
:104CA000EAE70123E06823756389C01AFFF7F4FA85
:104CB00010B940F23B11DFE76289E3689B1A236178
:104CC000E2E700BF580E002008B50C4B1A7802F03E
:104CD000FF0312B15A1E1A4203D0DF216B20FFF7E7
:104CE00031FD19B1034207D1E421F7E723EA0003BC
:104CF0009B0601D1E821F1E708BD00BF4800002074
:104D00000C4B10B501221A761A68DA615A689A6259
:104D1000094A93F8300002214FF4827411701C8408
:104D200003F11801FEF782FF18B921466B20FFF747
:104D300009FD10BD580E00204800002070B5EFF3AB
:104D4000108572B6264C94F831600023012E84F849
:104D5000313006D0022E1DD0002E3BD185F31088B5
:104D600070BD85F3108894F8323003F0FF0123B151
:104D70004FF4A8716B20FFF7E5FC1420FFF7A4FFA8
:104D8000184B84F832601B78012BE9D1BDE87040E4
:104D9000FFF7B6BF94F8322012B940F26111E9E78B
:104DA000104984F832300B78023BDBB21E2B0ED850
:104DB000012202FA03F30C4A1342CFD144F2040257
:104DC000134204D020230B70FEF780FDC6E740F2AB
:104DD0007D11CFE785F3108840F2A311CAE700BF29
:104DE000580E0020480000204100004070B5144CCF
:104DF00094F8335025B140F286216B20FFF7A2FCD6
:104E0000104B84F8325001261E700F4B0F484FF4A0
:104E1000C852C4E900230E4BA360FFF787FD294663
:104E200084F834000B48FEF7ADFE202884F83000EB
:104E300002D140F29521E0E784F8336070BD00BFF5
:104E4000580E002048000020FF3F420F3D4D00005B
:104E50000500B700C54F000008B5104B93F833208C
:104E600022B940F2F5216B20FFF76CFCEFF31081C3
:104E700072B693F8312022B1012A0DD040F20531EB
:104E8000F1E7022283F8312001B962B693F83400C9
:104E9000BDE80840FFF766BD0022F3E7580E00208A
:104EA0000B4B93F8333010B523B94FF445716B2099
:104EB000FFF748FCEFF3108472B6064B1A78102AFD
:104EC00003D108221A70FEF701FD04B962B610BDC5
:104ED000580E00204800002070B5164B1B78042B9C
:104EE00025D1154E337D1BB973893068C01A70BD4A
:104EF00000F04BFB10F11E0441F10005FEF790FE9F
:104F000033691B1841F100019C4275EB01004FF021
:104F100000020CD2181B4FF0FF3361EB05018342F6
:104F200072EB0103E3D2A6216B20FFF70BFC0020FC
:104F3000DDE700BF48000020580E002038B5144CB3
:104F400094F8333023B940F2CA216B20FFF7FAFB03
:104F5000EFF3108572B694F8313023B1022B0DD0E7
:104F600040F2DD21F1E7012384F8313005B962B662
:104F700094F83400BDE83840FFF7F4BC054B1B78CB
:104F80000022042B84F83120F0D111F07FFEEDE7F0
:104F9000580E00204800002008B5094B1978102948
:104FA000CAB207D0202A05D0042A04D110221A70D0
:104FB00011F07CFE08BD4FF4E1716B20FFF7C2FBDE
:104FC0004800002070B50C46FDF7A6FC062C48D81A
:104FD000DFE804F00451512823645D000121022020
:104FE000FFF772FE304B314A93F8321079B1042149
:104FF00011701A68DA6000221A7593F83130022BAA
:1050000001D011F043FEBDE87040FFF717BE20232A
:105010001370BDE87040FEF759BC40F20E216B20C2
:10502000FFF790FB204E96F83230D3B11F4B1B7820
:10503000042B17D100F0A9FA05460C46FEF7F0FD47
:10504000337D012B0BD13269121841F100039542D7
:1050500074EB030303D3BDE87040FFF79DBF0CF072
:105060008FFD70BD124B0222C3F88020BFF34F8F1B
:10507000BFF36F8FF5E701210220FFF725FE0A4BF2
:1050800093F8323033B1BDE87040FFF739BE0121EB
:105090002820F2E7054B01221A70E2E7024B1B7D44
:1050A000012BB0D1D7E700BF580E002048000020E8
:1050B00000E100E07BB972B90029BEBF00204FF0CB
:1050C000004106E008BF00281CBF6FF000414FF010
:1050D000FF3000F057B8ADF1080C6DE904CE00299F
:1050E00009DB002B1ADB00F09BFADDF804E0DDE9B8
:1050F000022304B07047404261EB4101002B1BDBEF
:1051000000F08EFADDF804E0DDE9022304B040424D
:1051100061EB4101524263EB43037047524263EB40
:10512000430300F07DFADDF804E0DDE9022304B07A
:10513000404261EB41017047524263EB430300F090
:105140006FFADDF804E0DDE9022304B0524263EBBC
:105150004303704753B94AB9002908BF00281CBF50
:105160004FF0FF314FF0FF3000F00CB8ADF1080CFC
:105170006DE904CE00F054FADDF804E0DDE9022325
:1051800004B07047704700BF034613F8012B002A94
:10519000FBD1181A0138704708B5FFF727FCBDE8A6
:1051A0000840FCF761BC801A00F3070038B540B234
:1051B0000D4659B21446FCF747FC002328702044E2
:1051C0006B7040B238BD73B5A0F10B040E46E1B26E
:1051D0000F29154603D94F216420FFF7B3FA0DF1CB
:1051E000030332460420FCF7EBFB034608B15821C9
:1051F000F2E704EB840404F665149DF90300A2B2FF
:1052000001A9FCF7CDFB9DF804302B709DF805300B
:105210006B7002B070BD00230360704770470020C0
:1052200070474FF0FF3070474FF0FF3070477047C6
:105230004FF0FF3070470020704700207047002378
:10524000037070470022FFF7AEBF002070474FF099
:10525000FF3070474FF0FF3070474FF0FF3070471E
:105260007047C0B270474FF0804301221A60704708
:105270004FF08043D3F8080400F0010070474FF06E
:105280008043D3F8140400F0010070474FF08043CE
:10529000D3F81C0400F0030070474FF08041024631
:1052A000D1F81804D1F8181410F4803004D001F0AB
:1052B0000300831A58425841704708B5FFF7EAFBCC
:1052C00028B14FF080430222C3F8342C08BDFFF709
:1052D000C1FB0028F5D1FFF7D3FB0028F1D1F5E79A
:1052E000FCF714BC38B5054691F827000C46FEF7CC
:1052F0007DFC18B9E7216A20FFF724FA0023A38474
:1053000084F826300921236A2846984718B1037883
:105310000BB1EB21EFE738BD426808B503461144F5
:105320001A785960012AA1F1500006D1FEF7B4FFA6
:1053300040B9CB216A20FFF705FAFEF7ADFF08B9A7
:10534000D021F7E708BDF8B504460E4619B9012388
:1053500084F829303BE00D78032DF8D8DFE805F01C
:10536000390212154868C72802D800252846F8BD1A
:105370000421FFF721F80028F7D171682046FFF7D4
:10538000CBFFF3E7FCF728FFF0E790F82470F7B9BC
:105390004D682846FCF7F4FE0028D8D02B78D3B906
:1053A000012222702B79003B18BF012363726B79B5
:1053B000002B0CBF022304232372AB686F3363609E
:1053C000EB682361032384F8263084F82520FCF75A
:1053D00003FF0225CAE794F82630052B04D040F2DB
:1053E0008F116A20FFF7AEF927702B7994F8270008
:1053F000003B18BF012363726B79002B0CBF0223A3
:1054000004232372EB68A9686F336360D4E9063222
:105410005B1842EBE172C4E90432042384F82630BD
:105420002146FEF703FC0028D1D140F29111D8E7C4
:1054300070B5FDF727F8002405462646E0B2854200
:1054400000D870BDFDF724F80134868480F826600A
:10545000F4E7F8B504460D46FDF714F800270646B4
:10546000F8B2864204D8082D0CD96FF0150008E078
:10547000FDF70EF890F826300137002BF0D04FF0F2
:10548000FF30F8BD2CB129462046BDE8F840FDF7B5
:105490000DB821462046F8E738B50546FCF7F8FF79
:1054A000014688B190F824408CB990F8263073B149
:1054B000013B012B04D82846FFF714FF204638BDD6
:1054C000012380F82430F9E76FF00100F7E76FF06F
:1054D0002200F4E770B50D46FCF7DAFF0446002819
:1054E00048D090F82660731E012B49D8002D44D077
:1054F0002846FCF745FE00283FD02B78FBB9012356
:1055000023702B79003B18BF012363726B79002B4A
:105510000CBF022304232372AB686F336360EB6814
:105520002361032394F8270084F826302146FEF7F0
:105530007DFB40BB4FF42F716A20FFF703F9022E69
:105540001ED1002323702B79003B18BF0123637207
:105550006B79002B18BF04262672EB68A9686F339D
:105560006360D4E906325B1842EBE172C4E90432AD
:105570000423D7E76FF0010070BD6FF01500FBE763
:105580006FF02200F8E70020F6E7FDF7CBB907B58A
:105590006846FDF7BBF8DDE900024FF0807300219B
:1055A000E2FB030103B05DF804FB03460020187022
:1055B0007047EFF3108272B603780121DBB20170FD
:1055C00002B962B6012B0CBF6FF0220000207047B9
:1055D000EFF3108372B60022027003B962B60020A6
:1055E0007047FFF7DBB9FFF77BBAFFF779BA0028FE
:1055F0000CBF6FF015000020704700207047072394
:10560000037000207047002070470020704710B5DD
:105610000446FFF761FCA04294BF0020012010BDAA
:105620002DE9F04786468C460846089E1546744686
:105630001946002B40F0C2808542B2FA82F245D969
:105640004AB1C2F1200300FA02FC2EFA03F395409E
:1056500043EA0C0C94404FEA154EA8B2BCFBFEF88E
:10566000230C0EFB18CC08FB00F943EA0C439945C8
:1056700028D9EB1808F1FF3704D2994502D9A8F1CF
:1056800002072B44A3EB0903A4B2B3FBFEFC0EFB01
:105690001C330CFB00F044EA0344A04214D92C193B
:1056A0000CF1FF3304D2A04202D9ACF102032C4426
:1056B000241A43EA07401EB1D440002334607360CB
:1056C000BDE8F0874746DDE76346F1E792BB431B41
:1056D00001214FEA154EAFB2B3FBFEFC200C0EFBCE
:1056E0001C330CFB07F840EA0343984562D9EB18DA
:1056F0000CF1FF3004D2984502D9ACF102002B44E2
:10570000A3EB0803A4B2B3FBFEFC0EFB1C330CFBA3
:1057100007F744EA0344A7424ED92C190CF1FF3392
:1057200004D2A74202D9ACF102032C44E41B43EAA1
:105730000040C0E7C2F1200320FA03F195409040F9
:105740002EFA03F303434FEA154EAFB2B1FBFEFC52
:105750000EFB1C10190C0CFB07F841EA00418845B0
:1057600004FA02F422D969180CF1FF3004D28845FA
:1057700002D9ACF102002944A1EB08019BB2B1FBB4
:10578000FEFC0EFB1C110CFB07F743EA01439F4292
:105790000ED9EB180CF1FF3104D29F4202D9ACF1C3
:1057A00002012B44DB1B41EA004192E76046E3E73C
:1057B0006146F7E76046A3E76346B7E7834206D949
:1057C00016B9002108467BE7C6E900E0F9E7B3FA1D
:1057D00083F78FB9834201D3724508D8BEEB020428
:1057E00060EB030301209C461EB9002168E73846A0
:1057F000FAE7C6E9004CF8E7C7F1200CBB4022FAF3
:105800000CF41C432EFA0CF120FA0CF3B8400143BF
:105810004FEA14490EFA07F5B3FBF9F81FFA84FEB4
:1058200009FB18300B0C08FB0EFA43EA00439A45BB
:1058300002FA07F240D9E31808F1FF3004D29A4582
:1058400002D9A8F102002344A3EB0A0389B2B3FBF7
:10585000F9F809FB183308FB0EFE41EA03418E45B7
:105860002CD9611808F1FF3304D28E4502D9A8F172
:105870000203214443EA0040A0FB0298A1EB0E0181
:105880004145CE46434602D306D14D4504D2B9EB3D
:10589000020E68EB04030138002EA6D0B5EB0E0211
:1058A00061EB030101FA0CFC22FA07F34CEA030353
:1058B000F940C6E9003198E74046C5E74346D9E7D5
:1058C0002DE9F04F93F81080046987B01F46B8F1B6
:1058D0007D0FDB68039381460E46154600F22C814E
:1058E00008F1020304F2196A039984F81836424653
:1058F00050461FF0B1F804F5C06B58460FF088FC15
:10590000022E53D005D9F31E012B6AD96FF08505FD
:10591000ADE00023ADF8153095F85B30C3F34002DD
:10592000C3F380038DF8113001238DF81330884BB9
:105930008DF8102093F8C4368DF8143006F0010667
:1059400004A904F5C3608DF8126009F0FBF8002883
:1059500000F091807E4BD3F8BC361BB13A46002153
:10596000484698474FF0FF334FF0FF3258460FF04C
:1059700029FC4246039851461FF06EF894F8C2265F
:1059800095F85B3062F3410385F85B3094F8C326E9
:10599000DBB262F3820385F85B3094F89836052B0E
:1059A00069D8DFE803F06B62C6CC68C60023ADF8A7
:1059B000143095F85B30C3F34002C3F380038DF8D5
:1059C000113001238DF81230614B8DF8102093F8BF
:1059D000C4368DF8133004A904F5C36009F0E4F867
:1059E000B5E70023CDF8133095F85B30C3F34002E0
:1059F000C3F380038DF81130331F5E425E418DF892
:105A000010208DF812601AF0F9F901238DF8143086
:105A10004F4B8DF8130093F8C4368DF81530D5E947
:105A200008024C4B83424FF00203934118D34A4B78
:105A3000A0FB030103FB0211AB6AC01841F1000196
:105A40004FF47A720023FFF735FB1BF055FE0B462F
:105A500004A90246009104F5C3601AF0F0F976E754
:105A60004FF0FF306FF00041EAE76FF00F05284676
:105A700007B0BDE8F08F6FF00405F8E7D4F8A4563E
:105A8000002DF4D0D4F8A836D4F8AC2613434AD06D
:105A90002D78206800220023CDE9002300231A4638
:105AA000294603F099FD064600283FD0D4F8A416F5
:105AB0002A46013119F075F9002831DB94F8B03627
:105AC00086F8593094F9B136AE339BB2FE2B28BF1D
:105AD000FE2386F85A30D4F8A806D4F8ACC64FF4A2
:105AE0007A75A0FB050105FB0C1117A3D3E9002370
:105AF000FFF7E0FAC6E90801B262304618F0DAFEB4
:105B00002068314607F0C6FD0025304618F07FFEBC
:105B1000D4F8A4061AF0C1F90023C4F8A436A6E705
:105B20006FF00B05F1E76FF02205F1E76FF00B0561
:105B3000EEE76FF022059AE76FF0790597E76FF0CF
:105B4000680594E7AFF3008000CA9A3B00000000AC
:105B5000C00E0020037DC12500CA9A3B0000000052
:105B60002DE9F34706464FF0FF384FF0FF3900F5B7
:105B7000886A4FF0FF324FF0FF3350460FF0BCFA07
:105B800043681F78044600231A463946CDE9008948
:105B9000306803F021FD61683A460131054619F08D
:105BA00000F90746002835D1237C85F8593094F94F
:105BB0001130AE339BB2FE2B28BFFE2385F85A303E
:105BC000A27C95F85B3062F3000385F85B30A06837
:105BD000D4F80CE04FF47A71A0FB010C01FB0EC16C
:105BE00011A3D3E90023FFF765FAC5E90801AA620A
:105BF000E27C95F85B3062F3C30385F85B30306874
:105C0000294617F02BFF002804DB606867601AF054
:105C100044F9AEE70023606863601AF03EF9284655
:105C200018F0F5FDA5E700BF00CA9A3B0000000090
:105C30002DE9F8433E4D3F4C2B683F485B683F4F92
:105C40009847A3883A68023B13822B688046A07964
:105C50005E6907F081FC01463748B047237F384E24
:105C6000C3F30002D6F80090C3F300135B0043EACD
:105C7000820399F85B2022F00602134318F4807F18
:105C800089F85B3021D06369FBB1206918441AF0B0
:105C900000F825A3D3E90023FFF70CFAC9E90801AE
:105CA000C9F82820A07907F077FC2B6832689C6936
:105CB0003B6804212048A047431D1CD0E0B110F1EF
:105CC000230F0CBF0E200F2016E0217FA07911F0CA
:105CD00004041ED007F060FC18F0100F2B6804D0ED
:105CE0009C6932683B680221E4E79B681248984748
:105CF00048B1421DE3D10B20124B1870BDE8F843A8
:105D0000042007F081BC2B6832689C693B6801461F
:105D1000D0E707F041FC2B6832689D6906483B6874
:105D20002146A847C8E700BF00CA9A3B0000000010
:105D3000F4500020F01A0020DC500200F85000203F
:105D4000FC500020D9610020014B1B68184700BFA0
:105D500000010020014B1860704700BF00010020C7
:105D600007B50B46002102460091034800F080F879
:105D700003B05DF804FB00BF495D000030B587B09B
:105D80000025CDE903010446009503A905480595C2
:105D900000F06EF8DDE904309842B8BF255407B032
:105DA00030BD00BF81CE0100F0B5094E016802464A
:105DB0000A2700200B4601311C78355D6D0701D4A0
:105DC0001360F0BD07FB0043A3F13000F2E700BF12
:105DD000456402002DE9F84F15469A46D378234AC8
:105DE00012F803B06F2B81460F460BF0030B2BD03C
:105DF00026D8582B0CBF10260A26DDF828803246FC
:105E0000002348463946FFF7A5F9092A08F1FF386B
:105E1000D4B21ED83034B145E4B277F1000788F827
:105E2000004001D3D04511D82B789B0605D5082E0C
:105E300015D1AB7843F00803AB704046BDE8F88F4E
:105E400003F0F703702BD5E70826D6E781460F4607
:105E5000D5E7BBF1010F0CBF37345734DBE7102E09
:105E6000EBD1AB7843F01003E6E700BF45640200D6
:105E70002DE9F04F97B08A46039016461C46002540
:105E8000307808B9284656E325280AD0039B5146A6
:105E900098470028C0F24F83731C01350493049E79
:105EA000EEE71822002110A81EF0FEFD7378252BC6
:105EB00000F0A3800023711C98469E469C4618461D
:105EC0000F4611F8012B2B2A00F0C68000F2BD808E
:105ED000202A00F0C480232A00F0C4802BB19DF852
:105EE000483043F040038DF84830B8F1000F05D03A
:105EF0009DF8483043F020038DF84830BEF1000F84
:105F000005D09DF8483043F010038DF84830BCF1BF
:105F1000000F05D09DF8483043F008038DF8483055
:105F200028B19DF8483043F004038DF848309DF8BF
:105F3000483003F04401442903D16FF386138DF8F0
:105F400048309DF84830099743F080032A2A8DF89D
:105F5000483040F08C809DF8493043F001038DF8C3
:105F600049307B1C1A782E2A9DF849200CBF01214C
:105F7000002161F341028DF849200CD15A1C09928D
:105F80005A782A2A40F083809DF8492042F0040282
:105F90008DF8492002331A786C2A00F0A48000F2B0
:105FA0008680682A00F08C806A2A00F0A5804C2A3E
:105FB00000F0AA801A4612F8013B0492782B9DF853
:105FC00049208DF84B3000F217816D2B00F2A9802B
:105FD000692B00F21181572B00F2BE80412B03D0B8
:105FE000453B022B00F208819DF84A30042262F3FF
:105FF00002038DF84A300123CAE08DF84B30B31C00
:1060000004939DF84930D90740F1FD8054F8048B82
:10601000B8F1000F07DA9DF8482042F004028DF82D
:106020004820C8F100085A0740F1F68054F804BB34
:10603000BBF1000F80F2F5809DF849306FF341030A
:106040008DF849304FF0FF3BEBE02D2A0DD0302A80
:106050007FF444AF012333E74FF0010C30E74FF0FA
:10606000010E2DE74FF001082AE7012028E709A8D3
:10607000FFF79AFE099BBB423FF474AF9DF848209E
:106080001390C00F60F341028DF848206AE709A819
:10609000FFF78AFE9DF848301490C3F3400242EAAD
:1060A000D07262F341038DF84830099B73E7742A7C
:1060B00026D07A2A7FF47EAF9DF8492006210CE095
:1060C0005A78682A9DF8492006D1012161F3C60259
:1060D0008DF8492002336DE7022161F3C6028DF885
:1060E0004920013366E75A786C2A9DF8492001D18E
:1060F0000421EBE70321F0E79DF849200521ECE7B7
:106100009DF849200721E8E7BDF8482022F4F04235
:1061100022F0020242F4804242F00202ADF848202E
:10612000DFE76E3BD9B201238B4040F282410B4244
:1061300038D113F0240F52D1DF075DD59DF84A30D6
:10614000032161F302038DF84A3002F07803A3F1D2
:106150004000434243411BE0A3F15801C9B2012072
:1061600000FA01F111F4624F7FF43EAF40F60107EF
:1061700039421DD111F4043F3ED09DF84A3060F3FE
:10618000020302F07802402A8DF84A3034D000230E
:106190009DF84820C2F340010B4363F341028DF8A0
:1061A00048202EE79DF84A30022161F30203E8E718
:1061B0009DF84A10022002F0780260F30201402AA2
:1061C0008DF84A1002BF9DF8481041F001018DF88A
:1061D0004810632BDBD1131E18BF0123D8E79DF8AD
:1061E0004A30032161F3020312F0780F8DF84A3030
:1061F00014BF01230023CBE79DF8483043F001038F
:106200008DF84830C3E79DF94820002AB4BFDDF877
:106210004C804FF0FF3806E79F077FF513AFDDF89E
:1062200050B09DF849100023CDE913339DF84A3052
:1062300003F00703012BC1F3C30132D1CB1E042BA2
:1062400004D8DFE803F02045452020002368012919
:106250004FEAE372CDE910321BD19DF94030DA17D5
:10626000CDE9103204349DF8483013F003074FD0C5
:10627000049B03983246514616F038FE0028C0F2BF
:106280005A8105440BE654F8043BDA17CDE9103285
:10629000E9E70229E6D11AB243F3C033CDE910236E
:1062A000E0E7022B24D1CB1E042B04D8DFE803F057
:1062B000181010181800012954F8043B4FF0000280
:1062C00014D00229CDE91032CDD19BB21093CAE788
:1062D000073424F00704F4E80223CDE91023C2E7D1
:1062E00054F8043B109300231193BCE7DBB2CDE7D5
:1062F000042B08D1073424F00704D4E90023083420
:10630000CDE91023AFE7032BADD154F8043BDDE713
:106310009DF84B0078283FF6C2AD62281ED825288C
:1063200050D058287FF4BBAD0DF13E030093DDE95A
:1063300010010AAB12AAFFF74DFDBBF1000F814619
:1063400080F2C280B9F1000F3FF4A9AD0DF13E0615
:10635000A6EB0903002F7BD0013379E063381528C1
:106360003FF69DAD01A252F820F000BF3F6400004F
:106370009D6400009F5E00009F5E00009F5E000025
:106380009F5E00009D6400009F5E00009F5E000015
:106390009F5E00009F5E0000EB640000C36400008D
:1063A000FD6300009F5E00009F5E0000D56300005B
:1063B0009F5E0000C36400009F5E00009F5E0000BF
:1063C000C3640000039B514698470028C0F2B38085
:1063D000013564E5BBF1000FDDF840900ADB59465A
:1063E00048461EF0FDFBB9F1000F3FF458AD09EB34
:1063F000000620E04846FEF7C7FEF8E710980028A0
:1064000000F087800DF13E060AAB009612AA00212B
:10641000FFF7E0FCBDF84A3003F0EF0343F4F0432C
:1064200043F01003BBF1000F8146ADF84A304ADA61
:1064300000283FF434ADA6EB0903002708E0109BC9
:106440008DF8283000270DF129060DF128090123C8
:106450009DF84A1011F01002069260D00233139A90
:10646000059213444A0644BF14995B18B8F1000F13
:106470006EDDA8EB03089DF848305807C3F3800B86
:1064800066D459065AD53FB1039B514638469847C2
:10649000002850DB01355F46302350E01E075CBF0B
:1064A000C3F300135F01DDE9102348BF2B27002B46
:1064B000BFF63AAF524263EB4303CDE910232D27D9
:1064C00032E7002730E700279DF848100DF13E0322
:1064D000A3EB09036FF386119B458DF848107FF6F7
:1064E00031AFABEB030313932CE7109B07293FF667
:1064F000D6ACDFE801F00C04060C08080C0C1D708B
:10650000CDE41D80CBE4EA17C3E90052C7E41D6067
:10651000C5E4314E0746A6F10509052398E70807AB
:1065200048BF01339BE7184607935146039B9847A2
:106530000028079B04DA17B0BDE8F08F2023C3467C
:10654000594600290BF1FF3BEDDC45446D1AD84656
:1065500037B1039B5146384698470028EBDB01359D
:106560009DF84A30DA0601D41B0706D5039B514635
:10657000302098470028DEDB0135069B3BB19DF8B3
:106580004B00039B514698470028D4DB0135059FFB
:106590002F4406E0039B5146302098470028CADB71
:1065A00001357B1B002BF5DC039833464A465146E8
:1065B00016F09CFC0028BEDB0544A844A8EB0503AC
:1065C000002B7FF76CAC039B514620209847002896
:1065D000B1DB0135F2E700BF095E020008B50446F1
:1065E000EFF31183402383F31288BFF36F8F06F01C
:1065F0002BFD204601F0B6FC024816F053FC17F0C4
:1066000004F8FCE70A5E02002DE9F047858B04469A
:106610002807904611D4022905F0070540F0CC80E8
:10662000204616F095FC78B10138A18B042811D8CA
:10663000DFE800F0C2106D85950001290CBF45F020
:10664000100545F02005A58388F31188BFF36F8FEF
:10665000BDE8F08701F0070AAA4500F0A5800027F1
:10666000B9463E46A368002B00F0BC8041F008010B
:10667000A18388F31188BFF36F8FA168002900F010
:10668000BA800D68002900F0B680D1F80480334646
:1066900052462046C047002D76D02B6829461D461D
:1066A000F0E701F007035A1F012A1BD8002221F04E
:1066B0000701062B276889B2C4E9002209D13B46AD
:1066C00003E0E28B0132E2831B68002BF9D141F039
:1066D0000201A183204616F03BFC00287AD041F04D
:1066E000200176E0042B0AD121F0070189B2A183B1
:1066F000204616F02DFC10B141F02001A183A18BA2
:1067000001F0070AAA454FD00027B946AAE7236936
:1067100021F0070141F00601062DD3F80090A18376
:106720002DD1B9F1000F3FD041F00801A18388F3CA
:106730001188BFF36F8F3A492046C84729E021F0FE
:106740000701236941F0040189B2042DD3F80490B4
:10675000A183E6D000273E464FF0040A82E721F0ED
:106760000701236941F0050189B2052DD3F808908E
:10677000A183D6D000273E464FF0050A72E70027D6
:106780003E464FF0060A6DE72B4687E7B9F1000F4A
:10679000D1D1EFF31188402383F31288BFF36F8FB9
:1067A000A38B23F00803A383A58BEA062ED525F03F
:1067B0001003A38305F00705A669A18B002EBFF681
:1067C00070AF00232768C4E9003321F0070141F0CE
:1067D0000101A183A18B01F0070AAA454FF000092E
:1067E0007FF440AF002F9CD041F00801A18388F3D3
:1067F0001188BFF36F8F002FC8D03D6839463346EC
:106800005246204616F0D0FB2F46F4E7AB067FF544
:106810001BAF25F02003A38305F0070500E700BFA9
:10682000D5CF0100014B036000207047D852020011
:10683000F0B40C4B0C4E5F6A0C4BB34203D36FF0B9
:106840008500F0BC70475D68BD4209D31C693CB14E
:1068500095F802C00579AC4502D12346F0BC184733
:106860002433EAE7E03900206409002040090020D1
:106870002DE9F047134CDFF85080DFF850900546C3
:106880000E461746444503D36FF08500BDE8F087F8
:106890006268D9F824309A4212D3A36983B1907800
:1068A0002979884205D13A4631462846BDE8F04765
:1068B00018475279012A03D13A463146284698476B
:1068C0002434DFE74009002064090020E03900207B
:1068D0002DE9F0410B4CDFF8308005460E46174697
:1068E000444502D36FF0850009E063690BB9243495
:1068F000F6E73A463146284698470028F7D1BDE8E2
:10690000F08100BF400900206409002010B5044652
:1069100018F08DFD10F1780F00D050B9054A2046CF
:1069200016F0E4FCD2F8C43023EA0003C2F8C43005
:10693000002010BDE0390020024B00221A605A608E
:10694000704700BF9B3A002070B50B4B0B4CA34225
:1069500001D3002070BD196A1E7F00220439D5B210
:10696000AE4201D82433F2E7013211F832508542A9
:10697000F5D10120EEE700BF4009002064090020A6
:1069800008B509480378C3F341130A3350F823309C
:106990003BB100F1080200F110019847C043C00F5D
:1069A00008BD1846FCE700BFE039002004282DE9A7
:1069B000F14FDFF8989004460F4616D001282DD1EC
:1069C000DFF88C8098F8B93043B300F0D9FD214D41
:1069D0004D4520D2D5F820B04FF0000A2B7F5FFA4A
:1069E0008AF6B34204D82435F2E7FFF7A5FFE7E7BC
:1069F0000BEBC6060AF1010A307918F018FD0246C1
:106A0000307916F073FCD8F8C430002A23EA00036A
:106A1000C8F8C430E2DA002388F8B9300D4D4D458E
:106A200008D30B4B1B6A6BB13946204601B0BDE859
:106A3000F04F1847EB681BB13A4621462846984765
:106A40002435ECE701B0BDE8F08F00BF64090020F9
:106A5000E03900204009002073B5C4B263060D463A
:106A60008DF8074007D02046FFF76EFF78B10D4B39
:106A700093F8BA0058B10B4E204655B103F0AAFD69
:106A8000F3691BB10DF1070108209847012002B0FE
:106A900070BD03F0C7FDF369002BF7D00DF10701BE
:106AA0000920F2E7E039002073B586788DF80060A0
:106AB000037942791C4C43EA0223ADF80230C378D3
:106AC000304603F003038DF8043016F00FFCD4F8C1
:106AD000C430184205460BD0304600F033FD304636
:106AE000FFF714FF1AF009FC10B996200FF0EEF82A
:106AF000684603F04BFD10F1780F03D010B1002071
:106B000002B070BD9DF8000003F0C8FD10F1780FD1
:106B100001D00028F3D1D4F8C43001202B4384F8ED
:106B2000B900C4F8C430EBE7E03900202DE9F047A4
:106B3000924DAB6904460E461746C3B9207800F063
:106B40001F00012876D0022800F0DC8000BB94F9F9
:106B500000103A68637800292EDA062B0CD0082B37
:106B600025D0ABB9537001231370022303E198477A
:106B70000028E3D100200DE06388190A0A1F012ACA
:106B80008C4605D9072903D8DAB26B6A1C781CB980
:106B90006FF01500BDE8F0875D78654503D182424E
:106BA00000F0E48001302344F0E71B78E3E095F83F
:106BB000BA3013700123DEE0052B11D0092BE7D189
:106BC00063886E6A002B32D1FFF7B6FE638885F8C2
:106BD000BA30EB69002BCDD0694903209847C9E74B
:106BE000A07803F0C1FC0028C4D0D1E77378042B4F
:106BF00010D0052B11D0022B04D177796388BB42CA
:106C000008BF012033781E443378002BEED10028D2
:106C1000BED0D9E796F80380F4E76388BB42F1D190
:106C2000B8F1000FEED13046FFF73EFFEAE7FF274D
:106C3000B846E9E795F8BA30D7F800C0002BA7D0DE
:106C40006F6AA28894F804E03B46187800289FD029
:106C50005978022904D193F80480F04500F292801B
:106C60000344F2E78CF800308CF80130316081E7A2
:106C70001F4493E00B2B8BD100264FF0FF08C14639
:106C8000B24606E07B78042B0FD0052B21D03B7851
:106C90001F443B78002BF5D1EB6913B15146072017
:106CA0009847002E7FF466AF72E797F80280A388BA
:106CB00097F803909845EAD163889945E7D1B8F1F0
:106CC000070F1CD805EB0803BA4683F8BB900126D2
:106CD000DDE7A3884345DAD1A3784B450AD0BE78D7
:106CE000304600F02FFC3046FFF710FEB0FA80F679
:106CF0007609CCE73846FFF7D7FE0646C7E7BA461F
:106D00000026C4E794F900206378002A18DA002BE3
:106D10007FF43EAF24793F6863060AD02046FFF730
:106D200013FE00283FF434AF95F8BA30002B3FF43F
:106D30002FAF3946204603F095FC00237B7014E703
:106D4000012B08D0032B7FF423AF6388002B7FF443
:106D50001FAF012103E0618800297FF419AFA088EB
:106D6000FFF77AFE00287FF405AF11E702293B60A8
:106D70007FF41BAF5B883360FCE600BFE039002086
:106D80009A3A002094F9000063780028BFF672AFA9
:106D9000002B3FF467AF0A2B7FF4FAAE3B78002B51
:106DA0003FF4F6AE797804297FF462AFB9788A426D
:106DB0007FF45EAF072A96BF5219002392F8BB30CA
:106DC0008CF80030F6E600BF13B5164C237DF3B9FE
:106DD000E268A168019201AB802016F095FA019A51
:106DE000A3681344A360E3689B1AE3606BB962B1C4
:106DF0002369E2889A4208DD94F8C82093FBF2F1F7
:106E000002FB11330BB90123237502B010BD00231F
:106E10001A4619468020237502B0BDE8104003F0E1
:106E200067BC00BFE039002030B585B000230246C2
:106E30000D460193002858D1002935D108220B4670
:106E40000DEB020118F00CFB002804DA802003F09F
:106E5000C1FB05B030BD2A4C029A2260039A6260E1
:106E600004F13802A2609DF90820BDF80E302575A6
:106E7000002AC4E903550ADB802B04D9802003F0E3
:106E8000A9FB0020E3E713B1C4E90333E1E7FFF70F
:106E900077FD0028DAD0E28823699A42D4BFE26005
:106EA000E360FFF791FFD4E7154CD4E90215002DFC
:106EB00001AB04DC18F0D4FA0028CADAC6E72A4687
:106EC00018F0CEFA0028D9DB019AA3681344A36016
:106ED000E3689B1AE360002BBBD104F13803A36085
:106EE000FFF74EFD0028DCD1B0E78028B1D1044B7C
:106EF000DA68002AD5D11B7D002BD2D1A9E700BFCB
:106F0000E0390020054B064A9A62064ADA62064AD0
:106F10001A63064A58629A6100207047E0390020DF
:106F20002D6B000031680000D1680000716800001E
:106F30002DE9F3410446474D47484FF0FF334FF0EA
:106F4000FF320EF011F895F8B830002B7BD16B6A48
:106F500083B142482C62E8616E6A03F0E3FC03F0FF
:106F6000D1FA041E10DA3C480EF076F8204602B042
:106F7000BDE8F08100F0BEF8FFF7C4FF6B6A002B9C
:106F8000E7D14FF0FF34EEE700F01CFB041EEADB14
:106F90007378012B5AD1F379002B57D0002668461D
:106FA00085F8C830ADF802308DF804608DF80060C7
:106FB00003F0ECFA041ED6DB802768468DF80070DB
:106FC00003F0E4FA041ECEDB2549304603F096FCBC
:106FD000041EC8DB2249384603F090FC041EC2DBC5
:106FE000204CDFF8848044451AD3002003F056FB80
:106FF000041EB8DBD5F8C430802043F00103C5F887
:10700000C43003F04BFB041EADDBD5F8C43043F4B1
:107010008033C5F8C430012385F8B8300024A2E7D6
:10702000276A0026227FF3B29A4201D82434DAE795
:1070300007EBC30257F83310107903F05FFC0136F9
:107040000028EFD09DE76FF077048CE76FF0150410
:1070500089E700BFE0390020F8060020AD69000094
:10706000296E0000400900206409002030B51F4B44
:107070008BB005AA03F1100518685968144603C4BB
:107080000833AB422246F7D11B782370102200212F
:1070900001A81DF009FD1222002115481DF004FD74
:1070A000102101A818F037FB00281BDD0828B8BF05
:1070B0000820093801AB0E491A18002012F8013FC8
:1070C0000AAC04EB131403F00F0328336B440130B4
:1070D00014F8144C13F8143C0C7008284B7001F190
:1070E0000201EBD102480BB030BD00BF335E02009D
:1070F0009B6100202DE9F04F724B93F800B087B0F0
:10710000BBF1000F03D0704807B0BDE8F08F6E4CA4
:1071100000264FF0011AB0463546B14623783BB9F8
:107120006A4B02349C42F3D1664A01231370EAE7AA
:107130006378052B1BD8DFE803F08E03C38E1D395F
:10714000402304A88DF810B0ADF812308DF814B0BB
:1071500018F058F940B1082304A8ADF8123018F01F
:1071600051F908B1ADF812B0BDF81230E3712378CF
:107170001C44D3E7E378002BF9D1A3786BB108F175
:1071800001085FFA88F8F2E76B689C4207D0243563
:107190004F4B9D42F8D30020B6E74E4DF8E7AB6861
:1071A000002BECD0414620469847E8E7002DF2D06E
:1071B00000222B7F9A42EED2296AA07801EBC2010D
:1071C0000B79984201D00132F3E70127E07800F013
:1071D00003008DF81400207994F805C040EA0C20D3
:1071E000ADF8120094F902000028FBB228DA07F18A
:1071F00010004FF0010C0CFA00F010EA0A0F26D133
:1072000043F080008DF8100004A8CDE9021301922C
:1072100018F0F8F8DDE90121039BC0B99DF81020B2
:10722000A27012F0800F18BF10330A7118BFDBB2C2
:107230004FF0010214BF9A40BA404AEA020A96E7A8
:107240000120B84010EA0A0F01D11846DAE70137E9
:10725000102FBBD1B7E7032E1AD1FFF707FF074660
:1072600050B1FDF791FF024630B11028A8BF10229F
:107270003946A01C1DF0F0FB23786FF00201E218E4
:10728000091B04EB5303D14213D50136F6B26EE766
:10729000002EF1D1B9F1000F3FF47DAFA4EB09034B
:1072A00089F80230C3F3072389F8033089F8048092
:1072B000EBE702F801BC13F8010902F8020DE2E75E
:1072C000A14654E79A610020600800203F09002091
:1072D000640900204009002010B5094B00211A461E
:1072E0001C78844205D15C681CB1482303FB012053
:1072F00010BD0131042903F14803F1D10020F7E763
:10730000AC3A00202DE9F34150F8303C10F8346CD1
:10731000103304460AD1036950F8282C980736D553
:10732000D2B9590715D5002344F8303C54F8303C05
:1073300010330BD054E9097554F81C8C19F0DDFF9B
:1073400000284FD02E48214619F0A8FF02B0BDE812
:10735000F08143F00403236154F82C1C01AB304648
:1073600015F0D2FF10B16FF01503DDE7019A54F864
:107370002C3C134444F82C3C54F8283C9B1A44F809
:10738000283C54F8243C134444F8243CCEE754F8F9
:107390002C1C01AB304603F027FA0028E3D1019DF5
:1073A00054F82C3C2B4444F82C3C54F8283C5B1BF0
:1073B00044F8283C54F8243C2B4444F8243C002D49
:1073C000B1D0304603F0B4FAB5FBF0F303FB10552F
:1073D000002DA8D154F8283C002BA4D0304603F04F
:1073E0004BFAA3E744F8200CA4F118000DF0B6FE08
:1073F000002DABD0424639463046A847A6E700BF2D
:10740000C01500204B1E012B73B506460D460FD844
:10741000FFF762FF044668B9012D09D101AB0122D3
:107420000DF10301304603F0DFF9019B002BF5D18C
:1074300002B070BD19F061FF04F1340108B1012DF3
:1074400005D1084602B0BDE87040FFF75BBF0348B6
:1074500002B0BDE8704019F021BF00BFC015002088
:107460002DE9F74F804600911746994615F097FF92
:10747000044600285CD1EFF3118B402383F312887C
:10748000BFF36F8F2C4900220846002301910DF0B5
:1074900099FE019968B9DFF8A4A0482262430AEB7B
:1074A00002056E6816F1100F12D108460DF056FE57
:1074B00006E00134042C01F14801E4D16FF00B0621
:1074C0008BF31188BFF36F8F304603B0BDE8F08FA8
:1074D0000AF802800C9A009B6A610D9A2861AA61E1
:1074E00040466FF00F02C5E90237C5F844906A6064
:1074F00003F01EFA58B1404603F01AFAB7FBF0F257
:1075000002FB10771FB16A6C42F004026A6419F042
:10751000020F08D0482202FB04A10948343119F0B7
:10752000BDFE0026CCE7404603F0A6F90646C7E7B5
:107530006FF00F06C8E700BFC83A0020AC3A002041
:10754000C015002010B5EFF31184402383F3128897
:10755000BFF36F8FFFF7C0FE50B14368103307D100
:107560006FF08B03436000F13401044819F096FE7C
:1075700084F31188BFF36F8F10BD00BFC0150020CA
:10758000F8B50E4C04254027EFF3118687F31288D7
:10759000BFF36F8F6368103307D16FF08B03084818
:1075A000636004F1340119F079FE86F31188BFF3AA
:1075B0006F8F013D04F14804E6D1F8BDAC3A0020DC
:1075C000C015002070B50A4C0A4E002531462046F1
:1075D00019F039FE0122A4F118001146013519F005
:1075E000B0FD042D04F14804F0D1002070BD00BFAF
:1075F000E03A0020057300000169012381F84B3057
:107600000B6833B191F849301BB10248083119F0C9
:1076100045BE7047C01500200169012381F84A303A
:107620000B6833B191F848301BB10248083119F0AA
:1076300035BE7047C015002070B50569EFF311869F
:10764000402383F31288BFF36F8FD5F8900015F0B5
:10765000D8FD044686F31188BFF36F8F30B104481C
:107660000022002305F118010DF046FF204670BDF1
:10767000C015002070B5012382F8483013680D460C
:1076800014463BB192F84A3023B10E4802F108018A
:1076900019F004FED4F890301A699B689A4205D11B
:1076A0007DB904F1180140F6CD4204E004F118015F
:1076B000002DF8D00022BDE87040024800230DF0F4
:1076C0001BBF70BDC015002070B504460E46017981
:1076D0001548154615F03FFE10B394F90020637865
:1076E000002A16DB202B04D0222B0ED06FF0850051
:1076F0000AE02B681A6840F8102C9A8820F80C2CA5
:107700009B7900F80A3C002070BD638800F8093CB2
:10771000F9E7212BEAD11038072328603360F2E71C
:107720006FF01200F0E700BFCC3B002008B5014627
:10773000034815F01EFE10B1012300F8073C08BDF8
:10774000CC3B00200D4A03460021A0F848101068E9
:10775000C3F8940090889279A3F8980083F89A204F
:1077600083F89C1083F89B10A3F89E1083F8A01058
:10777000402203F14C001DF097B900BFA85202004F
:10778000F0B5D0F88C305B681B6A1F7D85B004466D
:10779000384615F004FE0646F8B994F88630E3B191
:1077A000A06F4FF4806203A915F04AFD0546A0B111
:1077B0008306A4F1180308BF00F1FF3584F8306098
:1077C0000193074B039900932A4602233846FFF79B
:1077D00047FEA06F294615F053FD05B0F0BD00BF70
:1077E0007576000010B504690023C4F8A8300C4B6E
:1077F000C4F8A400596804F1A80269B9C3E90022D9
:1078000004F10800074919F01EFD04F118000649AB
:1078100019F054FD002010BD0A605A60F0E700BF67
:10782000CC3B0020C9D301008177000030B54FF474
:107830000033426805690D4C85B042F2A100CDE9E4
:107840000103002385F89D30106AADF80C10007913
:107850000A2201A915F058FD95F89D3023B90120A1
:1078600019F0AAFA013CF7D105B030BDA18601009C
:1078700073B504698DF80710002384F8483040255B
:10788000EFF3118685F31288BFF36F8F0122D4F8CE
:1078900090000DF1070115F0B4FC86F31188BFF3D9
:1078A0006F8F01280AD019F028FD10B994F8A13083
:1078B0006BB9094B1A780AB901221A7021220023E8
:1078C00004F1180105480DF017FE02B070BD00214B
:1078D000212019F0C8FDD3E7AD610020C0150020BC
:1078E00037B514460A1E054620DDD4F88C0004F195
:1078F0004C0115F086FC012384F8493023683BB124
:1079000094F84B3023B1114804F1080119F0C6FC7A
:10791000D4F88C104B684A699A1ACB699B1A3F2B92
:1079200004D8012384F8A03003B030BD94F89E3011
:10793000002BF9D0064B009301940123402204F15F
:107940004C012846FFF78CFDEEE700BFC015002074
:10795000E1780000F7B50D4601461D4815F0EFFC33
:10796000044610B30646691E56F8A4395F68052917
:107970001BD8DFE801F01C1A031C222610F8061C95
:1079800099B9012300F8063C3B6A3246187BFFF7A1
:10799000A7FF14F85C2C42B93B6A187D0D4B00938D
:1079A000019602231146FFF75BFD03B0F0BD3046A0
:1079B00003B0BDE8F040FFF7C5BE012304F8053C65
:1079C000F3E710F8053C002BEFD00023F6E700BFEB
:1079D000CC3B00207576000037B5094D09490024DD
:1079E00000944FF0FF334FF4806228460DF046FDBF
:1079F0000549284619F087FC204603B030BD00BF7A
:107A0000C0150020806C0020575E020008B50448B5
:107A100015F048FABDE80840024815F043BA00BF27
:107A2000605E0200965E0200014811F019BA00BFC4
:107A3000D852020038B5044618B90F4B0F485B689E
:107A400098476168B1F5683F10D0B1F5680F0DD067
:107A50000B4DA9420AD011F46861206807D0014695
:107A6000084819F075FA00232360656038BD1422B8
:107A70001DF01AF8F9E700BFAC020020C45E020056
:107A80002C5F5CA9D440002008B520B34368B3F54F
:107A9000683F10D101220368BFF35B8F53E8001FDA
:107AA000002903D143E800200028F7D1BFF35B8F02
:107AB0000DD1002008BD094A93420AD000684FF05A
:107AC000FF324FF0FF330DF04FFA0028F1D0044899
:107AD000F0E70448EEE76FF4E040EBE72C5F5CA9C9
:107AE000E98FFFFFEA8FFFFF08B5D8B14368B3F510
:107AF000683F10D100220368BFF35B8F53E8001F7B
:107B0000012903D143E800200028F7D1BFF35B8FA0
:107B10000BD1002008BD074A934208D000680DF041
:107B20009BFAF6E76FF4E040F4E70348F2E7034816
:107B3000F0E700BF2C5F5CA9E98FFFFFEA8FFFFF32
:107B400010B5044618B91D4B1D485B68984763681B
:107B5000B3F5683F2FD0B3F5680F2CD0194A934284
:107B600019D1236803BB18484FF0FF324FF0FF33A1
:107B700021460DF0CBF908B923681BB90F4B134808
:107B80005B6898472068142200211CF08DFF4FF499
:107B90006863636008E0B3F5683F0DD83A2B03D003
:107BA00040F6BA629342DED1206819F01BFA63688E
:107BB00043F03A03636010BD054AF3E7AC020020CE
:107BC000C45E02002C5F5CA9D4400020EA5E020083
:107BD0003A00003A08B5064906484023142219F035
:107BE000A8F9BDE808400449044811F0FDB900BFF8
:107BF000D43B0020D4400020E0520200F4520200A6
:107C000038B50C46154615F0D5FC034B43F83050FB
:107C100003EBC0035C6038BD7803002030BFFFF782
:107C2000FDBF00BF074A936893F90E10002907DBD8
:107C3000926993421FBF044A536843F080535360D4
:107C4000704700BF0056002000ED00E070B5264BE5
:107C500015469A6A12F0100F9A6A14BF1124102464
:107C600012F0080F9A6A18BF1224920706460AD526
:107C7000586B9A6A140634D519B19A6A22F08002B8
:107C80009A62132401E06FF01500174B9A6A12F004
:107C9000010F9A6A18BF142412F0200F9A6A18BFB5
:107CA0001524D20602D49B6A9B070AD50E4B5B684B
:107CB000190506D5314600F07FFA10B180F3098826
:107CC0000224094B9A6A920642BF5A6A22F4005271
:107CD0005A629A6A42F0FF029A6200232B70204691
:107CE00070BD6FF01500CCE700ED00E0134B9A6A11
:107CF00012F0007F9A6A14BF1E201D2012F0807FB0
:107D00009A6A18BF1F2012F4002F9A6A18BF212008
:107D100012F4802F9A6A18BF222012F4003F9A6A48
:107D200018BF232012F4803F9A6A6FEA02426FEA7A
:107D300012429A6218BF2420704700BF00ED00E095
:107D400010B5194B0246986A9C6A10F4805F14BF04
:107D50001720162014F4006F9C6A18BF1820A40581
:107D600009D5986B986A000404D51AB19A6A22F46E
:107D700000429A6219200C4B9A6A12F4806F9A6A38
:107D800018BF1A20D2050CD49B6A13F4005F18BFE9
:107D90001C20054A936A43F47F43936200230B70CF
:107DA00010BD1B20F5E700BF00ED00E0F0B5484B2B
:107DB0005B688BB00446C3F30803002585F3118884
:107DC000BFF36F8F02F07F40B0F17F4F11D102F00F
:107DD0000C0008280DD010074CBF0C4601250022CE
:107DE000033B8DF80720032B05D8DFE803F024635D
:107DF00067602C46F3E700239DF80720CAB902AE5E
:107E000004F1200720686168324603C20834BC428E
:107E10001646F7D1099A002D54D0C2F3080121B9B2
:107E20006FEA52226FEA4222099202A9184615F01F
:107E3000C2FB0BB0F0BD264BDA6A9107DBD4DA6ADD
:107E4000002AD8DBDA6A5200D5D55A69A16942F412
:107E500080725A61BFF34F8FBFF36F8F5A6931F849
:107E6000021C22F480725A61BFF34F8FBFF36F8FF1
:107E70004DF6027291420AD09A6AD2B24AB10DF11D
:107E8000070201212046FFF7E1FE0346B4E723681D
:107E9000B2E79A6A12F47F4F05D00DF10701012075
:107EA000FFF74EFFF1E79B6AB3F5803FA3D3FFF7DF
:107EB0001DFFEAE70DF107020021E3E70DF10701DD
:107EC0000020EDE722F4FF7222F00102ACE700BFD0
:107ED00000ED00E0044B5A6942F010025A615A6901
:107EE00022F008025A61704700ED00E0EFF30880CD
:107EF000EFF3098101B57246FFF758FF01BD00BFDE
:107F0000002080F31488BFF36F8F0CF071F800200D
:107F100011490860BFF34F8F104880F3088800F0C4
:107F200045F8402080F311880D484FF0AA014FF426
:107F3000307218F074FF0A484FF43071401880F323
:107F40000988EFF314800221084380F31488BFF3FB
:107F50006F8F00F0F9F8000094ED00E0C08700207A
:107F600040800020BFF34F8F0549064BCA6802F4DA
:107F7000E0621343CB60BFF34F8F00BFFDE700BF4C
:107F800000ED00E00400FA050749D1F89020002335
:107F9000C2F307221846934200DB7047C1F89830BD
:107FA000C1F8A0000133F6E700ED00E008B572B6B5
:107FB000002383F31388FFF7E7FF144B4FF0FF32E2
:107FC000C3F88020C3F88420C3F88820C3F88C202D
:107FD000C3F89020C3F89420C3F89820C3F89C20DD
:107FE000C3F88021C3F88421C3F88821C3F88C2109
:107FF000C3F89021C3F89421C3F89821C3F89C21B9
:1080000062B6BFF34F8FBFF36F8F08BD00E100E092
:10801000084B9B6883420BD1EFF3058343B1064BBA
:108020005A6842F080525A605A6A22F400425A62F8
:108030000DF096BE0056002000ED00E012498A685F
:108040004FF030001044EFF3098C80E8F01F40201F
:1080500080F31288BFF36F8F0C4F4FF000668A6970
:108060008A603E60906F0023936780F3118804B5A7
:10807000104600F001F9BDE8044002F1300090E83C
:10808000F01F8CF3098870470056002004ED00E0D3
:108090001EF0040F0CBFEFF30880EFF30980816935
:1080A00011F8021C0229FFD001B5724615F089FAB9
:1080B00001BD00BF40B2002807DB044A410901238B
:1080C00000F01F00834042F82130704700E100E0DB
:1080D00040B200280CDB4309064900F01F002033A2
:1080E0000122824041F82320BFF34F8FBFF36F8FEF
:1080F000704700BF00E100E0054B420900F01F009F
:1081000053F82220012303FA00F01040704700BF0B
:1081100000E100E040B2D30754BF02310021002843
:10812000ACBF00F16040074A4FEA4113ACBF00F515
:10813000614000F00F00DBB2B4BF135480F800338D
:10814000704700BF14ED00E00B4A08B50B4B22F05E
:108150007F029A60BFF34F8FBFF36F8FD3F88820F1
:1081600022F47002C3F888200CF0E0FD0DF02EFF21
:1081700000F058F80CF01CFE0010000000ED00E0CC
:1081800042F8203C009B42F81C3C0A49019B42F803
:10819000183C029B42F8143C21F001014FF080731F
:1081A00042F8043C42F8081C0023203A0265836729
:1081B000704700BFD9CE0100094A0346906870B1EC
:1081C00013F1160F806E05D0A0F140029A4205D837
:1081D000834203D2814228BF0020704700207047AD
:1081E0000056002008B5094B0E461546986000F071
:1081F00043F82C4686F309880020054B9847204613
:10820000002100220023034C204700BF005600201D
:10821000FDD50100D9CE0100014B10221A61704733
:1082200000ED00E0044800234021C2180133302B48
:1082300082F80013F9D1704700E100E008B5EFF3D0
:108240000583064A103B02EBC30152F8330049682C
:108250008847BDE80840FFF7E5BC00BF7803002071
:10826000024B034A0348012100F076B800000420C5
:108270000000002004530200826E054B403A1A6051
:10828000044A4021C3E901121846012100F06EB8EA
:10829000F440002000000B15084AC2F898000B6853
:1082A00023F01F03034343F01003C2F89C308B6894
:1082B00043F00103C2F8A030704700BF00ED00E0BA
:1082C0002DE9F043DFF8608085B00E461F46044676
:1082D0004FF00009B14523DA6068D8B13FB1411EC3
:1082E00008421BD11F2819D92368194216D12368C7
:1082F000019315F0A6F9A36803430393D8F89050AF
:10830000C5F30725D0B2013DA84207D801A9FFF760
:10831000C3FF421C09F101090C34DBE76FF01502C1
:10832000104605B0BDE8F08300ED00E0044B0522E7
:10833000C3F89420BFF34F8FBFF36F8F704700BF18
:1083400000ED00E0BFF35F8F024B0022C3F89420E2
:10835000704700BF00ED00E010B5034C0123227808
:10836000FFF7AEFF207010BDAE61002008B50B4ACC
:1083700000231278FFF7A4FF10F1160F07D0084A68
:108380000021D2F89030C3F30723984200DB08BDE8
:10839000C2F89800C2F8A0100130F2E7AE610020E8
:1083A00000ED00E02DE9F043534B544CD3F89030EE
:1083B0002568C3F307239D4285B000F29A80FFF73A
:1083C000C1FF00200C2685421AD14D4C4D4F25701F
:1083D0006846FEF727FADFF82081DFF82C91064681
:1083E0000025AE4213D1237843490020D1F89020D4
:1083F000C2F30722934276DBFFF798FF002042E0AA
:10840000616806FB0011FFF747FF0130DBE70098CA
:1084100000EB05114FEA051CCB683B40B3F5000F9C
:1084200048D00AD8B3F5001F30D0B3F5800F36D04E
:10843000B3F5801F10D00135D3E7B3F1807F42D070
:10844000B3F1007FF7D150F80C3088684A6815F016
:10845000F8F840F4802009E050F80C3088684A6849
:1084600015F0EFF840F0885040F43020CDE90123BA
:108470000390D8F890302078C3F30723013B98424B
:108480002AD96FF0150005B0BDE8F08350F80C3024
:1084900088684A6815F0D5F840EA0900E6E750F820
:1084A0000C3088684A6815F0CCF840F0007040F451
:1084B0000030DBE750F80C3088684A6815F0C1F8E6
:1084C00040F08270D2E750F80C3088684A6815F0A6
:1084D000B8F840F08870C9E701A9FFF7DDFE2378FE
:1084E00001332370A7E7C1F89830C1F8A000013329
:1084F0007CE74FF0FF30C6E700ED00E010530200CC
:10850000AE6100200000F0FF00000811014B186070
:10851000704700BF98010020F8B5084F06460D4689
:108520000024AC4208DA3B6898470A28305504F129
:10853000010401D00D28F4D12046F8BD940100209B
:10854000F8B50A4F0D46461EC0F10104A3199D421D
:1085500001DC2846F8BD73780A2B02D13B680D2058
:1085600098473B6816F8010F9847EFE798010020FD
:1085700010B5074C2368C2180648C0F1005101F538
:1085800080218A423ABF2260C0184FF0FF3010BDF0
:108590000041002080B2002008B5054814F082FC9C
:1085A000002383F31188BFF36F8F0423184602DF83
:1085B000265F020070B54169857A0C4E044659B1B8
:1085C000437ADB0706D4302303FB05639B6A1B68F1
:1085D0009B6898470023636105EB4505214606EB40
:1085E0000510BDE8704018F0A2BD00BF9007002044
:1085F000827A074B302101FB0233DA6A93F822308A
:108600001B33801A23F00303B0FBF3F0704700BF65
:108610009007002038B5074B827A302404FB0233E0
:108620009B6AD3E901240C601568FFF7E1FF04FBA6
:10863000005038BD900700202DE9F04385B0054675
:108640006846039190461C4618F088FFDDE90067F4
:10865000EFF31189402383F31288BFF36F8F2B8CC4
:10866000002B43D0EA8B9A4225D9002200232846CA
:108670000CF042FD0446F0B189F31188BFF36F8F0F
:10868000039B002B43D032463B46684618F08AFFD6
:10869000A27A274B302101FB023320469B6A1B68DC
:1086A00003A91D68DDE90023A847606180BB20465F
:1086B000FFF780FF26E0298C4B1E2B8489F311885D
:1086C000BFF36F8F95F82230EA8BEC6A1B3323F0EF
:1086D0000303521A02FB0344154B164AEB1A1B11F3
:1086E0005343A37295F82230E372C9E789F31188E6
:1086F000BFF36F8F2346424628460CF0FDFC04462C
:108700000028BDD10024204605B0BDE8F083636198
:10871000012300252381039B6382E27A6560294659
:1087200004F118001CF0C0F963692582E360EAE7F0
:1087300090070020ABAAAAAA70B50C4C302500B94E
:1087400070BD037A4668013BDBB20372002BF7D1A0
:10875000C3604360837A05FB03435B6A13B19847A8
:108760003046ECE7FFF726FFFAE700BF900700204E
:108770000E4A0123C2F840354FF080424FF080513D
:10878000C2F87835D1F83001082808D1D1F8341171
:10879000052904D80648415C09B1C2F838364FF0C3
:1087A00080430122C3F880250020704700E001408B
:1087B0002F5F020020B1034B800143F001031847F3
:1087C000704700BFC05202004FF08043D3F84036DC
:1087D000DB072ED54FF01023D3F8043303F0070343
:1087E000072B26D1144A0123C2F80435D2F80034ED
:1087F000002BFBD04FF01021D1F8043323F00703F6
:1088000043F00403C1F804330023C2F804350A4AD4
:10881000D2F80034002BFBD0BFF34F8F0749084B31
:10882000CA6802F4E0621343CB60BFF34F8F00BF0E
:10883000FDE70020704700BF00E0014000ED00E0D0
:108840000400FA05F7B506460D460D4883688AB25E
:108850001B6831469847002810DA00240CE02F1BD3
:10886000042F28BF042717F05EF93A46019001A9AA
:1088700030191CF0F1F83C44A542F0D803B0F0BD2B
:10888000A050020010B503460548826814688AB2F9
:108890001946A0470028B4BF6FF00400002010BDA7
:1088A000A0500200034B1B6808461A7919681CF097
:1088B000D3B800BF0441002008B5044800F0CAF94D
:1088C00010B1006800B1806808BD00BF4C080020EE
:1088D000F0B50B21054685B014F05CFF0C2128464D
:1088E00014F058FF002D3CD02C6804B1A4681F4B35
:1088F00002930123039304F13807384604F1F0068C
:1089000018F070FB1A49304618F09DFC5DB32B68D7
:1089100003B11033174A2046136014F05DFF0021A5
:10892000084617F09CF91AF08DFBC4E9000505F024
:1089300027FD54F8500B10490EF012FD384614F084
:1089400027FF02AB00934FF4A0626FF007032046AD
:108950000A490CF093FD3146204618F09FFC05B003
:10896000F0BD2C46C3E72B46D4E700BF355F0200BD
:10897000E7D701000441002029D70100C070002082
:1089800038B54FF0FF324FF0FF3305461D4815F064
:1089900065F91D4B1B687BB11A684FF0FF344FF42B
:1089A0007A705BB9631C1BD1184818F093FCBDE8C2
:1089B0003840144815F05BB91A46EEE7D9691B8CAC
:1089C000491B00FB0313002B09DD9C4228BF1C46FA
:1089D0001AB1116813460A46E3E71146FAE7002484
:1089E0004FF4004540F2E73000214FF47A72002343
:1089F000E4FB0501FCF7AEFB02460B4603480CF016
:108A0000D9FDD4E75806002054430020C0160020AA
:108A10002DE9F04F87B01F4603908B46049215F066
:108A20001FF9039B5B68002B00F0A580109A0024BF
:108A300002F00102191D0194A046A24626462046D6
:108A400005922C2202FB04324C4D926A22F07F42A6
:108A500022F47D0222F0FF02AA4246D131F8042C12
:108A6000022A42D18E4648F2FE023EF8045995424F
:108A70003BD00BF1FF3202924A1E94460022029D27
:108A800015F8019F02951CF8015FA94547D10832EE
:108A9000D2B2802AF3D1049DAA4228BF2A463D784B
:108AA000954222D82C2505FB043595F82A506D07F0
:108AB0000BD53F2A09D89BF80050FF2D15D19BF804
:108AC000015005F00F05032D0FD12C2505FB0435B2
:108AD000059E95F82A50C5F3C0059EBB002D08BF22
:108AE00092463A700E4608BF70460134062C01F1DA
:108AF0002C01A6D1109B990729D540B1041D314600
:108B0000204615F06FF810B987F800A026460398A4
:108B1000143015F0ACF8304607B0BDE8F08F89EAA4
:108B2000050515F0800FB6D102F108095FFA89F941
:108B30000132D2B26D009145EDB2ACD015F0800F8C
:108B4000F6D0A8E73A70019288460E46CDE7109B12
:108B5000DA070CD5B8F1000FD9D03146404615F0F0
:108B600041F80028D3D1019B3B704646CFE7109BCC
:108B7000DB05CCD5C1E71E46C9E700BF00010200F6
:108B8000F8B515F037F84FF0FF3306464FF0FF32D7
:108B90001C4815F063F81C490B682BB100221C68B7
:108BA0004FF47A7E17463BB93046FFF7E9FEBDE841
:108BB000F840144815F05BB8DD69188CAD1B0EFB4E
:108BC0000055002D9C460EDC186892B94D6808606F
:108BD000AB4200D1486093F822001F6067F30000A9
:108BE00083F82200944654B1206823466246044626
:108BF000D9E710604868834208BF4A60EBE7204627
:108C0000F3E700BF5806002054430020002808DD89
:108C1000431E054800EB8310044B984228BF0020F8
:108C200070470020704700BFF00700203008002088
:108C3000054B064A934205D0054A1068002808BF34
:108C40001846704700207047F007002030080020C9
:108C50005C43002008B50749074B02468B4202D30C
:108C60000023184608BD184614F068FF8242F8D069
:108C70004033F3E730080020F007002038B5044601
:108C80000D4614F0EDFF0721204614F07DFF20B3C0
:108C9000636843B105B12B60002504F1140014F0A2
:108CA000E6FF284638BD4FF0FF324FF0FF330C4847
:108CB00014F0D4FF0B4BD3F8282242B96360C3F8F9
:108CC000284205B12B60064814F0D1FFE4E70448C0
:108CD00014F0CDFF6FF00205DFE76FF08505DCE7EC
:108CE00058060020184100202DE9F74F1D4DDFF8F0
:108CF00078A080460F464FF02C0B554501D3002439
:108D000026E0284614F0ACFF6C6805F1140924B97C
:108D1000484614F0ACFF4035EFE7211D00260BFB61
:108D2000064393F82A309B0716D531F8043C022BF2
:108D300012D180224046019114F032FF019958B1BE
:108D400007B13D602C23484603FB064414F08FFF17
:108D5000204603B0BDE8F08F0136062E01F12C014C
:108D6000DDD1D5E7F0070020300800202DE9F74FCE
:108D7000234CDFF890A080460D464FF0180B544569
:108D800007D245B12B6833B1A34204D040345445D7
:108D9000F8D3002429E0204614F062FF676804F14C
:108DA000140927B9484614F062FF4034E7E707F595
:108DB000867100260BFB067393F81C31DB0718D570
:108DC00031F8043C022B14D180224046019114F06A
:108DD000E7FE019968B105B12C60182404FB067404
:108DE000484604F5847414F042FF204603B0BDE801
:108DF000F08F0136082E01F11801DBD1D2E700BF58
:108E0000F0070020300800202DE9F04385B0002352
:108E1000044617468DF80F300D46002958D00A88B1
:108E200048F2FE039A4233D00B78FF2B04D14B78E3
:108E300003F00F03022B2BD02946204615F023F810
:108E400060B190F82480FCB100970DF10F03424609
:108E500029462046FFF7DCFD044610E04FF080086D
:108E6000F1E7304600970DF10F0342462946FFF720
:108E7000CFFD4036002818BF04464E45F1D3CCB193
:108E8000204605B0BDE8F083124EDFF84C90F4E7C1
:108E900024B10121204614F0C9FFDDE7FFF7C8FE29
:108EA000012114F0C3FF04460028E9D1094D0A4E00
:108EB000B54204D305B0BDE8F04300F0C3BA0121C8
:108EC000284614F0B3FF04460028D9D14035EFE717
:108ED0000C46D5E7F007002030080020F0B587B039
:108EE0000023019301AB05460F46164614F0C1FE60
:108EF000044618B96FF0150007B0F0BDBFF35B8FE3
:108F00006369BFF35B8F04F11402002BF2D0BFF34F
:108F10005B8F581E52E8001F994204D142E8000CB2
:108F2000BCF1000FF6D1BFF35B8FE7D1012BE3DC7F
:108F300094F82A30022F6FF3410384F82A302CD1A1
:108F40005EB32846019F14F08BFE6B680BB394F858
:108F50002A30DB0714D4124E12484FF0FF334FF083
:108F6000FF3214F07BFE04F11801304614F0BAFD14
:108F7000336813B90C4818F0ADF90A4814F077FEBD
:108F8000012F06D1201D02A914F0C7FD284614F0B8
:108F900008FF05F1140014F06AFE0020ACE700BFE2
:108FA0004C43002058060020901600202DE9FF4178
:108FB00014F020FE0023CDE9023307464FF0FF33C3
:108FC0002F484FF0FF3214F049FE2E4B1C68B4B10D
:108FD0002568DFF8B0804FF0FF36BCB13946204637
:108FE00015F077F968B92146404614F07BFD02A8D8
:108FF00014F06EFD2DB32B682C461D46EDE725467B
:10900000E7E7864228BF0646AC42F3D1731C10D076
:109010004FF4004440F2E73000214FF47A7200230D
:10902000E6FB0401FCF796F802460B4616480CF0E6
:10903000C1FA134814F01BFE029C24B904B0BDE829
:10904000F0812B46D8E7206A14F00AFE94F8253008
:10905000206A6FF3410384F8253001A9FFF70EFE63
:1090600000280BDB206A94F82430019904F11002E7
:1090700014F0A6FF206A143014F0F9FD2468DCE730
:109080005806002044430020601600202DE9F047D8
:1090900014F0B0FD4FF0FF3380464FF0FF322D4803
:1090A00014F0DCFD2C4B1C68002C4DD054F81859E2
:1090B00005B1183D4FF0FF364FF02C090EE009FBCB
:1090C0000317BC4223D109FB0311043114F05CFFE8
:1090D0003DB3AB6903B1183B2C461D4604F1180A99
:1090E0004146504615F0F5F80746A8B951461A48CA
:1090F00014F0F8FC3A465046394615F0CBF81748BC
:10910000174A9042E4D241680023A142DAE70133D2
:10911000062BD4D14030F4E7864228BF0646A5424C
:10912000D6D1731C10D04FF4004440F2E730002138
:109130004FF47A720023E6FB0401FCF70BF80246B9
:109140000B4608480CF036FABDE8F047014814F029
:109150008EBD00BF580600204C430020F0070020C1
:109160003008002090160020F8B54FF0FF33054678
:1091700017460E484FF0FF320E4614F06FFD0C4BB1
:109180001B680BB11C6823B9BDE8F840074814F010
:109190006EBD5B683A463146284698471CB1226846
:1091A00023461446EFE72246FAE700BF58060020A0
:1091B00010410020F0B5002385B0CDE9003304460E
:1091C0000D4600294CD0294B1B68A3B1C96B95F8FB
:1091D000406081B1062E0ED80DF10A0318463246C2
:1091E0008DF809601BF038FC95F8413000908DF83F
:1091F00004608DF80530092120466F6914F0C4FC25
:1092000080B30D21204614F0BFFC38B94FF0FF3277
:109210004FF0FF3304F1280014F020FD204614F035
:109220008DFC29464368204698470D210646204676
:1092300014F0AAFC18B904F1280014F018FD002E4F
:1092400002DA284615F0E3FA1FB13146384614F029
:1092500084FC009B23B1324669462046FFF784FF19
:1092600005B0F0BD6FF07206EBE700BF10410020C3
:109270002DE9F0410D460646F8B1F1B10846FBF77D
:1092800083FF08281CD8114FDFF84480441C474551
:1092900008D32246294606F108001BF0DDFB00201A
:1092A000BDE8F081B74206D02246294607F1080002
:1092B0001BF0C2FB38B14037E9E76FF01500EFE76C
:1092C0006FF05A00ECE76FF07700E9E7F007002055
:1092D000300800202DE9F0433E483F4C3F4DDFF879
:1092E0000081404E85B04FF0FF324FF0FF3314F055
:1092F000B5FC15F0A4FD2746AC422BD33A4B3B4AB4
:10930000DB1B9B09AA4288BF0023EBB138493948CF
:10931000394C17F0D3FF3949394817F0CFFF4FF4D4
:10932000A073A4F82432204647F23053C4F8183210
:1093300014F015FE3349C4F81C02334817F0BEFF81
:10934000324B0022C3E90022224805B0BDE8F043B9
:1093500014F08DBC0022C4E902222274204614F0CD
:10936000F2FBD0F80890B9F1000F18D0D9F800300E
:10937000ABB10721204614F04AFC04F1140017F0A9
:1093800031FE04F1280017F02DFED9F800302046F8
:10939000984794F83C3023F0030384F83C30237A58
:1093A0008BB9204614F0CAFB80450ED1184A1368C9
:1093B000591C1160174A092101A813F080FD01A969
:1093C0002046FFF755FF403496E733685A1C326059
:1093D000114AF0E758060020F0070020300800206E
:1093E0004C080020084100206F080020B107002031
:1093F0008D9000009016002018410020AD8F0000D5
:1094000060160020818B0000C0160020544300200D
:109410000C410020405F0200495F020038B5074C54
:10942000074DAC4200D338BD0321204614F0ACFBFD
:1094300010B9204614F0FCFE4034F2E7F00700209B
:1094400030080020004870473C53020002484FF0AB
:10945000FF32012117F075BE60430020014601482C
:1094600015F0BAB9C007002073B5054616461C466C
:1094700017F043FF08B10026344601A932462346BF
:1094800028460BF043FD0146A8B9019C6022204606
:109490001BF00AFBFF2284F84F20084A6560012375
:1094A0009542236308BF84F85C30204615F002FA29
:1094B000204602B070BD0024FAE700BFC0050020BE
:1094C00002460B460148FFF7CFBF00BFC005002092
:1094D0002DE9F743DDE90A450646174698468946D1
:1094E00029B923B990F8473013F0700F46D017F020
:1094F00004FF08B100240025304615F0AFF996F8B6
:109500004730002846D113F0700FC3F3021243D046
:10951000022A0CBF28220022B8F1110F32D10832E2
:1095200009EB0201C3F30212B36913B11B6803B163
:109530001B8B022A32D1B3F5A06F38BF4FF4A06362
:10954000CDE900451B1A994228BF19467568164B8C
:10955000164C17483A46A54208BF184615F04EF873
:109560000146E8B1304615F0ABF93FB1B068394675
:109570000C3014F0BCF8304615F09CF9002003B014
:10958000BDE8F083B8F1010F02D0B8F13A0FC7D1AE
:109590000432C5E70022C3E70246C1E70B46CFE726
:1095A0006FF00B00EBE700BFC0070020C0050020F4
:1095B0009007002030B585B0DDE908450093CDE97E
:1095C000024513460A460146024815F0C2F905B0A5
:1095D00030BD00BFC005002030B585B0DDE90845CD
:1095E0000093CDE9024513460A460146024815F0AC
:1095F000B0F905B030BD00BFA0050020024BA82285
:1096000000FB023017F088BDF01600200828024B3E
:1096100028BF0020185C70474F5F020010B588B06B
:109620000F4C204617F06BFD4FF0FF324FF0FF3329
:10963000CDE906230023CDE90323CDE90133094910
:10964000094B00944FF4A07204F120000CF004F8D0
:1096500020B108B0BDE810400CF056BB08B010BDFA
:10966000F0160020007600201FEE01002DE9F341E6
:109670000746884616464FF0FF3315484FF0FF3235
:109680000BF072FC134B1C686FF0010534B91048E5
:109690000BF0E2FC284602B0BDE8F081227C337872
:1096A0009A4213D1637C72789A4200D073B9A3684E
:1096B00013B1BA69934209D1E368009365683346F0
:1096C000424639462046A847051EE0DB2468DDE710
:1096D0006C06002078430020F8B50F4616461D465C
:1096E0000446D0B1CBB1142200211BF0DDF9656036
:1096F000277466744FF0FF324FF0FF3308480BF0C9
:1097000033FC084B1A6822605A681C6002B95C601E
:1097100003480BF0A1FC0020F8BD6FF01500FBE73B
:109720006C0600207843002002460B4601480BF0EF
:109730001BBC00BF3006002001480BF08DBC00BFF1
:10974000300600202DE9F04F89B0CDE9052390F8CF
:109750004730C3F302130393013B012B05460E462A
:1097600000F2A080112A134601BF069B1B681A88CD
:10977000049208BFB3F802A0039B1CBF4FF0000A7D
:10978000CDF810A0022B3AD1086800210830FFF76D
:10979000ABFA34680746102204F1180104F10800FE
:1097A0001BF04AF900B117B1049B9A457AD094F89E
:1097B0001880A8F1FF04D4F1000848EB04084FF02A
:1097C000FF304FF0FF31FFF7AFFF544B4FF0000B6E
:1097D0001C684FF0FF330793D9469CB9B9F1000FCD
:1097E00074D1FFF7A9FFB8F1000F00F08A80BBF138
:1097F000000F57D0284615F00AF8002053E04FF02C
:109800000008DCE7A36B93BB94F84230002B3BD1FC
:10981000B4F84030059A934234D1E38813B1049AE6
:1098200093422FD1E38B0BB153452BD194F8437066
:10983000B90706D50123221D3146284615F01BFB2A
:1098400000B37A0707D5002304F11C0231462846ED
:1098500015F011FBB0B1079B07F07807BB4211DA96
:10986000B8F1000F14D13BB20793A1460AE0B3F858
:1098700076201005C8D5AF6993F97800FFF7C6F9CF
:109880008742C1D02468A8E7039A9A42C0D0F9E77A
:1098900040F6CD420023284615F060FA074628B965
:1098A000FFF74AFF022009B0BDE8F08FE36B009399
:1098B0000146069BD4F834C032462046E0470228D1
:1098C00002D1384614F0A3FFC346DBE7D9F8344091
:1098D000D9F83C70FFF730FFB8F1000F0FD0BBF1A3
:1098E000000F87D1002CDDD0069B00973246294619
:1098F0004846A047831E584258414000D3E7002CF9
:10990000F2D195F84730C3F30213022BCAD10023DA
:1099100004220121284615F082FBC3E78043002082
:109920000B4A002310B5C2E900330A4A1846114613
:1099300014460133042B086002F1480202D00846A5
:109940001146F6E7044B054AC3E9002410BD00BFE9
:10995000804300209043002088430020684400207A
:10996000024B034800228021FFF7B6BE3BEF010007
:10997000B04400202DE9F04F28238DB00026CDE91A
:10998000066308AB0A9308230B93836903938368E8
:10999000044688464BB906A9204615F01DFA05462F
:1099A00038B902200DB0BDE8F08F1A8A5B68164402
:1099B000F0E787887FBABFB22837B742F1DC03DA15
:1099C0003946204615F043F9AB6833B9EB6823B943
:1099D0002B6913B96B69002BE3D02B7AFF2BE0D0F6
:1099E00005F118060021304615F01FFC0028D8D1DB
:1099F000B8F1000F7BD02B786A781B0143EA121371
:109A0000DAB2C3F3850343EA821384F85030AB79AA
:109A100084F84F300023A4F84A30282384F84630D5
:109A2000A368DB68DB7984F8493094F84730022278
:109A300062F3061384F847302B7EFF2B00F08E80F4
:109A40000398314614F082F90028AAD02B7EFF2B10
:109A500000F084800799204614F0B3FF95F8069033
:109A6000B9F12C0F00F0A18000F29780B9F1000F3E
:109A700000F09D80A9F12B08D8F1000646EB0806FE
:109A8000B6004FF006084FF0000AB9F13A0FA4F8FB
:109A90004C8000F02081B9F1110F00F01C81B9F168
:109AA000060F00F01881B9F13B0F3FF47AAF204662
:109AB00015F0DEF8012280460DF10B01204615F06D
:109AC0006CF800287FF46DAF9DF80B302C2B00F064
:109AD000CC806ED82BB12B2B03D0112B6FD0062B43
:109AE0006DD0204615F0C4F80122431EEEE030464A
:109AF00015F08AFB00287FF454AF05F108084046B2
:109B000015F082FB00287FF44CAF0121304615F0A0
:109B10008CFB00287FF445AFFFF794FC01463046EC
:109B200015F08FFB68B10521304615F07EFB00284B
:109B30007FF437AF0821304615F077FB00287FF41B
:109B400030AF00214046FFF7CFF800283FF453AF75
:109B500090F92930002B3FF44EAF22E70121304627
:109B600015F063FB00287FF475AF0221304615F035
:109B70005CFB30B16749304615F063FB00287FF489
:109B800069AF03A93046FFF7F1F800283FF409AFA9
:109B9000037D98073FF55EAF03E7A9F13C0CDCF1CC
:109BA000000646EB0C0676006BE7082669E70126FF
:109BB00067E73C2B5FD1B10751D446F00206B9F1FB
:109BC000000F02D0B9F13C0F8BD10023012205A96F
:109BD00020461FFA87FB8DF8143014F0DEFF0028B2
:109BE0007FF4DFAE9DF814300133BBEBC30F4FEAB7
:109BF000C309FFF4D6AEA9F103034FF0020B0193A2
:109C0000204615F035F80122009004A9204614F0F2
:109C1000C4FF00287FF4C5AE9DF810208ABB9DF8D4
:109C20001020B2B3012A9DF8141037D0019B8B424B
:109C30007FF7B7AE02F0C002802A45D0C02A3FD0DD
:109C4000002A7FF4AEAE204614F0BBFE00287FF45D
:109C5000A8AE9DF8142002320BEB02031BE0720643
:109C60003FF53FAF46F04006A9E733073FF539AF70
:109C700046F00806A3E7A3F13B02012A9FD93A2B3D
:109C80002EE7012205A9204614F087FF0028C6D040
:109C900087E60BF101031FFA83FB07E08A1C0BEB3D
:109CA000020320461FFA83FB14F08BFED945A7D888
:109CB000D1441FFA89FA5FFA88F89DF80B90E4E620
:109CC0002B7EFF2B3FF46DAE009B02220421204629
:109CD00015F0A5F965E6B9F1110FA4F84AA008D06E
:109CE000B9F13A0F7FF45DAE2946204615F062FACD
:109CF00058E60AA9204600F057F8049000283FF4DF
:109D000050AE04AB4A4605A920460595FFF71AFD5B
:109D100048E600BF6C530200F0B585B008230393FA
:109D200090F847301E4A1F4FCDF808D0C3F30213F6
:109D30000E4602A90446022B08BF174615F04CF840
:109D4000054650B3A26800231ABBB4F84A1094F831
:109D500046200A449B1A5BBAAB80A069394614F0CE
:109D600063FA00B97EB11121204614F061FB4FF671
:109D7000FF73002818BF0346EB8094F8483043F087
:109D8000080384F8483002A9204615F043F805B0CE
:109D9000F0BD118A52680B44D6E76FF06800F6E711
:109DA0000004400001004000F8B590F847301C4A1C
:109DB0001C4EC3F3021304460F46022B08BF16467F
:109DC00015F00AF8054610B900252846F8BD3946B1
:109DD000204615F01FF803460028F5D1AA88A1688F
:109DE00052BA92B2B9B994F84610B4F84A00014494
:109DF0005B1A9A42E8D1A069314614F017FA00289C
:109E0000E3D0EB88002BDFD01121204614F010FBAB
:109E10000028DAD0D8E7088A49680344E2E700BF9F
:109E20000004400001004000020600F07F0312D54C
:109E3000082B05D1010700F00F0306D50E48704727
:109E400010F0780F12D100F00F034C2000EB4310FC
:109E50000A4B18447047082B05D1020700F00F0386
:109E600006D50748704710F0780FF6D000207047ED
:109E7000044800EB4310704710460020C444002003
:109E800030470020304600200149024817F006BA4A
:109E9000EC440020981700200146014817F03CB917
:109EA000740700200248002200230BF025B900BFF0
:109EB0007407002013B5124800F0C4FE114B9842FD
:109EC0001AD111480AF0FCFD002410480AF03EFEA9
:109ED0000F49104800944FF0FF334FF480620BF0AD
:109EE000CDFA0D490B4817F00EFA0C480C4917F043
:109EF000AAF9204602B010BD6FF00400FAE700BFD7
:109F000009A100000000AD0B655F02007C53020058
:109F10008077002098170020575F0200EC44002053
:109F200025A2000010B50E49BFF35B8F002351E856
:109F3000002F012A03D141E800300028F7D1BFF3F8
:109F40005B8F0CD151F8044C1439204613F0DDF826
:109F5000783004D12046BDE8104013F0B2B810BDEF
:109F6000E444002038B5002464F07F00C0B2FFF75D
:109F70005BFF013415F02FFA082CF5D10E4D0024AB
:109F8000E0B2FFF751FF036903B90561013415F031
:109F900022FA082C05F14005F2D1084815F01BFA09
:109FA000074BD3F87C2212B9064AC3F87C22064834
:109FB00015F011FA002038BD544B00201046002047
:109FC000C4440020544700203047002010B5054C01
:109FD000FFF768FF20B14168204616F0B9FFF7E7A8
:109FE00010BD00BF8005002007B500230E480022E9
:109FF00001A90AF08BFF90B1FFF7E8FF0A480022A1
:10A00000002301A90AF082FF38B9019804234060B7
:10A010000374FFF741FFFFF737FF002001E00198CD
:10A02000406003B05DF804FB80050020022810B5F5
:10A0300011D8094B1C5CFFF7D7FF60B100220274F6
:10A040000472FFF729FF054B93F824301BB1BDE8DC
:10A050001040FFF719BF10BD625F0200C44400202A
:10A06000F8B5877806463846FFF7DEFE3B06F578FA
:10A07000044612D5002D43D1FFF7B6FF0346002852
:10A080003ED00122A5770274032202739C60FFF781
:10A0900003FFBDE8F840FFF7F7BE4DB1012D2FD10A
:10A0A000FFF7A2FF034658B3657705740573EDE724
:10A0B000FFF79AFF20B3B278124B12F0800F02F034
:10A0C000080111D041B1D3F8A836E360012303742D
:10A0D000022303738460DAE702F00F02142101FB0C
:10A0E0000233D3F80836F0E711B1D3F8A837ECE71C
:10A0F00002F00F02142101FB0233D3F80837E4E722
:10A10000F8BD00BF00700240F0B5064689B01422C9
:10A11000002103A81AF0C8FC3378013B052B21D895
:10A12000DFE803F07A0314146A1603238DF8143061
:10A130000024FFF759FF0346A0B1047400F10802A0
:10A14000DDE9050182E8030018461DE00423EDE780
:10A15000B7783846FFF768FE837A044623B1013B9F
:10A16000022B43D909B0F0BD3B06F57813D5002D7D
:10A17000F8D1FFF739FF03460028F3D00122A57775
:10A180000274032202739C60FFF786FE09B0BDE8EB
:10A19000F040FFF779BE55B1012DE3D1FFF724FF61
:10A1A00003460028DED0657705740573EBE7FFF7FB
:10A1B0001BFF07460028D5D0012303740223037335
:10A1C000846004F10C01B07815F066F9134AE16877
:10A1D000B2F88C328B4206D95B1AA2F88C3201F0AD
:10A1E0007FF83846D0E7A2F88C52FAE7304609B03B
:10A1F000BDE8F040FFF734BF01A801F04FF89DF82B
:10A200000530052B04D19DF8043013F0600FA9D060
:10A21000034B059301248CE702248AE7C444002001
:10A22000304600202DE9F043A64CDFF89C9285B023
:10A230008046FFF737FE074610B905B0BDE8F0834A
:10A2400094F825303A7C3BB9002A00F08680796882
:10A250009D4816F07DFEECE7042A42D8DFE812F0B4
:10A260007D0005000001160140013B7BBD68032B0A
:10A2700037D8DFE803F0023D5A5F6E69934B002246
:10A2800032607260D3F880143170D3F88414717026
:10A29000D3F88814D3F88C0441EA00217180D3F8F4
:10A2A0009014D3F8940441EA0021B180D3F89814B3
:10A2B000D3F89C3441EA0323F3800823EB60306831
:10A2C0007168834B03C311462B68687A984796F9E7
:10A2D0000030002B08DBF38833B1A4F88C3200F097
:10A2E000FFFF79684846B4E70023A4F88C32F8E70A
:10A2F0006B7F002BF5D02B7F002BF2D000266E77E2
:10A300004FF0FF3273482E774FF0FF3315F076F899
:10A310006B6901936B68CDE9023601A9687A00F098
:10A32000E7FC6C4815F06CF8DBE72B680121687AD4
:10A330009847D6E7AB7A6BB9EB7F5BB965484FF0CE
:10A34000FF324FF0FF3315F059F800F0CFFF6148AE
:10A3500015F056F82B680221E9E73A7A042AC0D8AA
:10A36000DFE802F059032367730000F02BFC054679
:10A370000028B6D100F066FBBFF35B8F564901237E
:10A3800051E8002F002A03D141E800300028F7D11E
:10A39000BFF35B8FA5D141F8085C41F8105CE06920
:10A3A0006361143912F036FE9BE7002565F07F00EB
:10A3B000C0B2FFF739FD037A13B1407A01F0FAF821
:10A3C0000135082DF2D194F854311BB194F85501A0
:10A3D00001F0F0F80025E8B2FFF726FD037A13B18B
:10A3E000407A01F0E7F80135082DF4D194F8743281
:10A3F0001BB194F8750201F0DDF8002000F0C6FBF7
:10A40000012384F825302368002B3FF46AAF002134
:10A410000220984765E7002584F8255001F030F8C0
:10A42000FFF780FD2368002B3FF45BAF2946042033
:10A43000EFE7002B3FF455AF00F0CEFB2368002B75
:10A440003FF44FAF00210520E3E72268002A3FF4E4
:10A4500048AF002B3FF445AF00210620904740E76E
:10A4600008F110054FF0FF334FF0FF32284614F08B
:10A47000C5FFFFF777FD284614F0C2FF58F8283CC7
:10A48000002B3FF42EAF00210120C2E794F8743274
:10A490007BB1012584F8895284F88852FFF7A4FD26
:10A4A00038B10E4A057405738260FFF7F5FCFFF7BB
:10A4B000EBFC58F8283C002B3FF413AF00210A2096
:10A4C000A7E700BFC44400208005002000700240C0
:10A4D000C8440020FC440020E44400203047002011
:10A4E00016F05CFC00F0CCFF00F0A2FAFFF76EFD66
:10A4F000FFF738FD16F04BFC014800F0A3FBF0E637
:10A5000009A1000038B5164D95F824402CBB05F183
:10A51000380016F067FD204601F09AF92246012125
:10A52000E8612720FDF7F6FD16F031FCFFF71AFD74
:10A53000044610B9012385F824300A4B1B680BB17F
:10A54000FFF7A2FC4FF08043D3F83834DB0702D585
:10A550000020FFF76BFD204638BD0024FBE700BF5D
:10A56000C444002074070020074B93F824203AB11C
:10A5700093F82530002B14BF00206FF012007047B5
:10A580006FF01200704700BFC444002038B5104B74
:10A5900093F824300446C3B105782846FFF744FCFD
:10A5A00010B96FF0150038BD457223798372638846
:10A5B00043602078618810F0080F02D14B1E0B42D7
:10A5C000EFD114F064FF0020EDE76FF01200EAE72E
:10A5D000C444002038B5124B93F824200546CAB174
:10A5E00093F82530B3B1FFF71FFC0446A8B1837A76
:10A5F000012B12D007D9023B012B07D96369A36154
:10A600000020E06038BD00F077FEF7E7284600F054
:10A6100019FEF3E76FF01200F4E76FF01500F1E7B1
:10A62000C444002038B50E4B93F82420054682B16F
:10A6300093F825306BB1FFF7F7FB68B115F008040C
:10A640000AD1284600F020FE284600F0EBFF204605
:10A6500038BD6FF01200FBE76FF01500F8E700BFA0
:10A66000C444002038B50C4B93F8242005460C4612
:10A6700062B193F825304BB1FFF7D6FB48B144B136
:10A68000284600F0E7FD2070002038BD6FF0120072
:10A69000FBE76FF01500F8E7C444002070B5134ED7
:10A6A00096F824300446C3B1FFF7BEFB0546B8B1A7
:10A6B000230705D4204600F0E7FD204600F0B2FF56
:10A6C0002B7A83B901232B7296F825300BB9002021
:10A6D00070BD204600F06EFFF9E76FF01200F7E75B
:10A6E0006FF01500F4E76FF07700F1E7C444002045
:10A6F0002DE9F043DFF8E4801E4698F8243085B059
:10A70000074689461546002B61D098F82530002B66
:10A710005DD003065ED5FFF787FB0446002859D0BD
:10A72000037A002B56D04FF0FF334FF0FF3208F181
:10A73000380014F063FEA37F4BB108F1380014F029
:10A740005FFE6FF00A04204605B0BDE8F083A37AEF
:10A75000C5B13BB30123A3774FF0000801A93846E8
:10A76000CDE90195CDF80C8000F0C2FA1C4B98425F
:10A7700029D084F81E801EBB6FF00404194814F021
:10A780003FFEE0E7E27F02B1E577002BE2D100F087
:10A79000B9FD8742DED000F0A9FD124814F030FE6A
:10A7A0000024D0E7B8F80A30AB42F0D96268B5FBB4
:10A7B000F2F302FB1353002BE9D10123E377E6E721
:10A7C000C6F80080D8E706B135600024D6E76FF000
:10A7D0001204B8E76FF01504B5E700BFC4440020C9
:10A7E0000000AD0BFC4400202DE9F0411D46204B3C
:10A7F000174693F824200E46002A33D093F82530CC
:10A8000083B3030631D401B97FBBFFF70DFB0446C8
:10A8100058B3037A4BB34FF0FF3316484FF0FF3273
:10A8200014F0ECFDE368BB42984628BFB84646B931
:10A830003FB905B12B600F4814F0E2FD0020BDE8E0
:10A84000F081A169424630461AF006F9A3694344F3
:10A85000A361E368A3EB0803E360002DEBD0C5F828
:10A860000080E8E76FF01200E9E76FF01500E6E717
:10A87000C4440020FC44002070B51E4D95F82420EF
:10A88000034682B395F825206AB31B062ED4FFF742
:10A89000CBFA044650B3037A43B34FF0FF334FF083
:10A8A000FF3205F1380014F0A9FDE368B3B90126C1
:10A8B00063692677A361637F83B1FFF795FB30B9A6
:10A8C00005F1380014F09CFD6FF00B0070BD0674AC
:10A8D00084600673FFF7E0FAFFF7D6FA064814F033
:10A8E0008FFD0020F2E76FF01200EFE76FF0150028
:10A8F000ECE700BFC4440020FC44002010B5084B26
:10A9000093F824300C462BB1FFF78EFA28B104607F
:10A91000002010BD6FF01200FBE76FF01500F8E7A4
:10A92000C4440020014B1860704700BFC44400209D
:10A9300008B5074B93F8243023B1FFF775FA20B11F
:10A94000406808BD6FF01200FBE76FF01500F8E7F4
:10A95000C44400204FF08053D3F83021082A06D198
:10A96000D3F83431052B04D8034AD05C704700205B
:10A9700070470120704700BF665F0200064B10F071
:10A98000800FA3F1D80208BF134600F00F00182271
:10A9900002FB0030704700BF6C4E0020EFF31180C7
:10A9A000402383F31288BFF36F8F0A4BD3F8001C48
:10A9B000032261B949F27531C3F8001CC3F8142DA4
:10A9C000C3F8001C80F31188BFF36F8F7047C3F882
:10A9D000142DF7E700E00640EFF31180402383F3E6
:10A9E0001288BFF36F8F0A4BD3F8001C61B949F28C
:10A9F0007532C3F8002CC3F8141DC3F8002C80F383
:10AA00001188BFF36F8F70470022C3F8142DF6E74B
:10AA100000E006404FF08053D3F83031082B02BFDE
:10AA2000024B0022C3F81C2C704700BF007002408C
:10AA3000024A00231360024A137070474C4F0020F3
:10AA4000B361002008B54A4B4FF40062C3F80024FC
:10AA5000FFF780FF08B1FFF7A1FF4FF08053D3F855
:10AA60003031082B18D1EFF31180402383F3128883
:10AA7000BFF36F8F3F4BD3F8001CC02200296ED16B
:10AA800049F27531C3F8001CC3F8142CC3F8001C3C
:10AA900080F31188BFF36F8F354B0122C3F8002577
:10AAA000D3F800241205FBD54FF40062C3F800244C
:10AAB0004FF08053D3F83031082B17D1EFF31180CA
:10AAC000402383F31288BFF36F8F2A4BD3F8001C07
:10AAD000002947D149F27532C3F8002CC3F8141C81
:10AAE000C3F8002C80F31188BFF36F8FFFF732FF9C
:10AAF00030B1FFF771FFFFF72DFF08B1FFF74EFFF1
:10AB00004FF08053D3F83031082B194B0AD140F263
:10AB1000E372C3F800284022C3F80428BFF36F8F04
:10AB2000BFF34F8F8022C3F81C250122C3F83025C4
:10AB3000114B40F2FF121A60104B00211960104BAC
:10AB40001970FFF767FF0F4B19700F4B02221A7035
:10AB5000FFF700FF50B1BDE80840FFF73DBFC3F865
:10AB6000142C95E70022C3F8142CBBE708BD00BFE6
:10AB70000070024000E00640484F0020444F002093
:10AB8000AF610020B1610020B3610020094B0022B9
:10AB900010B51A70084A094B094C002808BF134623
:10ABA000C4F800332720FDF785FA0123C4F80435E3
:10ABB00010BD00BFB2610020FDFFDF01FDFFFF01FE
:10ABC00000700240034B1878012894BF0020012038
:10ABD000704700BFB361002010B54FF0FF324FF057
:10ABE000FF3315480AF0EEFAEFF31181402383F3A7
:10ABF0001288BFF36F8F114B1B7803F0FF0483B1F2
:10AC00000F4BD3F8002412F400720AD10120C3F8CC
:10AC10002C05D3F82C05D3F80004800502D5C3F821
:10AC20002C25002481F31188BFF36F8F02480AF0AE
:10AC300095FA204610BD00BF0C070020B26100202D
:10AC400000700240F8B51C4B1C7894BB1B4A106086
:10AC500001221A7040F2FF17264664F07F0514F0B7
:10AC6000080FEDB214BF39464021284614F00FFCFE
:10AC70002846FFF783FE0134092C867506730661AA
:10AC8000EBD1002440F2FF17254614F0080FE6B27E
:10AC900014BF39464021304614F0F9FB3046FFF727
:10ACA0006DFE0134092C857505730561EDD10448ED
:10ACB000F8BD0448FCE700BFB36100204C4F002002
:10ACC0000000AD0B0500AD0B084B10F0800F00F03D
:10ACD0000F0114BFD3F81025D3F8142501238B409E
:10ACE000134214BF01200020704700BF00700240D3
:10ACF0002DE9F8430246EFF31187402383F31288CE
:10AD0000BFF36F8F030703D1184B1B78834229D100
:10AD1000174B184E1C683568104614F0B0FBE4431E
:10AD2000A4B24FF001092C4309FA00F814EA080410
:10AD30001AD11046FFF722FE80F80C90034607C98F
:10AD40001C6183E807009C750B4B0C4845EA08051D
:10AD500080223560C3F8042187F31188BFF36F8F19
:10AD6000BDE8F8830648F7E70648F5E7B16100203B
:10AD7000484F0020444F002000E100E00000AD0BF0
:10AD80000A00AD0B0B00AD0B10F0080F074B06D0FF
:10AD9000D3F8C00410F4803F18BF0020704700F0C3
:10ADA0000F0000F5947053F82000704700700240C7
:10ADB0002DE9F74FAB4BAC4ED3F85421DAB100225A
:10ADC000C3F85421D3F80413890214D58DF8042054
:10ADD000D3F82025ADF80620D3F8C034002B336813
:10ADE00014BF4FF001224FF48072134333609F4B26
:10ADF00001A81B6898479B4BD3F8604134B10022EF
:10AE0000C3F86021D3F86C44C3F86C44D3F828210C
:10AE10004AB10022C3F82821954B187814F02FFB73
:10AE2000012383401C43DFF84C82934F98F8005075
:10AE300098F9009015F0080143D1B9F1000F05F021
:10AE40000F032EDA8D4A52F8230020B342F8231064
:10AE50001422534303F1804303F51C33D3F808361F
:10AE6000874A117803F001034B401370FFF7D2FDBE
:10AE700084480AF073F92846FFF780FD837D032B91
:10AE800037D1284614F0FBFA012303FA00F03B689F
:10AE900023EA00033B60DFF8D4A101254FF0060947
:10AEA0005DE0794A52F823000028F4D042F82310DC
:10AEB0001422534303F1804303F51C33D3F80837BE
:10AEC000CEE7B9F1000F674B09DBD3F85021002A18
:10AED000E1D00022C3F85021D3F8A837C0E7D3F857
:10AEE0002C21002AD7D00022C3F82C21D3F8A83671
:10AEF000B6E7037BDBB9284614F0C1FA012303FA55
:10AF000000F03B68B9F1000F23EA00033B6001DA6F
:10AF1000882DC0D106238DF8043000238DF807302A
:10AF2000524B8DF806501B6801A89847B3E7002DD7
:10AF3000B1D14C4B0122DA64ADE794FAA4F0326847
:10AF4000B0FA80F005FA00F31A430F28326024EAC1
:10AF500003043A6840F39C80134200F0A980002C5F
:10AF6000EBD1404BD3F800215AB1C3F80041474B15
:10AF70001C703F4B1C70012301933C4B01A81B68C4
:10AF80009847384BD3F85821002A2ED00022C3F816
:10AF90005821D3F80044C3F80044E30508D53B4BDF
:10AFA00001221A7002230193304B01A81B689847B5
:10AFB000A50508D5354B00221A70032301932B4BAE
:10AFC00001A81B68984760050FD5304B1A7862B10D
:10AFD00000221A70234B0122C3F808259A65042326
:10AFE0000193224B01A81B6898471E4BD3F85C3194
:10AFF00003B3244B9B681BB998F80030590619D04D
:10B00000184B0022C3F85C21D3F88034184A23F08F
:10B010007F0313703B6823F001133B60336823F414
:10B02000803343F001033360052301930F4B01A8E4
:10B030001B6898473A6833681A4200F0EB80114861
:10B04000002200230AF0BEF8002840F0E380054B00
:10B05000D3F82C35002B7BD00A4803B0BDE8F04F65
:10B060000AF07CB800700240484F00204C4F00208E
:10B07000B1610020B0610020444F002008710240FF
:10B08000AF6100200C07002030710240B261002047
:10B0900013407FF464AF60F07F018DF804908DF869
:10B0A00006108DF80730DAF8003001A8984756E707
:10B0B000A0F110018DF804908DF806108DF807505E
:10B0C000F1E749F080052846FFF758FC4368B0F8DF
:10B0D00014A001689A4528BF9A4601F06043B3F175
:10B0E000005F044604D05448524619F0B5FC52495A
:10B0F0002268636852442260A268A3EB0A03D20765
:10B1000068B2636053D5BAF1000F52D100232373A4
:10B110004FE011464FF0000A604545D1003B18BF93
:10B120000123002A42D0504540D9012303FA09F3F4
:10B130002BEA03033B6006238DF804303F4B8DF868
:10B14000065002221B68A2758DF8072001A89847B7
:10B15000D7F800B033681BEA03093FF47DAF19F05C
:10B16000012314BF93FAA3F999FAA9F9B9FA89F955
:10B17000B9F10F0FA5D9A9F11005EDB22846FFF7D7
:10B18000FDFB04462846FFF7FFFD6368B4F814C0D2
:10B1900022689842BDD81B1A00EB020E114663606C
:10B1A000C4F800E08246B7E70023BAE768B2002B94
:10B1B000ACD04FF08053D3F83031082B02BF204B76
:10B1C0008222C3F81C2C336888F80050012202FA4E
:10B1D00009F923EA09033360236915F0080F534482
:10B1E0002361174B19D1002805F00F054FF014000B
:10B1F00000FB0530A9BF0A3503EB8503C0F8001733
:10B20000C0F804A7AFBF43F82520C0F80016C0F867
:10B2100004A65A6003B0BDE8F08F0028B5BFC3F89C
:10B22000A016C3F8A017C3F8A4A6C3F8A4A7B4BF78
:10B230005A629A64EEE700BF544D00204C4F002044
:10B2400000700240024B40F48070C3F8180570474C
:10B2500000700240030713D400F00F0310F0800FBA
:10B26000084A0BBF03F5887303F5847302EB83026E
:10B2700052F8230008BF5068003818BF01207047FB
:10B280000020704700700240034BC3F80C0540F4E7
:10B290008070C3F80C057047007002400023036003
:10B2A00043600E4BD3F880240270D3F8842442709C
:10B2B000D3F88824D3F88C1442EA01224280D3F8D0
:10B2C0009024D3F8941442EA01228280D3F898247F
:10B2D000D3F89C3442EA0323C380704700700240D5
:10B2E000014B0122DA64704700700240014B0122D9
:10B2F0001A65704700700240014B01225A65704781
:10B3000000700240014B1878704700BFB161002007
:10B3100010B50246EFF31184402383F31288BFF384
:10B320006F8F14F0ACF80B49012303FA00F00B689F
:10B3300023EA00030B6012F0080101BF02F00F02C4
:10B34000054B02F5947243F8221084F31188BFF381
:10B350006F8F10BD484F002000700240F7B50146C6
:10B36000EFF31185402383F31288BFF36F8FFFF74C
:10B3700005FB0646084614F082F8012211F0800F02
:10B3800002FA00F22D4818D1036832EA03040AD009
:10B390000846FFF7BDFF0323B37585F31188BFF39C
:10B3A0006F8F03B0F0BD2649347323EA02030360B4
:10B3B0000B6823EA02030B60EDE70B0715D4802925
:10B3C000204B2FD001F00F0404F2DA346400C3F8EC
:10B3D0000048D3F80448D3F80478E4B244F00204F7
:10B3E0003C43C3F80448D3F80438154F04683B685D
:10B3F00064EA030C1CEA020FCFD013433B60002326
:10B4000033730323B3758DF807300F4B8DF8061097
:10B4100024EA0204062204601B688DF8042001A8B7
:10B420009847BAE740F2B474C3F80048D3F8044828
:10B43000D3F80478E4B244F00404D1E7444F002088
:10B44000484F0020007002404C4F002038B50446A1
:10B45000094D4FF0FF324FF0FF33284609F0B2FE9E
:10B460002046FFF77BFF284609F078FE034B802239
:10B47000C3F8042138BD00BF0C07002000E100E044
:10B48000F8B54FF0FF324FF0FF332B4809F09AFE2A
:10B490002A4B8022C3F884212720FCF72DFE98B187
:10B4A000274E284B34681B68240C24041C430127B6
:10B4B00064BB254D40F2FF1333602720C5F80445D7
:10B4C000FCF706FEC5F80043204A13788BB11E4BEB
:10B4D0000021C3F808110121C3F80026C3F804169F
:10B4E0005960D3F808110029FBD00021C3F80811D6
:10B4F0001170154B0022C3F80025FFF78BFA0E4898
:10B5000009F02CFE124B01221A70F8BD94FAA4F532
:10B51000B5FA85F50F2D2846C6BFA5F11000C0B2BB
:10B5200040F08000030701D4FFF718FF07FA05F584
:10B5300024EA0504BCE700BF0C07002000E100E09E
:10B54000484F0020444F002000700240AF610020AF
:10B55000B361002010B504464FF0FF324FF0FF33C7
:10B56000114809F02FFE2046FFF7F8FE04F00F0205
:10B57000012393400D4A14F0800F14BFD2F8101528
:10B58000D2F814156FEA030315BF0B400B40C2F845
:10B590001035C2F81435044809F0E0FD044B802250
:10B5A000C3F8042110BD00BF0C070020007002404A
:10B5B00000E100E070B50446FFF786FB68B904F0CF
:10B5C0000F02012514F0800F144B05FA02F205D08A
:10B5D000D3F810150A43C3F8102570BDD3F814151D
:10B5E0000A43C3F81425631E062BF6D8EFF3118621
:10B5F000402383F31288BFF36F8F2046FFF788FE46
:10B60000204613F03CFF064A1368854023EA0503F1
:10B61000136086F31188BFF36F8FDEE7007002407E
:10B62000444F0020030610B5044605D4FFF712FE70
:10B6300010B12046FFF76CFE014BC3F8184510BD52
:10B640000070024070B50D460649411A0446491182
:10B650000548402213F03FFF2B4601462046BDE837
:10B6600070401847644F00203C50020037B50C462C
:10B670000A490B4A411A40230093491105462346C3
:10B68000084813F054FF011E05DA2846234603B08C
:10B69000BDE83040184703B030BD00BF644F002004
:10B6A00099F501003C50020010B5EFF311844023DE
:10B6B00083F31288BFF36F8F074A136823F00201E8
:10B6C000DB07116002D4012014F092FA84F3118890
:10B6D000BFF36F8F10BD00BFBC4F0020002270B5BC
:10B6E000012104461046FCF715FD0F4801F060FDEE
:10B6F0000E4B984215D114F080FA26690C49304659
:10B7000011F075FC00280BDB0125B564246908499C
:10B7100004F1200011F06BFC002801DB65650020BE
:10B7200070BD6FF00400FBE735B800000000AD0B02
:10B73000805302007FB500220123CDE9022304AB30
:10B74000CDE90433094ACDF800D06B46CDF804D0DA
:10B7500013F01BFF002805DB4FF4804200236846EE
:10B7600009F030FD07B05DF804FB00BFB1F5010042
:10B7700030B4104B0C2202FB003301460020D3E909
:10B7800010521864EFF31180402484F31288BFF341
:10B790006F8F9C6C04F0C00444F002049C6480F33E
:10B7A0001188BFF36F8F1DB12B46034830BC18477B
:10B7B00030BC7047644F00203C50020010B4EFF3DF
:10B7C0001182402383F31288BFF36F8F17480168FB
:10B7D00041F002040460C80707D482F31188BFF364
:10B7E0006F8F012010BC01F0D3BC4FF08041D1F825
:10B7F0000C04D1F80C14C907EFD5EFF3118083F3D3
:10B800001288BFF36F8F0A498B6C03F0C00343F0BB
:10B8100002038B6480F31188BFF36F8F82F311886A
:10B82000BFF36F8F002010BCFFF7A2BFBC4F0020FA
:10B83000644F002010B1012804D07047034B9B6C6B
:10B840005B0701D1FFF794BF704700BF644F002032
:10B85000024BC0B203EB4010704700BF644F0020A2
:10B860002DE9F0413849BFF35B8F0746012251E8CB
:10B87000003F41E800200028F9D1BFF35B8F33B9C6
:10B88000324933484B60CB608A6011F0C3FB7B1EAA
:10B89000012B2BD8012F07D14FF08043D3F81C3454
:10B8A00003F00303012B21D015F027FD0546F8B95D
:10B8B000284B1B78E3B14FF080430222C3F80823E2
:10B8C0000646DFF894804FF08044D4F81824D4F86A
:10B8D0001834D20315D503F00303012B01D0012F37
:10B8E0000FD155B386F31188BFF36F8FBDE8F08198
:10B8F000EFF31186402383F31288BFF36F8F012586
:10B90000DFE7ADB1304611F08DFED4F81835002BCD
:10B91000DBD1D4F80421002AD7D0C4F80431D4F8FC
:10B9200004310123C4F81835C8F88031A360CCE78E
:10B930000021212015F097FDE7E74FF08043022218
:10B94000C3F80423D2E700BF604F0020504F00200F
:10B95000844F00203B6C002000E100E008B5074860
:10B9600015F02FFA38B10648FCF7D0FD0448FAF775
:10B97000F1F9002008BD6FF01200FBE778500200DB
:10B9800085B900000A2838B5074D044604D1AB68D4
:10B990000D215B6828469847AB6803485B68E1B2B5
:10B9A0009847204638BD00BF78500200EFF311825F
:10B9B000402383F31288BFF36F8F0A4BD3F8001133
:10B9C00061B10021D3F80805C3F80011D3F80031A4
:10B9D000C0B282F31188BFF36F8F70476FF00A0017
:10B9E000F7E700BF00D00040F0B5034610469C7852
:10B9F00093F803C0EFF31182402585F31288BFF35B
:10BA00006F8F1F7893F801E0E41B04EA0C04A04256
:10BA100088BFA0B23E180CEA06063D461E7082F3AF
:10BA20001188BFF36F8F0A188A4216D177450CD15F
:10BA3000EFF31182402181F31288BFF36F8F1978E1
:10BA4000597082F31188BFF36F8F1B79241AA342B8
:10BA500022BF064B01221A60F0BD5E1901357679CE
:10BA600001F8016B05EA0C05DEE700BF00D00040DD
:10BA7000DB432DE9F04713F001050E46144604D0D0
:10BA80002248FFF7B1FFBDE8F0879AB3EFF31188C2
:10BA9000402383F31288BFF36F8F0D20FCF72CFB3C
:10BAA00007460D20FCF714FB88F31188BFF36F8F56
:10BAB000DFF85CA0DFF85C80CAF80051DAF80031EA
:10BAC0004FF400590123CAF800302546C8F8809188
:10BAD000DAF8003183B1FFF769FF031EC8F88091DF
:10BAE000F6DB013DADB27355002DF1D117B10D203C
:10BAF000FCF7E0FA2046C6E7EFF31180402383F31A
:10BB00001288BFF36F8F11F08DFDE1E7F04F002039
:10BB100000D0004000E100E02DE9F041124F0D4659
:10BB2000144607F1450814B92046BDE8F0814FF0EE
:10BB3000FF334FF0FF32384609F044FB22462946D6
:10BB40004046FFF751FF0646384609F007FB3EB96D
:10BB50004FF0FF324FF0FF33044809F033FBE6E7C4
:10BB6000A41BA4B23544DEE7C04F0020D84F00200C
:10BB700038B5194C01221146204615F0E2FA01228F
:10BB8000002104F1180015F0DCFA40F20743A4F894
:10BB900048304FF0706323630C2384F83430002561
:10BBA0000E4B84F84550A4F84650D3F8042522F0F3
:10BBB0000102C3F804250121C3F80051D3F8002184
:10BBC000C3F804132A4619600D20FCF7A3FA0D20D0
:10BBD000FCF770FA284638BDC04F002000D0004066
:10BBE00010B5FFF7E3FE002820DB174B93F8322057
:10BBF00093F8314093F83310141B31EA0404C0B2B7
:10BC00000DD193F8472093F8464093F84810141B41
:10BC100031EA04040BD10D4B01225A600EE09C184E
:10BC20000132114084F8350083F8321010BD9C18A1
:10BC30000132114084F84A0083F847100448BDE8F7
:10BC4000104009F08BBA00BFC04F002000D0004068
:10BC5000D84F0020024B0B6001231360704700BFD8
:10BC60001450002000487047A453020010B5012270
:10BC700011460748074C15F064FA01F0E3FA15F095
:10BC800076F8206015F06FF86060002010BD00BFEE
:10BC90001C500020145000204FF08042D2F81015A4
:10BCA000D2F8103501F01E0123F01F030B4343F0BF
:10BCB0000103C2F81035024B00221A70704700BF12
:10BCC000B46100204FF08053D3F83031082B20D1DD
:10BCD0004FF08042D2F81015CB071AD5D2F81035A4
:10BCE00001F01E0123F01F030B43C2F81035D2F8F8
:10BCF00008315BB1D2F8103523F01F030B4343F03A
:10BD00000103C2F810356FF08B007047024B01221F
:10BD10001A700020704700BFB4610020F8B50446D7
:10BD200015F021F8237B05460BB113F075FF134F77
:10BD30000026FFF7C7FFE8B9606808F093FEA36824
:10BD40005B1BA36063682B4463603B780BB1FFF718
:10BD5000A3FF237B01363BB9A368002BE9D1A06880
:10BD6000003818BF0120F8BD304601F0E7FA00287E
:10BD7000F2D0F4E76FF08B00F5E700BFB46100206C
:10BD8000F0B587B00E46154614F0EDFF294607467C
:10BD9000304613F046FCC8B3B6FBF7F307FB13635A
:10BDA000A3BBB5FBF7F407FB14547CBBBD4222D305
:10BDB0004FF0FF324FF0FF33164809F003FA13F04B
:10BDC0001FFF02AB01461022C0B12146184618F0F1
:10BDD0006BFE01228DF814200F4ACDE900200F4898
:10BDE000CDE9036501F036FA684601F039FA0446F8
:10BDF000084809F0B3F9204607B0F0BD184618F01E
:10BE000053FECDE90365FFF789FFF0E76FF01504F6
:10BE1000F1E700BF1C5000201DBD0000645E010062
:10BE200070B5037B04460BB113F0F6FE194E0125E5
:10BE3000A368032B06D8184AD2F80034DB07FBD5D9
:10BE4000002070BDFFF73EFF08BB236860681968DB
:10BE500008F028FE33780BB1FFF71EFF6368043348
:10BE60006360236804332360A368043BA360237BDF
:10BE70000135002BDCD0284601F060FA0028D7D02D
:10BE8000054AD2F80034D907FBD50120D9E76FF075
:10BE90008B00D6E7B461002000E0014070B50D468C
:10BEA00086B01946284616461C4613F0BAFB60B306
:10BEB00045EA04039B0728D1FCB14FF0FF334FF054
:10BEC000FF32134809F07EF913F09AFE0346CDE9DC
:10BED000026502A804949BB101238DF814300D4B28
:10BEE000CDE9003041F64C5001F0B4F9684601F05C
:10BEF000B7F90446064809F031F9204606B070BD8E
:10BF00008DF81430FFF78CFFF3E76FF01504F4E7BA
:10BF10001C50002021BE0000F0B54068057B01F0F8
:10BF20001F0444EA4514056987B0002D64D0B2F5BA
:10BF3000001F00F1100506D12146284614F00BFF22
:10BF4000002007B0F0BD01AE0027B2F5800F0197C9
:10BF5000776039D1B3F1007F14BF052304238DF836
:10BF600004300023CDE904630393836823FA01F1CD
:10BF700011F001011AD1B2F1A07F17D104F01F0313
:10BF8000620903F5E0732AD0012A3BD11F4A52F817
:10BF90002330DB070AD40DF103063246214628463A
:10BFA00008F0BAFB1A4B98421CD0029603AA21460D
:10BFB000284608F073FA174B984220D101222146F7
:10BFC000284608F00DFCBBE7B3F1C06F05D0B3F114
:10BFD000007F14BF01230223C1E70323BFE74FF013
:10BFE000A042D4E73146284608F0F4FB094B9842BA
:10BFF000DBD06FF00B00A4E76FF08500A1E76FF0D6
:10C0000015009EE751F82330FFDE00BF000300500B
:10C010000400AD0B0000AD0B38B545682B69B3B11A
:10C020001035284608F0C6FB044680B9014628466C
:10C0300008F08CFB084B98420BD108492246284651
:10C0400008F064FB224605210620FCF763F8002077
:10C0500038BD6FF00400FBE70000AD0B61C00000CD
:10C06000420970B5034602D0012A17D070BD0D4EAB
:10C07000326951680029F9D003F01F0301250C68CB
:10C080009D400029F2D08A682A4002D04B68304691
:10C0900098472CB1236821461C46F2E7024EE7E799
:10C0A0002346F8E764500200505002002DE9F043A7
:10C0B000466840F20635D006337B87B002EA0505B4
:10C0C00054BFC2F34010032001F01F07B5F5837F72
:10C0D000144647EA43178DF8030045D00FD8062DC4
:10C0E00018D007D8B5B1022D40D06FF0150007B0B9
:10C0F000BDE8F083B5F5807FF7D101250AE040F275
:10C100000222954234D0B5F5407F33D0B5F5007F9B
:10C11000EBD102250123220303FA01F12CD5736828
:10C12000C3F80815326982BB07F01F037F0929D0C5
:10C13000012F77D13E4A02EB830284F48033D2F898
:10C140000017C3F30043C4F3404444EA430421F41A
:10C15000E16144EA800421F0070144EA05230B432E
:10C16000C2F800370020C2E70725D3E70425D1E74E
:10C170000525CFE70325CDE7630344BF7368C3F804
:10C180000C15CFE74FF0A042D5E710360DF10202B3
:10C190003946304608F0C0FA14F4403F80460CD1CE
:10C1A0003946304614F0D5FD224B9845DAD19DF83A
:10C1B0000210304608F008FBD4E701AB4FF000094D
:10C1C00003AA39463046CDE90439CDE90199CDF8C5
:10C1D0000C9008F063F9174B984286D114F40033A1
:10C1E00015D09DF803308DF80E3084F48034C4F3FC
:10C1F00000444B4603AA394630468DF80C508DF862
:10C200000D4008F005FA0B4B9842CDD06DE7CDE913
:10C21000043303AA0DF1030339463046039308F0B3
:10C220003DF9F0E703F5E07352F82330FFDE00BF7D
:10C23000000300500000AD0B014BB3F8C00670477F
:10C24000C00E0020024B002083F8C416704700BFC8
:10C25000C00E002038B50B4DD5F8B84664B94FF480
:10C260007A704843C5F8B82613F010FE38B9C5F8FF
:10C27000B8066FF00F0038BD6FF07700FBE720467F
:10C28000F9E700BFC00E002008B5064B93F9C406BD
:10C2900013F0B6FD13F0C6FD00280CBF6FF00400CC
:10C2A000002008BDC00E002010B5044613F0B2FDFA
:10C2B00038B1054BD3F8BC361BB100220221204611
:10C2C0009847002010BD00BFC00E002021B10129F9
:10C2D00006D06FF001007047012313600020704703
:10C2E000004BFAE71C5402002DE9F04114468AB0D5
:10C2F0000C2914D8DFE811F00D001F0036003A00B9
:10C300003E00430065006900DE00F500D2006D00CC
:10C31000F900137843B1507820B1012802D06FF0B2
:10C32000150005E013F0CFFD207813F0DCFD0020B0
:10C330000AB0BDE8F08153791179106833B113F078
:10C34000D4FD0028F3D16FF00B00F1E730B113F00A
:10C35000D5FD0028EBD16FF00100E9E7084613F0A6
:10C36000D0FDE4E7107813F0ACFDE0E7107813F0AF
:10C37000A4FDDCE7634B1268C3F8BC26D7E7156859
:10C3800013F0DFFD05F110040026503554F8103C81
:10C39000002BCCD01034A542C9D0049314F8173C1C
:10C3A0008DF8143054F8143C0896CDE9063614F88C
:10C3B000183C04A883F001038DF8243013F0BFFD6E
:10C3C000E4E7106813F0B7FDB1E7106813F0B5FDAE
:10C3D000ADE7937A43B10121002013F082FD0121E2
:10C3E000084613F07EFDA2E7B2F808804FF6FF730F
:10C3F000984535D053689BB304A9ADF8088003F184
:10C4000008020F4612F8010D01F8010B9A42F9D10A
:10C41000266816B135786B060ED14FF6FE73984537
:10C4200004D00122002102A813F059FD0122114677
:10C43000384613F054FD7AE77278334B02F07F02EE
:10C44000520019889B78ADF80C1052EAD5128DF87D
:10C450000E3008D1032203A9B01C18F0EDFA20B168
:10C460006FF0850064E71A2AFAD14FF6FE739845FB
:10C4700009D0012205F07F030092023332460021E9
:10C4800002A813F022FD22681378012103F07F0334
:10C4900000910233384613F018FD48E74FF47A72E2
:10C4A0000023D4E90001F8F705FE15F029F913F08F
:10C4B0004CFD3CE7167CD4E902014FF47A7200236C
:10C4C000F8F7F8FD4FF47A7205460023D4E900012D
:10C4D000F8F7F0FD002300932A46334613F0D4FC0E
:10C4E00025E7108813F02FFD21E7107813F0E7FC03
:10C4F0002378044A82F8C536002B7FF418AF13F076
:10C5000089FC14E7C00E0020D15F0200034B1868BD
:10C5100010B1006800B10068704700BFC00E002075
:10C5200070B5054688B04668046904F5886014F063
:10C53000E6FD0122002104F5C06014F002FE012294
:10C54000002104F2E45014F0FCFD02F0CFFA13F0E5
:10C55000E4FC82B2D301110101F4016103F48073A0
:10C5600012020B4302F48062134343F49553144ABE
:10C5700043F00F03A2F8C036012384F8C5363368B0
:10C580002846984704F5707600220023CDE906235B
:10C5900000256FF00D03CDE90335CDE90155094BB9
:10C5A00000944FF4487204F14001304609F054F809
:10C5B0000549304614F0A7FE284608B070BD00BFFC
:10C5C000C00E0020615B0000D55F02002DE9F04144
:10C5D0008C46184C0746DDE9060100232646D4F8B0
:10C5E0006484B8F1000F06D00133102B04F1180455
:10C5F000F5D1BDE8F08118245C433519C5F86474A1
:10C6000085F871C485F870243A7815F06FF805F54F
:10C610008D63C3E90001B6F8E035A5F8723404F57E
:10C620008C61A6F8E08531440348BDE8F04114F080
:10C6300073BD00BFC00E00200013002073B5044678
:10C64000FFF764FF1C4D0A46064659B9082C09D16C
:10C6500095F8C53653B3D5F8BC360BB102219847CF
:10C66000002316E0013C072C22D801A353F824F044
:10C6700061C60000B5C6000091C60000B1C600004A
:10C68000B1C60000B1C60000B1C6000061C600001E
:10C6900002238DF807300023A5F8E035D5F8BC3625
:10C6A00023B10DF1070201213046984702B070BD59
:10C6B0000323EEE70123ECE7C00E00204378054A90
:10C6C000C3F3001382F8E0354378C3F3C00382F864
:10C6D000E1357047C00E002010B5154B002283F8DD
:10C6E00098260A7883F8C2264A7883F8C3268A688F
:10C6F000C3F8A4268AB191F90D0083F8B106887BAE
:10C7000083F8B006D1E9040150EA010403F5D664C8
:10C7100008D10022002344E902230648BDE8104066
:10C7200008F01CBD127814F0E1FF44E90201F4E7BF
:10C73000C00E0020C0140020064880F89816137818
:10C7400080F8C236537880F8C33600F5C06008F030
:10C7500005BD00BFC00E0020034B83F8FC0503F2AB
:10C76000E45008F0FBBC00BFC00E002003480023CB
:10C7700080F8FC3500F2E45008F0F0BCC00E002058
:10C7800010B5084BD3F8B846024654B10021C3F89F
:10C79000B816FFF7BBFE234692F90010BDE8104023
:10C7A000184710BDC00E002010B5074BD3F8B826AF
:10C7B0004AB10021C3F8B816FFF7A8FE47F6FF718B
:10C7C000BDE81040104710BDC00E0020036803F004
:10C7D0001F025B09026004D0012B034818BF002030
:10C7E00070474FF0A0407047000300502DE9F04F14
:10C7F000DFF86091DFF860A185B01546834600EB55
:10C80000810140F2FF18594503D1002005B0BDE871
:10C81000F08FDBF800305804C3F3C322C3F30804DD
:10C8200000F191801B0E19F80270444508BF4FF0CB
:10C83000FF34192B00F28A80DFE803F00D141A1D73
:10C8400020261D8888888836638888888888888814
:10C850008888667C7F82C5F80C45621C5ED10BF12E
:10C86000040BD0E7C5F81445631CF8D000265FE040
:10C87000C5F80845F1E7C5F81045F5E7661CC5F8A9
:10C880000845ECD0002604E0601CC5F80C45E6D055
:10C89000012603A80394FFF799FF039B012202FAE4
:10C8A00003F3C0F80C3508E0C5F80845002FDBD1CC
:10C8B000631CD4D0002632460627DBF800300193F3
:10C8C00003F40040002818BF002203A8009218BFFC
:10C8D00001260394FFF77AFF039C019B009A00EB6B
:10C8E0008400C3F3412CD0F800473B0243EA8C0399
:10C8F000134304EA0A04234343EA4603C0F800371B
:10C90000ADE7C5F80C45D1E7C5F86045621CDBF81A
:10C910000030A4D0C3F30043002BB9D003A8039484
:10C92000FFF754FF039B012606FA03F3C0F808350E
:10C930003246C2E7C5F86445E8E7C5F86845E5E76B
:10C94000C5F86C45E2E76FF015005FE76FF0850012
:10C950005CE700BFE85F0200F0F8FCFF2DE9F04162
:10C96000044647680D4614F0C8FC4FF0400888B9EB
:10C97000264B1B7873B16426606813F00FF8F0B98A
:10C98000012014F05CF9013EF6D10021212014F0C1
:10C990006AFDF0E7EFF31186314688F31288BFF3A2
:10C9A0006F8F606812F0FAFFA8B986F31188BFF3A1
:10C9B0006F8FEFE786F31188BFF36F8FE5E7EFF333
:10C9C0001186314688F31288BFF36F8F606812F0CA
:10C9D000E5FF0028EED0BB691D706368BA691B686B
:10C9E0000020C3F844250122C3F84825C3F82001DC
:10C9F000D3F82041C3F85801D3F858019A6081F365
:10CA00001188BFF36F8FBDE8F08100BF3B6C002041
:10CA1000F7B50546002201210220FBF77BFB02202F
:10CA2000FBF748FB6A6811681369C1F82435137D68
:10CA3000507D927D03431343C1F86C356E68D6E98F
:10CA4000004313F0010348D02F6907F10C0014F0E4
:10CA500002F9304B98425AD1387B04F10C0204F5AC
:10CA6000907114F0EEF8387B012707FA00F007F018
:10CA7000E7FB0823C4F80035B369C4F84435002344
:10CA8000C4F84835A760D4F85831002BFBD00021FA
:10CA9000C4F800156B68DC6801AA204612F0C7FED6
:10CAA000002805DB019B226819791868FFF79EFEB4
:10CAB0006A6813680821C3F80015117A51B9D26960
:10CAC000C3F834250122C3F83825C3F81011D3F870
:10CAD00010111A60002003B0F0BD0822C4F8002530
:10CAE000B269C4F84425C4F848350123A360D4F8DA
:10CAF0002031002BFBD00023C4F82031D4F82031A2
:10CB00000123E3604FF48073C4F80433BBE76FF094
:10CB10000400E0E70000AD0B70B5012383400E4A2E
:10CB2000BFF35B8FDC4352E8001F01EA040542E8D3
:10CB30000056002EF7D1BFF35B8F4FF48032824056
:10CB40000648C0F80823BFF35F8FBFF36F8F0B4217
:10CB500014BF0120002070BD54500020001001407F
:10CB600070B40E49D1E90034D01AC31844F100045E
:10CB700022F07F46C1E90034A6F50013B3F5400F5B
:10CB800009D2074B1B681A0A1B069C19054B42F178
:10CB90000005C3E9004570BC09F0D8BA801900202F
:10CBA000585000208819002011B3BFF35B8F012378
:10CBB000104A834052E800CF4CEA030C42E800C11F
:10CBC0000029F7D1BFF35B8F0B4A4FF480338340CA
:10CBD000C2F80433094BBFF35B8F1B68BFF35B8F55
:10CBE000C340DB0742BF064B4FF40032C3F80021BD
:10CBF000704700BF54500020001001404C500020EE
:10CC000000E100E0C3B202489B001844704700BF37
:10CC100040110140D0B50446FFF77EFF124B01469C
:10CC200003EB04134FF0FF364FF0FF372046C3E904
:10CC3000026712F050FF0D4A4FF48033A340C2F850
:10CC400048330123A3400A4ABFF35B8FDB4352E81A
:10CC5000006F1E4042E80064002CF8D1BFF35B8FE8
:10CC6000BDE8D040FFF7A0BF4019002000100140F0
:10CC70004C5000200D4B1868010A0006BFF35F8F6F
:10CC80000B4BD3F80435181841F10001B3F5801FA0
:10CC90000AD2084BD3E90023904271EB030303D27D
:10CCA00010F1807041F10001704700BF5850002022
:10CCB00000100140881900202DE9F04F85B016467C
:10CCC0001F469DF840A00446FFF726FF0190FFF79E
:10CCD000D1FFB04271EB070354D23E4B301A67EBE1
:10CCE0000101984271F100014FD23B4B03EB041359
:10CCF000D3E902239F4208BF96425ED037494FF4E2
:10CD0000803804F1500508FA04F8AD00C1F84883F2
:10CD10002046ADB212F0DFFE26F07F4B05F18045D4
:10CD200004F5A87305F58835DC464FF00309029336
:10CD3000029A2CF07F4341F82230C1F84483D1F8A5
:10CD40000435274A6FF00200C01A604420F07F408B
:10CD5000904232D9286868B1D1F804350393A3EB27
:10CD60000B0020F07F40B0F5000F26D9204612F0CE
:10CD7000B2FE039BBAF1000F07D109EB030C09F1D6
:10CD80000109D5E7BAF1000F09D06FF0150520466B
:10CD90000199FFF709FF284605B0BDE8F08F012390
:10CDA000104ABFF35B8FA34052E8000F184342E8DC
:10CDB00000010029F8D1BFF35B8F07490E982301CA
:10CDC00001EB0412C8500F9B5360C2E902670025B3
:10CDD000DDE700BF01008000401900200010014085
:10CDE000FDFF7F004C5000207FB5264C264BC4F839
:10CDF0000833C4F84833254B00254FF0FF304FF07F
:10CE0000FF314FF48032C4F808554FF48026C3E94F
:10CE10000201C4F804234FF40032C3E90601C4F848
:10CE20000423C3E90A01C4F80463C3E90E014FF403
:10CE30000023C4F80433164B02260121C4F804630E
:10CE40001120C3F880212A46FBF764F91120FBF773
:10CE500031F90123A36023600E4B0F221A600E4BA1
:10CE60000E221A600D4B0E4A0093CDE901550023A6
:10CE70002846FFF721FF3046FEF7F2FC284604B0B3
:10CE800070BD00BF0010014003000F0040190020DA
:10CE900000E100E0545000205050002061CB000021
:10CEA000FFFF7F002DE9F04F354ED6F804339A0787
:10CEB00087B00BD5D6F8043143B1324A0023C6F807
:10CEC0000431D6F804311368013313602E4DDFF8B6
:10CED000BCA00024A9464FF48038D6F8042308FAF1
:10CEE00004F7174228D0BFF35B8F0122A240284BE2
:10CEF000D24353E8001F01EA020043E8000CBCF1F2
:10CF0000000FF6D1BFF35B8F21FA04F2D30702D4EE
:10CF10005AF8242082B1204612F0DDFDFFF7AAFE68
:10CF2000EFF3108B72B609EB041CDCE9022390428C
:10CF3000994109D28BF310880134042C05F11005B6
:10CF4000CBD107B0BDE8F08FCDE90423D5E90013BC
:10CF50004FF0FF32039300204FF0FF332860CCE9FD
:10CF600002232046C6F8487312F0B5FD8BF31088F3
:10CF70000029E1D0039B0093DDE904238847DBE728
:10CF8000001001405850002040190020401101407D
:10CF90004C5000200F4B70B501241868B0B1BFF39E
:10CFA0005B8FB0FA80F0C0F11F0004FA00F1C943B2
:10CFB00053E8002F02EA010543E80056002EF7D19E
:10CFC000BFF35B8FC240D207E7D570BD6FF00B0097
:10CFD000FBE700BF5050002030B5431C124C85B019
:10CFE00005D08442A8BF0446012CB8BF0124FFF736
:10CFF00041FE0E4B0C4DD3E90013401AB0F5000F63
:10D0000010D22218AA4228BF2A4652184FF0000018
:10D0100007490091CDE9010043F10003FFF74CFE01
:10D0200005B030BD2A46F0E7FFFF7F0080190020E1
:10D0300061CB000008B5FFF71DFE024B1B68C01A4C
:10D0400008BD00BF8019002010B5084C01236360A3
:10D050001120FBF73DF8064BC4F80833C4F84833F9
:10D06000044B4FF40032C3F8802110BD0010014082
:10D0700003000F0000E100E002460B46014807F004
:10D0800073BF00BF80060020014807F0E5BF00BF66
:10D090008006002008B50A46014607480FF002FF47
:10D0A00006480FF0FFFE002383F31188BFF36F8F54
:10D0B0000323184602DF08BDFE5F02002D5F020059
:10D0C00037B53223ADF80430154A00230125192164
:10D0D00068468DF80630ADF800508DF80230F7F74D
:10D0E000EBFA0446C0B94FF4AF60F5F739F80D48D4
:10D0F0002946F8F7AEF9044670B901462A460820D9
:10D10000FBF708F82A4621460B20FBF703F82A46CE
:10D1100021462846FAF7FEFF204603B030BD00BF87
:10D1200095D000005C5000200149024814F0B6B8C8
:10D130008C5000209019002037B50D4D0D4900246A
:10D1400000946FF00F034FF40072284608F096F930
:10D150000949284614F0D7F80849094814F073F82B
:10D16000224604211920FAF7D5FF204603B030BD2E
:10D1700090190020C07B00201360020067FB0100B3
:10D180008C500020014B00201B6818479C50002049
:10D1900020B1012806D10448F4F756BF034B012003
:10D1A0001B681847704700BF85D100009C500020C5
:10D1B000014B1860014870479C5000200000AD0BE7
:10D1C00010B51D48BFF35B8F0368BFF35B8F23B9B6
:10D1D000062904D8042923D839B1002010BD072915
:10D1E000FBD1403807F0BAFFF7E750F8203CA0F138
:10D1F0004004D3E900209047012805D00223E063D2
:10D2000084F834300D48E9E747F2305323630323B1
:10D2100084F8343004F1240384F82900A363F1E78F
:10D2200000F8173C064B40F8103CA0F11C014038B8
:10D23000007EF8F74FF9D0E7E0500020D4500020EE
:10D24000FF3F420F02480122002113F07ABF00BFC6
:10D25000A0500020014BD861704700BFA0500020B3
:10D2600038B54FF0FF3105464FF0FF30FFF704FFB0
:10D270002E492F48F5F7C8F80446FFF705FF002CA4
:10D2800051DB2C4C40F201132385E36925626433A2
:10D29000E36247F23053236300226FF0730384F894
:10D2A0002420E36304F14005BFF35B8F55E8003FA2
:10D2B00045E800210029F9D1BFF35B8F4FF0FF3122
:10D2C0004FF0FF30FFF7D8FE04F12401207EF8F77D
:10D2D00001F9FFF7D9FE184A0023204607F072FF34
:10D2E00000280ADABFF35B8F012355E8002F45E8D9
:10D2F00000310029F9D1BFF35B8F4FF0FF314FF0C0
:10D30000FF30FFF7B9FE207EF8F7C6F8FFF7BCFE46
:10D31000BFF35B8F236CBFF35B8F13B1054807F03E
:10D3200077FFE06B38BD6FF00B00FBE7B8500020D3
:10D33000C1D10000A0500020447B0B00074B01220C
:10D340001A64D3F84035B3FBF0F01844044BDB69A2
:10D35000984234BF00200120704700BF0080004089
:10D36000A050002010B50C29036912D118680A4C8E
:10D3700080EAE073A3EBE073990803F0030300284D
:10D3800004FB03F3BCBF49425B42C2E90013002027
:10D3900010BD6FF08500FBE790D00300024B012227
:10D3A0001A7010F016BA00BFD8610020024B01229B
:10D3B0001A7010F00EBA00BFD761002010B5094BEB
:10D3C0001A7804461AB100221A700AF061FC064B62
:10D3D0001A7832B100221A702046BDE810400AF0D7
:10D3E00033BC10BDD7610020D861002008B514F00F
:10D3F000B3F84FF47A72A0FB020302FB0133C00BB7
:10D4000040EA4340014B1B68C01A08BDE8500020A9
:10D4100037B58C18FFF7EAFF241A002C16DD4FF4FD
:10D42000004540F2E73000214FF47A720023E4FB1C
:10D430000501F7F78FFE02460B4600210020CDE9DB
:10D440000001064808F068FF03B030BD044B01221C
:10D450001A7003B0BDE8304010F0BBB910050020D1
:10D46000D8610020014814F0BEB800BF10050020AC
:10D47000014814F0B8B800BF4805002008B514F002
:10D480006BF8064AA0FB020302FB0133C00B40EA23
:10D490004340034B1B68C01A08BD00BF40420F0049
:10D4A000EC50002010B5FFF7E9FF0446002012F011
:10D4B00006FC054B201A18604FF47A7390FBF3F0CA
:10D4C000024B186010BD00BFEC500020E850002057
:10D4D00037B58C18FFF7D2FF241A002C14DD0E4844
:10D4E0000E4A4FF4004500210023E4FB0501F7F745
:10D4F00031FE02460B4600210020CDE9000108481C
:10D5000008F00AFF03B030BD064B01221A7003B0C9
:10D51000BDE8304010F05DB93F420F0040420F00BF
:10D5200048050020D761002010B5094C204613F0B3
:10D5300048FC50B12269A168136843F400231360CA
:10D540000B68044A1321204698471B2010BD00BFDA
:10D5500064500200010006000D4BA0F10B020F2ADF
:10D5600093F9003003D97F2B0BD100207047094A73
:10D5700002447F2B12F90B0C04D17F2808BF002036
:10D5800070477F209842A8BF184640B2704700BF3E
:10D59000ED610020DB610020034B1880034B1B680A
:10D5A0000146DB680248184790610020F4500020D3
:10D5B000DC500200024B1980024807F0CFBD00BFCB
:10D5C0008C61002024070020054BBFF35B8F1B6894
:10D5D000BFF35B8F43FA00F000F00100704700BF1B
:10D5E000F050002001238340064ABFF35B8FDB43EA
:10D5F00052E8000F184042E800010029F8D1BFF3BB
:10D600005B8F7047F05000200123074ABFF35B8F08
:10D61000834052E8000F184342E800010029F8D186
:10D62000BFF35B8F10F0D5B8F0500020044B83425D
:10D6300004D1044B06201980FFF7E6BF704700BFF6
:10D64000DC5002008C610020012908D002291AD088
:10D65000D9B90E4B1878032817D1FFF7D5BF0B4B5C
:10D660001B78022B11D11378012B08D0022B08D084
:10D67000002B08BF1221064B02201970EDE7112183
:10D68000F9E71621F7E70720E7E770476D6200200A
:10D69000DA6100202DE9F0418B680C461D46002719
:10D6A00025B97F2F06D90120BDE8F0812A8A6D684F
:10D6B0001744F5E7DB681B7803F00703022BF2D170
:10D6C000DFF86C803A464146204611F066FA0028A1
:10D6D000E9DB184E94F85930B37594F85A30C6F80F
:10D6E0000080FF2B18BFAE3BD4E9080218BF5DB223
:10D6F000114BB78083424FF002039341757511D3EC
:10D700000E4BA0FB030103FB0211A36AC01841F1F9
:10D7100000014FF47A720023F7F7CCFCC6E902014E
:10D720000020C1E74FF0FF306FF00041F1E700BF8C
:10D73000EE610020D01A0020037DC12500CA9A3B6B
:10D7400030B5002189B00020FBF7BAFE204D214CF6
:10D750002860002200237F20FBF780FE0146206026
:10D7600028681D4D11F0ACF823681C48DA681C4B82
:10D770001C4C1A607F21102217F096F9AB682360C9
:10D780001BB300230093184918486FF007034FF4A8
:10D79000007207F073FE1649144813F0B4FD2368B5
:10D7A00028465B68984710F0200006D180F3118866
:10D7B000BFF36F8F0423184602DF0E4B02932368DA
:10D7C00005485B6A02AA0421984709B030BD00BF32
:10D7D000FC500020F8500020DC500200DB610020EB
:10D7E000F01A0020F4500020007E0020301A0020A3
:10D7F0002B60020049D6000008B50146034813F02B
:10D800008BFC0120FFF700FF002008BD3C07002033
:10D8100008B50146034813F07FFC0020FFF7F4FE33
:10D82000002008BD5807002013B5064BADF80610C0
:10D830001B6805481C6902220DF106030121A0475F
:10D8400002B010BDF4500020DC50020013B5054BAF
:10D8500001911B6804481C69002201AB0121A0470B
:10D8600002B010BDF4500020DC50020013B5064B8E
:10D87000ADF806101B6805481C6901220DF106036E
:10D880001146A04702B010BDF4500020DC50020049
:10D89000024B1878003818BF012070476D620020D5
:10D8A000044B1A78012A9DBF012200201A700D2016
:10D8B000704700BF6D620020034B1A78012A9ABF9F
:10D8C000002018700D2070476D62002010B5084CC4
:10D8D0002378013B012B08D8064B07481B681B6ABD
:10D8E000984701232370002010BD0D20FCE700BFE6
:10D8F0006D620020F4500020DC5002002DE9F0435E
:10D90000054689B00020FFF75FFE00287DD1012089
:10D91000FFF75AFE78B10120FFF764FEDFF824829A
:10D92000DFF82492894F00220023404607F0E4FBF1
:10D930000446002878D10220FFF746FE40B10220BD
:10D94000FFF750FE824B00211A78284616F02BF97B
:10D950000320FFF739FE30B10320FFF743FE7D4976
:10D96000284616F027F90420FFF72EFE7A4C30B334
:10D970000420FFF737FE2378032B40F0B280022308
:10D980002370764B73491B68754E93F85B30C3F375
:10D990004002C3F3800343EA02130A7F22F011021C
:10D9A00013430B77B388002B6E4B18BF32461B789E
:10D9B00008BF0022284616F004F90023B380072090
:10D9C000FFF702FE28B10720FFF70CFE2846FFF7FD
:10D9D0007DFF2378032B00F0B2800520FFF7F4FDD4
:10D9E000002840F087800620FFF7EEFD002800F0B9
:10D9F000A6805D4B284693F9001016F0ECF806203F
:10DA000009B0BDE8F043FFF7EDBD0020FFF7EAFDE8
:10DA1000564C00220023204607F06EFB00283FF4FE
:10DA200076AF10F0F4FEF4E720220021684617F0EC
:10DA30003BF8A0680FF04AFEC3680093A368002279
:10DA4000002B45D1ADF80420494A94F85B60128858
:10DA50008DF8062094F859208DF8162094F85A2055
:10DA6000FF2A1CBFAE3A53B28DF815309DF817301F
:10DA700066F300038DF81730D4E9080302228145CC
:10DA80009A4129D3A0FB070107FB0311A36AC01821
:10DA900041F100014FF47A720023F7F70BFB9DF878
:10DAA0001730C6F3C00666F341038DF81730636D77
:10DAB0000493CDE9020194F858308DF814302846CB
:10DAC0000022694616F06FF8204610F0A0FE2AE703
:10DAD000198A5B680A44B3E74FF0FF306FF00041EA
:10DAE000D8E7244B24481B685B68984783053FF5BB
:10DAF00046AF64E71F4C214A23681178DB681E4853
:10DB0000984723681E499B6A1E4A09881A48984705
:10DB100088B10620FFF758FD40B1134B284693F912
:10DB2000001016F058F80620FFF75CFD09B0BDE8BC
:10DB3000F0430FF04EBE0520FFF754FD53E709B048
:10DB4000BDE8F0833C070020037DC12500CA9A3B55
:10DB5000DA610020F01A00206D620020FC500020E5
:10DB6000D01A0020D96100208C61002058070020C5
:10DB700090610020F4500020DC500200EB61002096
:10DB80008E6100202DD60000F8B50E4D2A78B2B176
:10DB90000D4C0E4E23680E48DB6831809847236891
:10DBA00030785F69FFF7D8FC01460948B847236819
:10DBB0000748DB69984702232B700020F8BD0D2031
:10DBC000FCE700BF6D620020F4500020906100204F
:10DBD000DC50020038B50E4B0E4D1B680E485B68DA
:10DBE00098472B78022B05D0012B01D00D2038BD92
:10DBF0008305FBD5094813F02FFB04460028F5D117
:10DC00000323064906482B7013F048FB2046EEE735
:10DC1000F45000206D620020DC500200C0010020A2
:10DC2000301A002000487047F01A002010B50E4C42
:10DC30000E4823685B68984710F0010010D02368F5
:10DC40000B4A9B6A09480121984750B94FF0FF33AE
:10DC500008484FF0FF3207F0B5FA074B93F9000080
:10DC600010BD7F20FCE700BFF4500020DC50020014
:10DC7000B5D50000240700208C61002008B5134BA7
:10DC800013481B685B689847024600F00103580080
:10DC9000D30648BF40F00800910648BF40F001009D
:10DCA000930548BF40F01000110548BF40F0200028
:10DCB000D30548BF40F04000510548BF40F0800008
:10DCC000D30448BF40F4807008BD00BFF45000206A
:10DCD000DC50020010B586B00C46182200216846C0
:10DCE00016F0E2FE054B8DF800401B6804485B6AA5
:10DCF0006A460C21984706B010BD00BFF4500020C2
:10DD0000DC500200014B1878704700BFEC61002026
:10DD100010B586B00C4618220021684616F0C4FEE5
:10DD2000064B8DF800401C70054B06481B686A4680
:10DD30005B6A0321984706B010BD00BFEC6100206C
:10DD4000F4500020DC500200F8B5114E114B37683A
:10DD5000114D1970BB6A2A800C46B3B10520FFF73C
:10DD600041FC0620FFF73EFCFB680C482146984723
:10DD700033680B4A9B6A29880848984708B90020ED
:10DD8000F8BD0520FFF740FCF9E70C20F8E700BFDD
:10DD9000F4500020EB6100208E610020DC50020076
:10DDA0002DD6000010B586B00C461822002168461A
:10DDB00016F07AFE054B8DF800401B6804485B6A3C
:10DDC0006A460021984706B010BD00BFF4500020FD
:10DDD000DC50020010B588B00C461422002103A8C4
:10DDE00016F062FE01AB0293084BADF804401B68CD
:10DDF00007485B6A01218DF80D1002AA9847002898
:10DE000014BF0320002008B010BD00BFF450002054
:10DE1000DC50020010B586B00C46122200210DF134
:10DE2000060016F041FE094B00941B6808485B6A27
:10DE300001218DF804108DF805106A4698470028D6
:10DE400014BF0320002006B010BD00BFF450002016
:10DE5000DC50020010B588B00C461422002103A843
:10DE600016F022FE01AB0293074BADF804401B688D
:10DE700006485B6A02AA01219847002814BF0320C4
:10DE8000002008B010BD00BFF4500020DC5002009C
:10DE900010B586B00C46132200210DF1050016F0D6
:10DEA00003FE084B00941B6807485B6A01218DF84C
:10DEB00004106A469847002814BF0320002006B0CB
:10DEC00010BD00BFF4500020DC5002007FB51822C6
:10DED0000021684616F0E8FD044B05481B686A46B9
:10DEE0005B6A0121984707B05DF804FBF4500020FD
:10DEF000DC5002007FB518220021684616F0D4FDE0
:10DF0000054B06481B6801215B6A8DF804106A46C0
:10DF1000984707B05DF804FBF4500020DC50020085
:10DF200021B1034B1B780B7000207047072070470E
:10DF3000ED610020014B002019707047ED61002059
:10DF400008B50C4B1B680BB1DB6A5BB913F004FB23
:10DF5000094AA0FB020302FB0131C00B40EA414029
:10DF6000C90B08BD054898474FF47A720023F7F7AC
:10DF7000A1F8F6E7F450002040420F00DC50020008
:10DF800030B5104687B00D461C4611F082FE4FF4A6
:10DF90007A73A4FB0343CDE90243084B8DF810507C
:10DFA0001B68CDE900015B6A05486A46082198476D
:10DFB000003818BF012007B030BD00BFF45000206A
:10DFC000DC500200F0B59FB00EADCC088DF80720F4
:10DFD00000214022284604AF1E4616F065FD10229F
:10DFE000002138468DF841408DF851408DF8614050
:10DFF00016F05AFD012C08AC0BD10DF10F03119353
:10E000000DF107031593249B1293259B0E961994EB
:10E0100016931422002109A816F046FD9DF807303A
:10E020000648002B08BF3D46054B08951B68224655
:10E030005B6A052198471FB0F0BD00BFDC500200AD
:10E04000F450002010B586B00C461422002101A81F
:10E0500016F02AFD044B00941B6804485B6A6A466C
:10E060000621984706B010BDF4500020DC50020095
:10E0700010B586B00C461422002101A816F014FD3C
:10E08000044B00941B6804485B6A6A460721984762
:10E0900006B010BDF4500020DC50020010B50F4C4B
:10E0A00086B018220021684616F0FEFC23680C4852
:10E0B0005B6A6A4609219847012360B98DF80A30E6
:10E0C000236807485B6A6A460B219847003818BFE7
:10E0D000012006B010BD1846FBE700BFF450002039
:10E0E000DC50020010B586B00C46182200216846AC
:10E0F00016F0DAFCA4F1200011F0CBFD054B1B68F3
:10E10000CDE900015B6A04486A460A21984706B0D7
:10E1100010BD00BFF4500020DC500200024B034849
:10E120001B681B6B184700BFF4500020DC50020036
:10E1300070B58AB00C4615460021102206A81E466E
:10E1400016F0B2FCC4F34001C4F380028B18C4F390
:10E15000C0041B190596ADF818500FD18DF800308A
:10E16000184BCDF810D01B6817485B6A04AA0B2126
:10E170009847003818BF01200AB070BD04338DF8ED
:10E18000003000238DF801304BF69B03ADF80230D0
:10E19000EA23ADF8043099B103238DF80630072344
:10E1A00032B15A1C28336B44022103F8281CD3B225
:10E1B000002CD5D028336B44012203F8282CCFE75C
:10E1C0000623EDE7F4500020DC500200A1F10B0320
:10E1D0000F2B10B512D80A4B0B4403F80B2C094B2C
:10E1E0001888884201D0002010BD074B1B685C696D
:10E1F000FFF7B2F901460548A047F4E70720F3E727
:10E20000DB61002090610020F4500020DC5002000F
:10E210002DE9F743484E0446A368DB6B002B7DD104
:10E22000A3689B6B002B40F08180A368DB6AFBB97D
:10E230004FF00008306801A9C2690EF0AEFFA36874
:10E24000074600284AD01B690199002B3BD00246A3
:10E25000204698470546002838D0306829460EF0F9
:10E26000BBFFBD424FF00108E4D00FF0B2FA03E06B
:10E27000204698470028DBD1A368DB691BB1204604
:10E2800098470028C8D02D4DBFF35B8FD5F800907C
:10E29000BFF35B8FB9F1010FBED1DFF8A480B8F8EE
:10E2A00000703FB3A368274DDB682968FBB13A468D
:10E2B000204698472B6803442B60B8F800301B1A9F
:10E2C000A8F80030A8E76FF05705C6E701463068A8
:10E2D0000EF082FFB8F1000FCED0C6E71B69002B0D
:10E2E000F8D001220DF1030120469847F2E76FF0C4
:10E2F0005700DFE7204611F0E6FC2B4643F808798B
:10E300000C33BFF35B8F53E8002F43E800910029E3
:10E31000F9D1BFF35B8F0FF05CFA7DE72046984799
:10E3200000287FF47DAF03B0BDE8F0832046984716
:10E3300000287FF47AAFF6E7D0010020D801002052
:10E34000926100200051002037B50C4D286801A9CA
:10E35000C2690EF075FF044630B9EB6813B113F0D3
:10E360005BFCEC6003B030BD0198A1B213F05DFC22
:10E37000286821460EF084FFE8E700BFD0010020A6
:10E3800010B5124C1248606012F01BFD08B9012054
:10E3900010BD6068836823B11B6C13B10D49224620
:10E3A00098470020F8F7C4FD08B17830EFD16068D5
:10E3B000082111F08DFC6068102111F089FC606863
:10E3C00083681B6A03B198470020E1E7D001002071
:10E3D0007850020011E20000F8B5124E124D338859
:10E3E000E3B90024114BAC600122BFF35B8F53E80B
:10E3F000001F43E800200028F9D1BFF35B8F0FF026
:10E40000E8F92046F8BD3B686868195D83685B6879
:10E41000984701343388A342F5D8E2E7044F00243B
:10E42000F8E700BF92610020D0010020DC0100204D
:10E4300000510020034610B50120C3B1BFF35B8F2C
:10E44000104A52E8004F002C04D142E8000CBCF105
:10E45000000FF6D1BFF35B8F12D10B4803600B4B5B
:10E4600019800B4B1B781BB1FFF7B6FF002010BDC6
:10E4700052F8040C83685B69002BF7D09847F5E7E6
:10E480000520F4E7D801002000510020926100200F
:10E490006E62002030B5144687B005460A4699B131
:10E4A00094B1042111F026FC70B105AB28680293E9
:10E4B0001023CDE90043064900680AF00DFA07B0C1
:10E4C000BDE8304011F00ABC072007B030BD00BFE6
:10E4D0000044400438B5064B064C9D6805492B683E
:10E4E0000348042298472368002BF7D038BD00BFAB
:10E4F000A050020004510020044B186880EA40300C
:10E5000080EA504080EA40101860704704510020B3
:10E51000024B01221A7008F0D5BB00BF6F620020C9
:10E5200008B50020FDF794F905490023CB60054BA1
:10E530004B6003238B60BDE808400EF06BBD00BF4D
:10E540000851002011E5000010B50020FDF780F90A
:10E55000064904460EF0D9FD783002D120460EF06F
:10E56000B0FD034B00221A7010BD00BF08510020FF
:10E570006F62002040B2002808DB4309044900F024
:10E580001F0001224033824041F82320704700BF22
:10E5900000E100E040B2002808DB4309044900F034
:10E5A0001F0001226033824041F82320704700BFE2
:10E5B00000E100E040B20028A7BF00F1604000F594
:10E5C000614000F00F00034BACBF90F80003185CF3
:10E5D0004009704714ED00E010B5064C064920468E
:10E5E00012F06CFE00220023204606F0AFFF002050
:10E5F00010BD00BF101B0020FDE5000037B50F4C1B
:10E60000A5683F21EB682046984770B90C212B691B
:10E610006A462046984740B9094B009A93F9001082
:10E62000914202D01A7011F0EDFB4FF4F01200236A
:10E63000044806F0BFFF03B030BD00BFF050020039
:10E6400074030020101B0020014B93F90000704759
:10E6500074030020084BD3F8082542F00302C3F8E6
:10E6600008250422C3F81025D3F8042522F003025C
:10E67000C3F80425704700BF00900040014B012201
:10E680001A60704700900040014B01221A617047E8
:10E69000009000400048704748900040054A0649F5
:10E6A00001235364D2F84435013B0B60C2F848356E
:10E6B000704700BF009000401851002008B5094B7A
:10E6C000D3F8483528B9084B084A09485D210DF0B0
:10E6D00041FA084A12689A4216BF036000200120DE
:10E6E00008BD00BF009000403A6002009B6002003D
:10E6F0004E60020018510020004870474C900040C6
:10E70000014BD3F84C0570470090004008B5084B0A
:10E710001B69834205D0074B074A084846210DF084
:10E7200019FAFEF7A7FABDE8084008F0B1BB00BF30
:10E73000701B0020BD60020085610200D0600200F5
:10E7400010B508490C69844205D0074B074A0848B0
:10E7500054210DF0FFF9C1E90223BDE8104008F093
:10E76000B9BC00BF581B00202F610200726102007B
:10E77000D060020038B5174A174C0023137023608D
:10E78000FEF708FC0028606006DA144B144A40F2D9
:10E79000031114480DF0DEF9134D4FF0FF33A36061
:10E7A000124B134C2B60134B2360FEF7F3FB002836
:10E7B000286104DA094B0A4A40F20D11E9E7FEF735
:10E7C000E9FB0028206104DA044B054A40F21311EA
:10E7D000DFE738BD70620020401B00204761020067
:10E7E0004D610200D0600200701B00200DE70000A8
:10E7F000581B002041E7000002460B46014811F07B
:10E80000C3BA00BF701B0020014B1869FEF702BAA3
:10E81000701B002070B5EFF3108672B6084C237899
:10E820005BB9084D286911F062F96861064D2869E5
:10E8300011F05DF901236861237086F3108870BDC3
:10E8400070620020701B0020581B002010B5EFF3F1
:10E85000108472B60A4B00221A700A4B5969186963
:10E86000891A18BF012111F044F9074B5969186939
:10E87000003918BF012111F03CF984F3108810BD54
:10E8800070620020701B0020581B002010B5FEF79E
:10E89000F1F9C21CBDE81040024841F1000311F03B
:10E8A00073BA00BF581B002002460B46014811F006
:10E8B0006BBA00BF581B0020014B1869FEF7AAB9BC
:10E8C000581B0020014B1869FEF79CB9581B00200B
:10E8D000014BD3E902017047581B00202DE9F74F87
:10E8E000464CBFF35B8F05460E461746012354E89E
:10E8F000002F002A03D144E800310029F7D1BFF3EB
:10E900005B8F0CBF98464FF00008A14673D14FF0C3
:10E91000000ACDE900AA2A466068334611F0F7F8EC
:10E92000E0B1BFF35B8F54E8003F012B03D144E813
:10E9300000A2002AF7D1BFF35B8FFEF79BF9A84234
:10E9400071EB060338D22E4B281A66EB0101984270
:10E9500071F1000130D34FF002082DE06068FEF73E
:10E9600051F98246EFF3108B72B6FEF783F902304D
:10E9700041F10001854276EB010121D28BF3108831
:10E980007A1C06D06068FEF73DF90146F8B205F042
:10E9900065FC4FF0FF336068A360FEF73BF9BFF3FF
:10E9A0005B8F002359E8002F012A03D149E8003189
:10E9B0000029F7D1BFF35B8F404603B0BDE8F08F6D
:10E9C0007B1C03D05146F8B205F040FCA760C4E9B7
:10E9D00004568BF31088BFF35B8F022359E8002F96
:10E9E000012A03D149E800310029F7D1BFF35B8F39
:10E9F0004FF00008E0E74FF00308DDE7401B002080
:10EA00000100400070B5174CBFF35B8F042054E841
:10EA1000003F022B03D144E80002002AF7D1BFF3E4
:10EA20005B8F25461CD16068FEF7F4F8A668731C5E
:10EA300006D06068FEF7E6F80146F0B205F00EFC7D
:10EA40004FF0FF33A3600020BFF35B8F55E8003F1A
:10EA5000042B03D145E80002002AF7D1BFF35B8FF6
:10EA600070BD00BF401B0020F8B51F4CBFF35B8F8B
:10EA70000546032354E8002F022A03D144E800315D
:10EA80000029F7D1BFF35B8F26462AD1EFF3108719
:10EA900072B66068FEF7B6F80146E8B205F0D6FB3C
:10EAA0006068A560FEF7AEF80568FEF7E3F8D4E904
:10EAB00004239042994112D2281E18BF012087F3E7
:10EAC00010880223BFF35B8F56E8002F032A03D17F
:10EAD00046E800310029F7D1BFF35B8FF8BD012074
:10EAE000EDE70420FAE700BF401B002008B504F062
:10EAF0003DFE01F04DFB11F025F901F099FD1048A4
:10EB000007F07CFE11F0FDFA01F068FF01F0E2FF72
:10EB100004F088FB08F05CF9FFF7DCFC02F0DEF89B
:10EB200008F0F4F807F03AFF02F084F911F022F946
:10EB300008F006FA04F03EFDBDE8084003F082BE8E
:10EB4000845402007FB505460C4631B34B792BB394
:10EB500088792388ADF808300026A378CDF80A60BC
:10EB600021798DF80D30E378ADF80E6043EA01218C
:10EB70000DF10A028DF80C0011F0D6FE9DF8090087
:10EB80009DF8083000B933B90021009602AB2A463F
:10EB9000084611F0F1FC04B070BD024C01F0F2FF28
:10EBA000D7E700BF99610200064B002918BF0B464A
:10EBB0005A78197802B911B9194611F018BE1046E1
:10EBC000704700BF9361020037B5EFF3108372B650
:10EBD000054CD4E9124583F31088CDE90045FDF7D3
:10EBE000F5FC03B030BD00BF1020002010B5094A6D
:10EBF000094C53780949013353702046102211F013
:10EC0000A8F994E80F0004E90F00054B01221A70DF
:10EC100010BD00BF826200203C510020A462002091
:10EC20007162002070B50F4E96F8243004460D46F0
:10EC30000BB9002070BD10220021284615F034FFCA
:10EC400096F824202301DBB29342F2D2D21A102A82
:10EC5000316AA8BF1022D2B21944284615F0FCFE32
:10EC60000120E7E7881B002030B5124B1249587885
:10EC70000B46012203F8012B104A02F10C0452F852
:10EC8000045B43F8045BA242F9D112781A700023A6
:10EC90008B73094B0A4CC87303F110051868596847
:10ECA000224603C20833AB421446F7D1054B01227A
:10ECB0001A7030BD8262002084620020AD1B0020EB
:10ECC0002C5100207162002070B5144C14496078FA
:10ECD000FFF7A8FF054618B1BDE87040FFF786BFF3
:10ECE000104B114A93F832301049D65C1048324626
:10ECF00015F0B2FE02230F49657028462370FFF716
:10ED000091FF28B101236370BDE87040FFF7ACBFED
:10ED10001EB1FFF7A9FF0323237070BD826200209C
:10ED2000A4620020881B0020A06102003C5100204A
:10ED30007262002094620020014B00225A637047E7
:10ED4000881B002070B50446406B00283DD0D4E9F4
:10ED50000632134302D02069002836D094F82430BC
:10ED60000BB1206A88B394F83230032B30D8194D98
:10ED7000234604F13806186859682A4603C2083346
:10ED8000B3421546F7D1636B256A1A78F5B9551C5D
:10ED9000802D01D910F0EFFFE8B203F07FFA606B2D
:10EDA00003F02EFA0C4B616B186006460B4B2E4499
:10EDB0002A461E6015F050FE636B1A780132521B12
:10EDC0000021304615F070FE012070BDED1ADFE71E
:10EDD0000020FAE7881B00204C51002050510020F1
:10EDE0002DE9F74F7A4C636B8342014626465DD18D
:10EDF00000285BD0D4E90632DFF8D891134394F8A9
:10EE0000323019F8037014BF01250025AD0117B188
:10EE1000023FC7F34707DFF8C0A1DFF8C0B1DAF857
:10EE20000000DBF80020DFF8B881121A15F014FE9C
:10EE3000102200216B4815F037FE45EAC70543460E
:10EE4000694A45F0010503F8015B02F10C0152F833
:10EE5000040B43F8040B8A42F9D112781A7094F823
:10EE600024305F495F4888F80F301022002388F86B
:10EE70000E3011F06EF896E80F005C4D85E80F003B
:10EE8000584B103503F11006186859682A4603C21A
:10EE90000833B3421546F7D1554F564A00237B70CD
:10EEA0003B7001231370534B1B7813B903B0BDE8BB
:10EEB000F08F504A4D4800231370F5F7F7FC3B786C
:10EEC000032BF0D8DFE803F0023B3E6BD4E9065396
:10EED00055EA03027E7801932DD04148102200218B
:10EEE00015F0E2FD019B96B90F2D4FEA152273F143
:10EEF00000032169404888F8002088F801502A461C
:10EF000028BF0E2215F0A8FDFFF770FECBE73601F3
:10EF1000023EF6B2AE424FF000029A410BD2AA1B5B
:10EF200063F1000321692E48112A73F1000328BF01
:10EF300010223144E6E700237B7001233B70FFF78A
:10EF4000C3FEB0E72D492E48102211F002F87D785B
:10EF500094F82420DBF8000029496B1E1B01DBB26A
:10EF6000D21A102AA8BF1022D2B2184415F074FD8C
:10EF700023492846FFF756FE20B101357D70FFF783
:10EF800073FE90E794F8323019F803501DB1032353
:10EF900078703B70F3E703F075F9656383E794F8E5
:10EFA0003230164919F8035016482A4610F0D1FF9E
:10EFB000DAF8000013490278EB43134418442A4658
:10EFC00015F04AFD03F05EF9002363636BE700BFB1
:10EFD000881B0020A06102004C51002050510020ED
:10EFE000A4620020B4620020AD1B00201C51002050
:10EFF0008262002071620020A66200203C51002045
:10F000009462002072620020034B5A6B824204BF5C
:10F0100000225A63704700BF881B0020034B18680A
:10F0200008B190F8800000F0010070477C5100208A
:10F0300008B5FFF7F3FF08B1014B186808BD00BF22
:10F040007C51002008B5082811D8DFE800F012052F
:10F050000507090714141400012008BD0420FCE76B
:10F06000064B1B7813F0100F18BF0120F5E710F0C6
:10F0700082FE0020F1E70220EFE700BFCA62002015
:10F0800010B5064B1C78064B1878FFF7DBFFE4B28F
:10F09000844234BF0020012010BD00BFC8620020A0
:10F0A000CB62002010B5044601F062FB044B204601
:10F0B0001968012211F077F9BDE8104001F0EEBAAD
:10F0C0005451002010B5044601F052FB054B1A784C
:10F0D000054B204693F9001011F05CF9BDE8104093
:10F0E00001F0DCBAD1620020CD620020014A10702C
:10F0F00010F04CBFCB62002038B504460D4601F03D
:10F1000037FB054B2A461868214610F046FFBDE83C
:10F11000384001F0C3BA00BF745100200348044BCB
:10F1200000680022114611F0F2BC00BF7C510020A3
:10F130005851002008B5064B1B7833B112F0F0FB94
:10F140003B2894BF0020012008BD0120FCE700BF40
:10F15000C962002010B5114C10F0C9FF07F0B8FAD1
:10F160002378012B17D912F0FCFB0D4BD3E90423B4
:10F17000904299410FD20123237007F059FA01F010
:10F1800067FD012803D1074B187810F0FFFEBDE89A
:10F19000104001F059BA00232370F0E7C562002047
:10F1A000C01B0020CB620020F0B5144B87B0044692
:10F1B0000E4615460021182268461F6815F074FC9B
:10F1C00002948DF80D608DF80E504CB1EFF3108362
:10F1D00072B60B4AD2E91001CDE9040183F310881D
:10F1E00001F0C6FA384610F06EFF6946384611F055
:10F1F000DCF801F053FA07B0F0BD00BF74510020F5
:10F200001020002008B5074B1B7853B1AE2012F038
:10F210003BFB30B1FFF734FF18B1BDE8084002F006
:10F220004BBC08BDC962002010B501F011FE0F4BA8
:10F230001860FFF7FDFE044602F0C8F84CB9BFF3B2
:10F240005F8F0B490122D1E84F3FDBB213B1BFF30F
:10F250002F8F10BDC1E8432F002BF4D1BFF35F8F78
:10F260000B20BDE81040FFF71DBF00BF7C51002000
:10F27000CC620020F7B5244B1B7807460E46154696
:10F28000002B37D0047810F0CBFE631C5B01002804
:10F2900034D103F1CE000DB1A83080B212F0F4FAEF
:10F2A00040B3FFF7EDFE044620B355B302F068FE0D
:10F2B00007F09EFE154B187811F017FB144B291E12
:10F2C0001A7818BF012161F3C30238461A7002F0A0
:10F2D0009FFF104B1B7800932A460F4B314602F0DC
:10F2E000D5F9012E07D111F004FB07F0AFFC10B9DE
:10F2F00002F024FB0024204603B0F0BD03F22E40B0
:10F30000C9E702F045FED3E7C9620020CE620020C3
:10F31000CA620020C6620020CF62002073B51F4B76
:10F320001B7805460C46BBB3FFF7AAFEA0B31C4AE8
:10F33000137823F007031370FFF770FE0646FFF7FC
:10F3400077FE02F043F8002301A8ADF8043011F075
:10F35000FFFA01F017FC11F0C8FA124A01AB12785B
:10F360002946032002F066F8012D09D111F0C1FAF7
:10F3700007F06CFC20B90CB910F0FDFC01232370E0
:10F3800002F002FE07F034FE0EB9FFF74DFFFFF763
:10F39000C5FE054B00221A6002B070BDC962002094
:10F3A000CA620020C7620020785100207FB510F0AB
:10F3B0004FFE18220021684615F076FB054B694682
:10F3C000186802F031FF69460220FFF795FE07B08A
:10F3D0005DF804FB7451002010B5114B1B78EBB1A4
:10F3E000FFF74EFED0B10F4C204607F095F912F012
:10F3F00097FAB0F5C07F11D32268C009831EB3EB22
:10F40000D21F4FEAD21094BFA2EBC3120022226097
:10F41000BDE8104098BF184602F07EBB10BD00BF8B
:10F42000C96200207051002010B5044602F086FA2F
:10F43000082C1ED8DFE804F0211D051D0B131D1537
:10F4400019000021BDE810400846FFF767BF012200
:10F450000A4BBDE8104018680021FFF70BBF0022DF
:10F46000F6E7BDE81040FFF7B7BFBDE81040FFF773
:10F47000C9BEBDE8104010F07EBC10BD7451002024
:10F4800010B586B008284FD8DFE800F03333050FF9
:10F4900024243542480061B3264B19680122062016
:10F4A00006B0BDE8104010F07EBF234C2368002258
:10F4B00083F88020214B0621186810F006FE204BAF
:10F4C00020681A781F4B93F9001006B0BDE8104071
:10F4D00010F060BF1C4C18220021684615F0E4FAB9
:10F4E0006946206802F0A0FE6A460621206810F0F6
:10F4F00054FD06B010BD144C18220021684615F0CA
:10F50000D3FA6946206802F08FFE6A460521EDE7CE
:10F51000012006B0BDE8104010F068BF012006B021
:10F52000BDE8104010F074BF06B0BDE8104010F008
:10F5300022BC00BF545100207C5100207851002093
:10F54000D1620020CD620020745100202DE9F041ED
:10F550000646174601F01AF8054680B11F4C23787D
:10F56000022B10D02278022AD3B216D04FF0000816
:10F57000022B17D9033B052B12D910F0FCFB0025F9
:10F580002846BDE8F08101F007FF2278022A804674
:10F59000D3B2EDD136B90028F1D14FF0000801E027
:10F5A000002EECD002F0CAF92378022B0AD10C4BC2
:10F5B0000C4800221A7007F053FC07F017F8207867
:10F5C00010F0E4FC2378072B01D107F0D9F8002FC5
:10F5D000D6D020784146FFF753FFD1E7CB62002019
:10F5E000C5620020C01B002010B5FFF7AFFF044626
:10F5F00058B1074B1B782BB10120FFF777FD02F0C4
:10F6000035FA10B90020FFF771FD204610BD00BF8C
:10F61000C962002073B50D461E46FFF797FF0446EA
:10F6200028B312F0C4F938B101F012FB421ED2B275
:10F63000022A01D910F09FFB0E4B03221A700E4BC9
:10F6400002201E60FFF752FD6B1F584258410026F2
:10F650000DF107018DF80760FFF760FE9DF8073098
:10F660002BB102F06BF931463046FFF757FE2046CA
:10F6700002B070BDC7620020545100202DE9F04156
:10F68000704A1378107086B0044603F0FF0783BBFE
:10F69000002800F09C8001F05DFD6B4B01221A7088
:10F6A00007F068FC694E3578EDB22846FFF7CAFCD2
:10F6B00080462846FFF7C6FC4745C0F08B80844251
:10F6C0006DD2357802210120EDB200F05FFF08B95C
:10F6D00010F051FB022D40F08D8001F05DFE0746D9
:10F6E00002F02CF9002F00F098800620FFF7DAFCDA
:10F6F00094E00028D6D1544B1A78002A4FD0534DAD
:10F7000018702B78022B02D101F046FE044601F05E
:10F7100093FD07F051FC07F0A1F90221012000F050
:10F7200035FF08B910F027FB2B78082B4AD8DFE803
:10F7300003F036050B12252539363600002006B0B9
:10F74000BDE8F041FFF7D2BC4CB3052006B0BDE8E0
:10F75000F041FFF7A7BC3E4C0220FFF7C7FC23682F
:10F76000002283F880203B4B0421186810F0ADFC88
:10F77000206806B0BDE8F041FFF7A4BC0220FFF707
:10F78000B5FC18220021684615F08EF9324B694607
:10F79000186802F049FD69460420FFF7ADFC06B089
:10F7A000BDE8F0810220FFF7A1FC18220021684685
:10F7B00015F07AF9284B6946186802F035FD69465C
:10F7C0000520EAE706B0BDE8F04110F0D4BA07F032
:10F7D00045F967E78442E2D33378204A022F127852
:10F7E000DBB205D1042C03D1042B01D1032AD6D0DE
:10F7F00030781FE002F0A2F8082D20D8DFE805F0ED
:10F800000D0D1F0A050A0A0D0D00154B1A786FF32E
:10F8100004121A700220FFF769FC002728463946B7
:10F82000FFF72EFE3578EDB22846FFF70BFC844239
:10F83000B5D3284606B0BDE8F041FFF7F5BD10F09E
:10F840009AFAEAE7C8620020C9620020CB62002071
:10F850007C5100207851002074510020C4620020A7
:10F86000CA62002008B5054B1B78062B01D010F0AA
:10F8700082FABDE8084010F02CBC00BFCB6200202B
:10F8800070B5002006F09EFF224B1B7803F00103A9
:10F890001843C0B208B910F06EFA1F4B1B78022B48
:10F8A00001D010F068FAEFF3108172B61B4A93682A
:10F8B0000133936081F3108806F0BAFE002006F051
:10F8C00081FF044601F0C4F9012820D1022012F082
:10F8D00029F812F046F8124D044628460E4607F065
:10F8E000BFFAA0344FF0010346F100062B772846FB
:10F8F0000C4B2B62C5E9044607F07AFA08B110F008
:10F900003AFA094A13780133DBB2137001E0002C94
:10F91000DFD170BDC7620020CB6200201020002024
:10F92000C01B002055F10000C562002008B51A4B2D
:10F930001B78022B01D010F01EFA184B1B789B0786
:10F9400001D410F018FAEFF3108172B6144AD3689C
:10F950000133D36081F3108801F07AF901280FD0C8
:10F96000022813D0002006F02DFF98B10D4B0E4851
:10F9700000221A7007F074FABDE8084006F06CBE69
:10F98000084B094800221A7007F06AFA022011F0A9
:10F99000C9FFE7E708BD00BFCB620020C7620020B7
:10F9A00010200020C5620020C01B00202DE9F84374
:10F9B000DFF874915D4D99F800302C79022B804668
:10F9C00001D010F0D8F9042C15D8DFE804F0031AA0
:10F9D0000714180001240126274601E0042400260C
:10F9E0002B685B7803F00703052B0CD1504A137882
:10F9F00043F00103137000242046BDE8F88305247A
:10FA0000EDE70224E7E749482246414611F098F81D
:10FA1000F0B13EB14548394603F05AF8064608BBF6
:10FA2000022F0AD001F07AF8022C37D0042C67D0CC
:10FA3000012C67D1EC7C013432E03D4A1378384622
:10FA400043F00103137011F06DFF11F0CDF8E9E7F9
:10FA500001F064F820B12B6893F90030002BE3DC4F
:10FA6000012607E001F05AF820B12B6893F9003025
:10FA7000002BD9DC01F062FF00210846FFF74EFCA5
:10FA800099F8000010F082FA2B685B7803F0070306
:10FA9000022BB0D03046FFF705FBACE72C7D0234DB
:10FAA000E4B2234E33785A0718D4DFF888802868E8
:10FAB000D8F800301A7810F0AAFA531C5B0118BB72
:10FAC00003F1A00011F0E0FE074600B33378D8F848
:10FAD000000043F00403337010F0F9FA3378DB07C9
:10FAE0008AD5286810F093FA002885D001F032F802
:10FAF000002881D00D4811F07EF80F4B18607BE78D
:10FB00006C7D98E70024CCE703F53070DAE701F06C
:10FB100015FF39463846FFF701FC084B01221968EA
:10FB2000052010F040FCD9E7CB620020585100209E
:10FB3000CA6200207C5100207851002054510020DE
:10FB400013B5114C2378022B01D010F014F90F4A91
:10FB5000137823F007031370FFF7E0FA207810F012
:10FB600015FA002401A8ADF8044010F0F1FE084A8F
:10FB700001AB12782146032001F05CFC0220FFF764
:10FB800091FA02B010BD00BFCB620020CA62002013
:10FB9000C762002008B5054B1B78062B01D010F07A
:10FBA000EAF8BDE80840FFF701BC00BFCB620020C7
:10FBB0002DE9F047664EDFF89C813568664F10F0FE
:10FBC000FBF9664B18702B782B4413F8010C10F0DE
:10FBD0005CFE00B28000FF28614B28BFFF20187038
:10FBE000D8F80030197801310622C9B2404610F029
:10FBF000A7FF8146002868D03B78D90765D4032148
:10FC0000404602F065FF044680B94FF4087011F0D9
:10FC10003BFE00285BD03B7823F0050343F005034F
:10FC20003B7010F0E1FF306810F051FA3B78DA07D2
:10FC30004FD5EFF3108272B64A4C636801336360AC
:10FC400082F3108810F0C0F902460B4652EA030115
:10FC500051D1EFF3108172B6C4E9122381F31088F9
:10FC600006F01AFD3B78DB075ED5B9F1000F5BD0DB
:10FC7000D8F8000010F0CBF9002855D000F06AFF4A
:10FC8000002851D03848394F02F0A2FA314810F01C
:10FC9000B2FF3860002847D00320FFF727FA344B23
:10FCA0001B78032B2ED9386802F0B2FAC02101F07C
:10FCB000C1FD00284AD1336883F8800010F0C8F9EC
:10FCC0002846BDE8F047FFF7FDB90424AEE7052458
:10FCD000ACE700F023FF82460028AAD1254B187814
:10FCE00010F054F950465146FFF718FB2046BDE886
:10FCF000F047FFF7D7B9B2F1170043F1FF310246E1
:10FD00000B46A6E70421022006F0B6FF38B9EFF350
:10FD1000108272B6A3690133A36182F3108833683D
:10FD2000002283F88020C9E7124B187810F02EF9D2
:10FD30006B7803F00703022BF1D100F0EFFE0146D0
:10FD40000028ECD1BDE8F047FFF7E8BABDE8F0873E
:10FD50007C51002058510020CA620020CD62002052
:10FD6000D162002010200020A46102007851002000
:10FD7000C8620020CB62002030B51A4B1A78052AE1
:10FD800087B004D01B78042B01D00FF0F4FF164D80
:10FD90002B685A7812070AD42C68204600F036FCEB
:10FDA000F0B1204607B0BDE8304010F0D1B81C7863
:10FDB00011F0B6FD013424018442EDD901F0BEFDFD
:10FDC00010F046F918220021684614F06DFE2868EC
:10FDD000694602F029FA28686A46042110F0DDF825
:10FDE00007B030BDCB6200207451002070B5164BB7
:10FDF0001B78032B01D00FF0BEFF144D2B685A78EF
:10FE0000120707D4286810F066F92868BDE870402A
:10FE1000FCF754BC1C7811F083FD013424018442AA
:10FE2000F0D90B4C266801F089FD23682868002270
:10FE300083F88020052110F048F910F009F93046C8
:10FE4000BDE87040FFF73EB9CB620020785100203A
:10FE50007C51002010B5094B1B78032B01D00FF00B
:10FE60008AFF074B1C68002384F8803010F0F0F8FC
:10FE70002046BDE81040FFF725B900BFCB62002047
:10FE80007C51002070B510F09FF802460B46EFF34E
:10FE9000108172B61F4EC6E90E2381F310881E4CE6
:10FEA0001E48217811F0080F10D06FF30411217053
:10FEB000016809784901D431541A63F10005EFF360
:10FEC000108372B6C6E90C4583F31088006810F001
:10FED000A7F80446A0B10620FFF708F9FFF79EF83F
:10FEE0000446FFF7A5F801F071FA02F04DF807F0AB
:10FEF0007FF801F04BFB64B9BDE87040FFF794B99F
:10FF000010F0A6F8224621462046BDE87040FFF7D3
:10FF10004BB970BD10200020CA620020745100202F
:10FF2000F0B54B4E4B4D30682C688DB0002838D062
:10FF3000BCB3637803F00703022B32D1837803F05C
:10FF40003003202B32D1017801316B460322C9B234
:10FF500010F0DDFD28B32178013106AB0322C9B2D0
:10FF6000204610F0D4FDDDF818C09CF8023003F0F4
:10FF70003003202B15D19DF80970FF2F11D09DF86B
:10FF80001F10009BFF290CD09DF812209DF829E03E
:10FF900038B1D81905D0724503D1614414F04CFD35
:10FFA00070B10DB0BDE8F040FFF700BA2378052B23
:10FFB000F7D1A3789A06F4D4E278C3789A42F0D1C4
:10FFC00010F002F802460B46EFF3108172B6224899
:10FFD000C0E9102381F310882D683068002785F868
:10FFE00080700178013106AB0622C9B210F08FFD96
:10FFF00058B3069A537803F00703032B25D19DF8D5
:020000040001F9
:100000002830FF2B21D0D35C042B1ED16378DB0674
:100010001BD50220FFF76AF839463846FFF77EF90C
:100020000FF0CAFF2B782B44044613F8010C10F094
:100030002CFC02B29200FF2A28BFFF22D2B2214636
:100040002846FFF7B1F80DB0F0BD10F001F8E7E772
:10005000745100207C5100201020002038B5144B32
:100060001B78042B01D00FF086FE124B1B789B07E8
:1000700001D40FF080FE0FF0A7FF0D46044601F0FB
:1000800087FF06F0B5FFEFF3108372B60A4AC2E9A4
:100090000A4583F31088094B1B78032B07D10420F2
:1000A00011F040FC064B1A786FF304121A7038BD39
:1000B000CB620020C662002010200020C462002015
:1000C000CA6200207FB5EFF3108172B60C4A136844
:1000D0000133136081F310880FF0BAFF182200215A
:1000E000684614F0E1FC074B6946186802F09CF87A
:1000F00069460120FFF700F807B05DF804FB00BF78
:10010000102000207451002037B51F4D1F4C2B7854
:100110008342236838BF28707F2B16D911F000FC6A
:10012000B0F5C07F2ED32268C009831EB3EBD21F67
:100130004FEAD21096BFA2EBC312002218462260EB
:1001400003B0BDE8304001F0E7BC06F011FB044607
:1001500020B103B0BDE83040FFF73EB900F012FD1A
:1001600010F0C3FB0FF074FF28788DF8044010F0F6
:100170009DFB8DF8040000F0FBFA01A810F02DF9AA
:1001800000F08CFA03B030BDD26200207051002024
:10019000094A0A4808B500231370094A1370094A2E
:1001A0001370094A137011F0E3FB10F097FBBDE8E0
:1001B000084010F012BD00BFCB620020C01B002021
:1001C000C9620020C5620020CC62002038B5054617
:1001D0000FF08AFF044668B1074B1A7842B11B78CA
:1001E000012B05D0012211462846FFF7FDF90446F0
:1001F00000F02AFA204638BDCB6200202DE9F041FC
:1002000006460F46154698460FF06EFF0446C8B1E5
:100210000E4B1A78022A0DD01B78032B0AD0FEF75A
:1002200089FF044630B1069B424639463046FFF707
:10023000F1F904460DB12046A84700F005FA204622
:10024000BDE8F081002DFAD0A847F8E7CB62002086
:100250002DE9F047089F8146884616461C460FF058
:10026000CBFE054600286DD0384A214630460FF0B7
:1002700028FF002852D0012241464846FFF766F980
:1002800000284AD0204601F0A3FF304A21463046DC
:1002900000F090F900283ED000F0E0FCDFF8B0A0BC
:1002A00094F805908AF8000011F081FB40B100F04D
:1002B000D5FC03283FD039D80138C0B2012837D83F
:1002C0004FEA49095FFA89F9224B234A83F80090E3
:1002D0009AF80030D91E4B424B41117863F3041158
:1002E00011706079C0F10500C0B2FEF7FFFE1B4B34
:1002F00062881E601A4B1A801A4B22791A70627932
:10030000E2B9A8F10503594259413046FEF7B2FF60
:10031000A3791BB110B90FF09BFE00250FB1284641
:10032000B84700F091F92846BDE8F0870428C7D007
:100330000FF021FDC4E74FF00209C5E7E279531C35
:10034000DAB2DEE7002FEED0B847ECE79BFF010002
:10035000C4620020C6620020CA62002074510020DE
:10036000CF620020CE62002030B587B004460FF087
:1003700043FE054618B3174B1B78062B1DD1164BB1
:1003800022681B689A4218D100F0D8FB0246C8B90F
:1003900004210120FFF728F908B90FF0ECFC18221E
:1003A0000021684614F080FB2068694601F03CFF9C
:1003B00020686A46052110F007F800F045F9284644
:1003C00007B030BD6FF00103002204210120FFF7C8
:1003D00021F9E1E7CB6200207451002070B5064698
:1003E0000D460FF009FE0446A8B101221146304621
:1003F000FFF7ACF8044660B1084B802D38BF80256C
:100400001D60074B002207201A70FEF76FFEFEF7F3
:10041000E3FF00F019F9204670BD00BF70510020C5
:10042000D262002010B504460FF0E6FD012384F8E7
:100430008030BFF35F8F0B4B00221A70BFF35F8FCA
:1004400068B1094B1B7843B100F0ACFF28B1074BF2
:100450001C60FEF7EDFD00F0B9FF00F0F5F801209B
:1004600010BD00BFCC620020C96200207C5100207A
:1004700038B505460FF0C0FD0446B0B10C4B1B78F3
:100480001BB100F07FFB10F030FA0A4B1B78022BF7
:1004900009D1012229461046FFF758F818B100216A
:1004A0000846FEF73BFF00F0CFF8204638BD00BFFE
:1004B000C9620020CB62002010B50FF09DFD0446FC
:1004C00030B1044B1B780BB110F011FA00F0BCF8FE
:1004D000204610BDC962002010B50FF08DFD044606
:1004E00068B1094B1B7803F0FF0433B1074B1B784D
:1004F000022B06D101F088F8044600F0A5F820464A
:1005000010BD0024F9E700BFC9620020CB620020C3
:1005100038B5054601F0A2F810B90024204638BDD0
:100520000FF06AFD0028F8D0094B1B781BB9002496
:1005300000F08AF8F2E701F091F80028F7D001F016
:100540009BF804460028FAD00FF036FD2870EFE73C
:10055000C9620020014B93F900007047CD62002072
:10056000014B1878704700BFD162002010B50FF022
:1005700043FD044630B1044B1B780BB100F0C4FEC0
:1005800000F062F8204610BDC9620020F8B5084F9F
:1005900005460E46002457F8043B33B13146284641
:1005A000984718B10134042CF5D10120F8BD00BFE3
:1005B000C45402002DE9F041094C05460E46174689
:1005C00004F1100854F8043B33B13A46314628464A
:1005D000984710B14445F5D10120BDE8F08100BF36
:1005E000B4540200F8B5084F05460E46002457F8EB
:1005F000043B33B131462846984718B10134042CE6
:10060000F5D10120F8BD00BFA454020070B5074E1B
:100610000546002456F8043B2BB12846984718B1EC
:100620000134062CF6D1012070BD00BF8C540200AD
:10063000034B00221A70034BFF221A70704700BF51
:10064000D4620020D362002070B5134EEFF3108502
:1006500072B6337803F0FF0433B90FF08CFBFF243C
:10066000347085F3108870BD013C14F0FF04F7D19D
:1006700006F08AFB20B185F3108806F075FBE5E7EC
:100680000121084606F0F8FA10B101200FF067FBCF
:10069000FEF7DCF8E4E700BFD462002010B5074C99
:1006A00023781B0601D50FF066FB054B1B780BB9B1
:1006B0000FF061FBFF23237010BD00BFD362002049
:1006C000D462002010B5104B5C68C4F30804BCB1C0
:1006D000E4B2A4F11002D3B252B2511D06DA0FF007
:1006E0004AFB0A4B04F00F04185D07E0002AF8DB10
:1006F00003F1604303F5614393F80003400910BD23
:100700004FF0FF30FBE700BF00ED00E014ED00E02C
:1007100038B50446FFF7D6FF431C08BF7F20EFF330
:10072000108572B6104A3CB913782BB10F4B19786B
:1007300043B249B2994206D114780134E4B2012C93
:10074000147004D0012485F31088204638BDFEF7CC
:1007500061F82146204606F08FFA0028F2D02046A4
:100760000FF0FFFAEEE700BFD4620020D362002052
:1007700010B5094C2378FF2B01D00FF0FCFA074B82
:100780001B780BB90FF0F7FAFFF79CFF431C08BF6B
:100790007F2040B2207010BDD3620020D4620020C0
:1007A00038B50446EFF310830B4D2B6072B60B483F
:1007B0000FF073FE08B10FF0DEFA08480FF04FFE9D
:1007C000047006480FF051FE054B01221A602B6899
:1007D00083F3108838BD00BF805100208451002071
:1007E00000400140F8B50D4C07460E462046152145
:1007F00015460FF0B4FDFF2803464FF000000CD063
:10080000282202FB0344607063F07F00C0B2A7603F
:1008100026736573FFF7C4FF0120F8BD881C002014
:10082000F8B5114B114C002A18BF1C460D46064660
:1008300014BF04211521204614BF002780270FF084
:100840008EFDFF280ED003B203EB830304EBC3033A
:1008500038430124C0B25C701E72DD60FFF7A0FF58
:100860002046F8BD0020FCE7E81B0020881C002083
:10087000F8B5104C07460D46204615210FF06FFDC8
:10088000FF28064613D0282303FB0044022363708D
:10089000A7600FCD10340FC495E8030084E803006F
:1008A00066F07F00C0B2FFF77BFF0120F8BD00209B
:1008B000FCE700BF881C00202DE9F041114C804668
:1008C0000F462046152115460FF049FDFF28064624
:1008D00016D0282303FB004403236370C4F8088068
:1008E00027730FCD10340FC495E8030084E803008C
:1008F00066F07F00C0B2FFF753FF0120BDE8F08132
:100900000020FBE7881C002038B50C4C054615215B
:1009100020460FF024FDFF280DD0282303FB0044C0
:100920000423637060F07F002B782372C0B2FFF75E
:1009300037FF012038BD0020FCE700BF881C0020E5
:1009400038B50B4C0546152120460FF008FDFF2851
:100950000CD0282303FB004460F07F000523C0B2C5
:1009600063702572FFF71CFF012038BD0020FCE7F3
:10097000881C002038B50B4C0546152120460FF089
:10098000EEFCFF280CD0282303FB004460F07F001E
:100990000623C0B263702572FFF702FF012038BD45
:1009A0000020FCE7881C002038B50B4C05461521BB
:1009B00020460FF0D4FCFF280CD0282303FB004472
:1009C00060F07F000723C0B263702572FFF7E8FE76
:1009D000012038BD0020FCE7881C002008B51A2241
:1009E0000123064906480FF01CFD064B0122C3F8FF
:1009F0000423BDE8084000F03DBA00BFD5620020E6
:100A00008451002000400140F8B52E4BD3F800215E
:100A10005AB10022C3F80021D3F800312A4D2B4EE1
:100A20002B4FAA79EB799A4200D1F8BD28460FF0F6
:100A300025FD047814F0800F04F07F0404EB840497
:100A400014BF07EBC40406EBC4046378072B36D845
:100A5000DFE803F00412171D24292D31627B94F97D
:100A60000C10A0680FF08AFA28460FF00DFDBFF3B6
:100A70005F8F00232370D4E7E168207A0FF080FABB
:100A8000F2E7A06804F110010FF07CFAECE7217B9B
:100A9000A06804F110020FF077FAE5E704F108000E
:100AA0000FF068FAE0E7207A0FF066FADCE7207AC8
:100AB0000FF05CFAD8E7207A0FF05AFAD4E70FF07B
:100AC0005AF9D1E70040014084510020E81B002082
:100AD000881C002010490B464FF6FF7223F80129AD
:100AE000FE22DA70FF221A710022C3F805208A6004
:100AF0005A732D229A73DA7302221A745A2203212E
:100B00005A7401229A74D9740422597505211A75F0
:100B10009975DA75704700BFF0620020024B587C6F
:100B200000F00100704700BFEF620020024B5A7CCA
:100B300060F300025A747047EF620020014B987C0A
:100B4000704700BFEF620020014B9874704700BFF0
:100B5000EF620020024B587CC0F34000704700BF9A
:100B6000EF620020024B587CC0F38000704700BF4A
:100B7000EF620020024B5A7C60F382025A74704785
:100B8000EF620020014B587CC0087047EF620020E4
:100B9000024B5A7C60F3C7025A747047EF62002020
:100BA000014B93F900007047EF620020014B187071
:100BB000704700BFEF62002000487047F0620020DD
:100BC000024B0288A3F80120704700BFEF620020AB
:100BD00000487047F4620020034A0368C2F80530F9
:100BE0004368C2F809307047EF6200200048704740
:100BF000F2620020024B0288A3F80320704700BF76
:100C0000EF6200200378012B0BD004D9023B012BAB
:100C10000ED90FF0B0B8094B00225A7342789A737C
:100C20007047064A53738378D373C378137470473D
:100C3000024B0268C3F80D20704700BFEF6200202E
:100C4000024BD3F80D300360704700BFEF62002005
:100C5000014BD87C704700BFEF620020014B187D2C
:100C6000704700BFEF620020014B587D704700BF06
:100C7000EF620020014B987D704700BFEF620020BB
:100C8000014BD87D704700BFEF62002008B5EFF33D
:100C90001082074B1A6072B606480FF0FEFB08B1CF
:100CA0000FF069F8BDE8084002480FF0D8BB00BF5C
:100CB0008C5100209051002008B505480FF0D5FB5D
:100CC000044B01229A60044B1B6883F3108808BD13
:100CD00090510020004001408C51002008B5402276
:100CE0002023064906480FF09CFB064B0422C3F85C
:100CF0000423BDE8084000F0BDB800BFD01F0020AD
:100D0000905100200040014073B5484BD3F80821B2
:100D10004AB10022C3F80821D3F80831444DAA791A
:100D2000EB799A4201D102B070BD28460FF0A6FBC4
:100D300003780446122B76D8DFE803F00A131D2748
:100D40002C327575373C41464A4F535C606A6F00E0
:100D5000C668007AFFF73AFA307028460FF094FB25
:100D6000DDE722694669837B417B007B0092A268B4
:100D7000FFF744FAF0E7A3688669417B007B0093A4
:100D8000D4E90423FFF764FAE6E7D0E90206FFF7A7
:100D9000EBFAE1E7D0E90361007AFFF71FFBDBE73D
:100DA000C668007A0FF077F9D6E7D0E90206FFF7B8
:100DB00039FBD1E7C668007AFFF75AFBCCE78468B5
:100DC000FFF77AFB2070C8E78468FFF785FBF9E737
:100DD000D0E90206FFF79CFBBEE78468FFF7C6FB7D
:100DE000F0E7D0E906360093D0E90423806801F0EB
:100DF0004DFDB1E7846801F0E5FDE3E78269C6696E
:100E0000037D00920269D0E9020101F093FDA3E79E
:100E1000D0E902060FF026FE9EE7D0E903168068AF
:100E200001F04EFB98E70EF0A6FF96E70040014068
:100E300090510020054A002301210133102B82F834
:100E4000801002F18102F8D1704700BF07630020D3
:100E5000074A0023114692F8800018B103EBC31330
:100E6000C81870470133102B02F18102F3D170478B
:100E70000763002010B5074C23784BB9064A0121BF
:100E800014200EF060FF14200EF069FF0123237080
:100E900010BD00BF176B0020B9080200074BD3F844
:100EA000502502F0F702042A06D00022C3F81021D0
:100EB000D3F8102101221A61704700BF00100040D2
:100EC00008B5F0F74FFD064B01221A61D3F8002256
:100ED00022F48072C3F80022BDE8084001F048B94E
:100EE0000080004010B50021094C042001F0BCF83E
:100EF0000023C4F80032FFF7E3FF4FF4C023C4F827
:100F0000083301232363BDE81040FFF7C7BF00BFCC
:100F10000010004008B50021042001F0A5F8FFF7FB
:100F2000CFFF074B4FF40042C3F808230022C3F859
:100F3000002201229A62BDE80840FFF7AFBF00BF60
:100F40000010004010B5094CD4F8003223F480732F
:100F5000C4F8003208B1F0F705FDF0F7FDFC01F030
:100F600007F90FF0DAFC0123236110BD0080004077
:100F700008B501F0B5F830B9034B01221A61C3F886
:100F80001001D3F8103108BD0010004008B5084822
:100F90000021F0F7DBFC50B9064AD2F8003243F4E6
:100FA0008073C2F80032BDE8084001F0CFB808BD38
:100FB000105502000080004013B501A8FFF740FE65
:100FC0009DF805009DF804400FF06EFC9DF8073079
:100FD0009DF806201B0643EA02432343034A43EAE3
:100FE0000023C2F86C3602B010BD00BF00100040F4
:100FF00010B500EB80040B380F2804F62E140CD922
:101000000EF0B9FEB4F5166F07D2A4F6381444F406
:101010008074034BC3F8084510BDA4F51664F8E7C7
:101020000010004010B5184B184A1B681848B3FB55
:10103000F2F33222534300229A421ED10EF09BFE5D
:101040000FF06BFC0FF040FCF0F78CFC114A1049DC
:10105000D2F8003223F48073C2F800320E4A002323
:1010600043F213401370C1F808030C480824C0F879
:101070000843C1F80032537010BDD0F85015C9B202
:101080000029DDD00132D7E70402002040420F00E2
:1010900000100040008000401A6B0020004001401A
:1010A00010B50A4C20780FF032FC01F00BF82078D4
:1010B000FFF748FF064A074BC2F808330023C2F87F
:1010C0000032054A1371537010BD00BF196B002028
:1010D00000100040130006081A6B002010B5002114
:1010E0000D4C042000F0C0FF43F20203C4F80833A3
:1010F000F0F738FC01F03CF8084BD3F8002222F45A
:101100008072C3F8002201221A61054A0023C4F844
:101110000032537010BD00BF00100040008000403E
:101120001A6B0020064A00231370064A1360064A11
:101130001370064A1360064A1360C2F80330704702
:10114000216B00209C510020196B00209851002039
:101150001A6B002070B5324D2B780BB10EF00BFEE0
:10116000304B314C01211961D3F8042522F00302E0
:10117000C3F80425D3F8082542F00302C3F8082574
:101180000422C3F810250023C4F8FC3FC4F8FC1F58
:10119000F0F710FCA0B14FF08053D3F83003D3F830
:1011A0003413D3F83823204B461C18BFC4F84C071F
:1011B000481C18BFC3F88415511C18BFC3F88825F4
:1011C000194C0F23C4F81035184BC4F814357F237D
:1011D000C4F81835012640F20223C4F85066C4F85A
:1011E0003435134BC4F838350FF087FBFFF7E4FEB6
:1011F000FFF7C8FCFFF7FCFE0EF0A9FE30460EF02C
:10120000AEFDD4F800320BB10EF0B5FDF0F78CFB5B
:1012100008480121F0F7B8FB01232B7070BD00BF17
:10122000216B0020008000400010004008000006F4
:10123000211001001011004010B52D4C2378002B17
:1012400041D02C4B0022C3F8FC2F2378013B0B2B01
:101250004BD8DFE803F008080608394047394A4A06
:1012600039080FF031FB0FF049FB0120FDF792F92F
:10127000214B0822C3F808230022C3F80C21D3F81D
:101280000C311E4BD3F8002222F44072C3F8002226
:1012900001221A61A3F5E043C3F8FC2FF0F762FBCB
:1012A000F0F75AFBF0F776FB2378012B04D00320EC
:1012B000F0F75EFBF0F73EFB114A0023137053700A
:1012C00053711371237010BD0021042000F0CCFE77
:1012D00000F04EFFC7E70B4B18780FF018FB00F03B
:1012E000F1FEF5E700F024FFBDE70EF044FDBAE79C
:1012F000216B0020001000400040014000800040B1
:101300001A6B0020196B002010B5224C23780BB902
:101310000EF031FD2378033BDBB2082B09D8012006
:1013200000FA03F340F21312134203D113F02C0F0F
:1013300028D110BD002005F045FA012807D0022869
:101340000DD00028F5D0BDE810400EF014BD0020EF
:1013500005F046FA10F0ECF90028EAD1F3E722781C
:10136000072AD3B20AD006D8033B012BEBD8BDE83D
:10137000104005F027B90B2BDBD0E4E7BDE81040A7
:1013800005F004BA05F01EFA0028D2D00128DAD1FF
:10139000DEE700BF216B0020014B1878704700BFCB
:1013A0001A6B002008B5074B07491B784878032BB8
:1013B000DAB203D0052A01D008B9002008BD0EF02A
:1013C000DAFCFAE7216B00201A6B0020134B70B592
:1013D0000446186000B3124E7578BDB1114B1B78EE
:1013E000032BDAB214D0052A14D00EF0C4FC00226C
:1013F000002373700C4BC3F80445C3F80022D3F8E4
:101400005025D2B2022A01D101229A60284670BD2D
:10141000064AEDE7064AEBE70546F7E79851002054
:101420001A6B0020216B00200010004052000800C1
:10143000120008002DE9F04798464B4B4B4C4FF0FB
:10144000010AC3F810A04A4B154603221A704FF048
:101450000009C5F34003A37084F8019084F800905C
:1014600084F8059084F80690064698F900000F4627
:10147000F3F7F7FE3F4B404AC0B2C3F80C051168C2
:10148000002961D0126884F80190C3F804253B4A12
:10149000C3F800220EB90EF06EFC364C0023F600A5
:1014A000C4F86065C4F83431D4F83421C4F8283164
:1014B000D4F82821C4F83031D4F83021C4F80431EC
:1014C000012FD4F8042105BFC4F80031D4F800314D
:1014D00043F2024443F2134415F0010038D00C20CB
:1014E00000F054FE234B0022C3F86821D3F8683182
:1014F000234BC3F80C21D3F80C210822C3F8042392
:101500001C4B2048C3F804430021F0F71FFA164B88
:1015100018BBD3F8404598F80100F0F72FFA1A4BA2
:101520001C60FFF7F1FE104AD2F8003243F48073DA
:10153000C2F8003239460122042000F02DFD87B99F
:10154000BDE8F047FFF714BD84F801A052229FE7E1
:1015500005F038F90028C2D1D2E70124C3F840458C
:10156000D9E7BDE8F08700BF008000401A6B00207B
:10157000216B00200010004098510020520008000C
:1015800000400140105502009C51002010B5194B3D
:10159000194905221A700868184A194B28B3002007
:1015A00050700A68C3F80425164AC3F800220024C4
:1015B000C3F80441D3F80421C3F83041D3F83021F3
:1015C000C3F83441D3F8342143F20202C3F80423B0
:1015D000FFF7DCFCFFF798FE22462146042000F0CE
:1015E000DBFCBDE81040FFF7C3BC012151701222A3
:1015F000DBE700BF216B0020985100201A6B002010
:10160000001000401200080038B5104B1B78032B67
:101610001AD10F4CD4F85035023BDBB2012B13D852
:101620000C4DAB793BB90C4B4FF4707043F0010398
:1016300098470123AB710023C4F81C310120D4F872
:101640001C316061687138BD0020FCE7216B00200F
:10165000001000401A6B0020D0520200014B587954
:10166000704700BF1A6B0020024BD3F8480500F00A
:101670007F00704700100040034BD3F81C01003876
:1016800018BF0120704700BF001000402DE9F74F40
:1016900001935C4B9DF83090DFF86CA15B4CB2F18C
:1016A000000816464FF001021A61594B4FF006022E
:1016B0001A70584B18BF4FF0010883F80080564B42
:1016C00000271E70019B8AF80370834693F900007F
:1016D0000D46F3F7C6FD012EC0B2C4F80C05C4F8E0
:1016E00004B531D94D4AC4F8002200F093FCC4F887
:1016F0006C71012DD4F86C2105D1C4F80071D4F8B7
:101700000031474801E04FF00060404B002219F0E3
:10171000020FC3F84821D3F848111BBFC3F8442176
:10172000D3F8442140F4802040F4C02019F0040F85
:101730001ED00022C3F80021D3F80031012340F06D
:1017400001008AF8033013E003D1364AC4F80022BE
:10175000CDE74FF4A012C4F80022012DC4F86C713B
:10176000D4F86C2133D1C4F80071D4F800312C487E
:10177000264B0024C3F8044140F00200D3F80421B2
:101780008AF80440C3F80403019B5878F0F7F6F890
:101790008EB325492548F0F7D9F80146D0B922483B
:1017A000F0F7CEF8174AD2F8003243F48073C2F84B
:1017B000003200F0CBFCFFF7A7FD294640460FF0B2
:1017C000A0F8DDB903B0BDE8F04FFFF7D1BB4FF093
:1017D0000060CDE714482146F0F7B2F80028E1D0C8
:1017E000084BD3F8002242F48072C3F80022022290
:1017F000C3F84025DFE70E483146EDE703B0BDE80A
:10180000F08F00BF008000401A6B002000100040E5
:10181000216B0020196B0020186B002000181400A9
:101820001100000800381400E054020010550200B6
:10183000F85402002DE9F0413A4D2B78042B07466D
:101840000C4601D00EF097FA0FB90EF094FA072368
:101850003F2C2B70344D04D801232B610020BDE8B0
:10186000F081324B1E682644314CA6F13F08C5F882
:1018700044854FF4A013C4F804750027C4F800325F
:10188000C4F85471D4F854312A4B182218463946FA
:1018900013F00AF9173E0522394645600274C66006
:1018A000F0F74EF8D5F8003298BB43F48073C5F8D2
:1018B0000032FFF729FD0023C4F86C31D4F86C2105
:1018C000C4F80431D4F80431194C00F01FFC164B55
:1018D0000122DA64D3F84C25D3F84035904503D97A
:1018E000984519D9934217D30FF017F8D4F850350B
:1018F000DBB2092B10D0D4F854316BB900F018FCCE
:10190000F0F72AF80120F0F733F8074B01221A61AB
:10191000A4E743F40073CAE7074BC4F8043301207B
:101920009DE700BF216B0020008000409C510020FB
:1019300000100040A051002012000008F8B5434CF0
:1019400023780C2B7ED8DFE803F00D0D070E2D3128
:101950004A62777D7D7A0D003D4B1022C3F8082343
:101960000C232370F8BD0EF0AFFFEFF7FBFF3949F2
:101970003748D1F80032384A23F48073C1F8003276
:1019800043F2134500231370C0F80853334D082663
:10199000C5F80863C0F800325370FFF77FFA0123DF
:1019A0000B61DDE72B4B01221A61D9E70021284D9D
:1019B000042000F059FB43F20203C5F80833EFF7A7
:1019C000D1FF00F0D5FB2349234AD1F8003223F49C
:1019D0008073C1F800320023C5F80032DCE7204FE5
:1019E0001B4D387800260EF092FF00F06BFBC5F817
:1019F00000623878FFF7A6FA1A4BC5F80833164B81
:101A00001E715E7001232B63FFF748FAA8E7104DA3
:101A100000F08EFB0023C5F80032EFF79DFF0D4B61
:101A2000D3F8002222F44072C3F8002201221A6186
:101A30000D4BC5F80833E7E7FFF754FA90E7FFF7D7
:101A400069FA8DE7BDE8F8400EF095B9216B0020EA
:101A500000100040008000401A6B00200040014050
:101A6000196B0020130006080200000808B50F4A91
:101A70001378013B0B2B07D8DFE803F00815060AA3
:101A8000060606060606060D0EF075F900200BE0A8
:101A9000074B0121196102231370FFF7FFF9054B72
:101AA0001022C3F80423012008BD00BF216B0020D1
:101AB000008000400010004010B5154C2378012B29
:101AC00004D023780C2B01D00EF055F90823237095
:101AD000104B00244FF42052C3F80022C3F84841B1
:101AE000D3F84821C3F84441D3F844214FF4C0222D
:101AF000C3F80423FFF74AFAFFF706FC2246214603
:101B0000042000F049FABDE81040FFF731BA00BFE9
:101B1000216B00200010004038B5174D2B780C2B9E
:101B2000044604D02B78012B01D00EF024F9013C9F
:101B30000B23B4F5001F2B7001D30EF01CF90F4BD3
:101B4000C4F31404C3F864464FF400420024C3F8FD
:101B50000022C3F83C41D3F83C11C3F80423FFF73B
:101B600015FAFFF7D1FB22462146042000F014FAB3
:101B7000BDE83840FFF7FCB9216B002000100040A1
:101B800070B50EF0B4FA994BD3F80423150714D5A9
:101B9000974AD2F8681181B10021C2F86811D2F8D1
:101BA0006821C3F80C11D3F80C31924B1B78032B2E
:101BB00001D00EF0E0F8FDF763FE8D4BD3F804235F
:101BC000D40718D5D3F80021AAB10022C3F8002108
:101BD000D3F800210122C3F8082300F02DFA854B29
:101BE0001B78032BDAB206D0062A1ED1824BDB7893
:101BF0000BB10EF04EFA7E4BD3F8042390071CD5A0
:101C0000D3F80421CAB10022C3F80421D3F8042177
:101C10001022C3F80823774A1278033A042A5FD8BF
:101C2000DFE802F0065E494F58000EF0A4F8E2E744
:101C3000714B9B780BB1FDF779FE6D4BD3F8042304
:101C4000510521D5D3F82821F2B10022C3F828216B
:101C5000D3F82831674B1B78032B01D00EF08BF89B
:101C6000654B634D01221A70D5F8343163B9D5F84C
:101C70006045C4F3C7042046FDF798FE84423EBF8A
:101C800000B2C000C5F86005594BD3F80423920494
:101C900032D5D3F834217AB30022564CC3F834211C
:101CA000D3F834312378032BDAB21CD0052A3AD08A
:101CB0000EF061F820E0504B01225A71FDF7D2FD81
:101CC000BBE70222C3F808234B4B01221A71FEF72F
:101CD00053F8B2E70222C3F80823FEF787F8ACE70F
:101CE0000EF049F8A9E7FFF79DF9444B01221A616C
:101CF0000C232370FDF724FF3D4BD3F80423D604B7
:101D000021D5D3F83021F2B100223A4CC3F830216A
:101D1000D3F830312378032BDAB20BD0052A29D03F
:101D20000EF029F80FE0FFF7D9F90C232370FDF727
:101D300031FFE1E7304B01225A71FFF773F90423B9
:101D40002370FDF735FF2A4CD4F804331D011ED54E
:101D5000D4F86C31DBB1274D0026C4F86C61D4F89F
:101D60006C312B78062BDAB20BD0072A27D00EF075
:101D700002F80CE0FFF7B2F90C232370FEF7D0F85D
:101D8000E1E7FFF78DF90C232B70FEF77BF8184B7A
:101D9000D3F80423D40638D5D3F81021AAB30022EF
:101DA000144CC3F81021D3F8102121780329CAB2AA
:101DB0002BD027D8022A5BD00DF0DDFF25E000F004
:101DC000B7F9C4F80062EFF7C7FD0C4BD3F8002257
:101DD00022F44072C3F8002201221A61084BC4F8B1
:101DE00008330C232B70FEF735F8D0E70040014094
:101DF00000100040216B00201A6B00200080004082
:101E000012000008063A012AD6D84B4BD3F8042317
:101E1000900315D5D3F8442192B10022474CC3F862
:101E20004421D3F844312378062BDAB22DD0082A86
:101E30002ED1FFF757F80C23012023700EF01CF968
:101E40003D4BD3F8042351034DD5D3F84821002A44
:101E500049D03A4C0025C3F84851D3F8483123788B
:101E6000062BDAB217D0082A5ED00DF084FF3AE0D4
:101E70001022C3F808230320EFF77AFDEFF75AFD8D
:101E8000012323700EF0F5F8BFE7FEF7E7F8D7E778
:101E90000DF071FFD4E72A4B1B780BB90DF06BFFE7
:101EA000284A1378012B18D91378013BDBB2137041
:101EB0001378012BDDB216D100F004F91E49224B34
:101EC000C1F80032D1F848316BB10D63FEF7E6FF7F
:101ED0000023C1F84831D1F84831FFF7E1F80C236D
:101EE0002370FEF7EFF8144BD3F80423120417D530
:101EF000D3F83C21A2B1114C0022C3F83C21D3F805
:101F00003C3123780B2B01D00DF035FF0A4BD3F871
:101F10006856FEF7FFFF0C23E8B22370FEF7F4F8D3
:101F2000BDE87040FEF790BBFEF7DCFF0C232846AF
:101F300023700EF0A1F8D6E700100040216B0020BE
:101F4000196B0020186B00200038140010B5EFF357
:101F5000108472B6094BD3F8042312070AD5D3F8BC
:101F60000C213AB10022C3F80C210120D3F80C3126
:101F7000FCF700FB84F3108810BD00BF0040014057
:101F800000487047DC54020000487047D8540200F3
:101F900000487047D454020010B5174B0024C3F812
:101FA0003C41D3F83C31154B154CC3F8484500F182
:101FB000804000F58050C3F84C051248C3F82C0946
:101FC000BAB1114AC3F850454FF4E070C3F8542534
:101FD0000E4A11B90E49C3F84015C3F84425074B02
:101FE000D3F8002842F08002C3F80028C3F80405A3
:101FF00010BDC020ECE700BF0040014000F00140F0
:102000003C41014004F00140008000403C40014060
:1020100010110040064B074AC3F86025A2F58E72E6
:10202000C3F864254FF48062C3F80425704700BFED
:1020300000F0014048110040084B0022C3F83C2149
:10204000D3F83C31064A074BC3F8402502F59732D6
:1020500002F59672C3F84425704700BF0040014066
:102060001011004000F00140154BA1B9C022C3F887
:102070000825C3F84815C3F84C15C3F82C19C3F844
:102080004015C3F844150E4AD2F8003823F08003F7
:10209000C2F8003870474FF4E072C3F808250022F8
:1020A000C3F84825C3F84C25C3F82C29C3F84025AC
:1020B000C3F84425C3F85025C3F85425E3E700BF0F
:1020C00000F00140054B4FF48062C3F80825002260
:1020D000C3F86025C3F86425704700BF00F00140D5
:1020E00008B5084BD3F85035DBB243B9064B0EF0B8
:1020F00014FCD3F83C01003818BF012008BD0120B2
:10210000FCE700BF0010004000400140054B064ABC
:10211000C3F85825054AC3F85C254FF40072C3F88C
:102120000425704700F00140448100400010004049
:10213000054B4FF40072C3F808250022C3F8582558
:10214000C3F85C25704700BF00F00140054B064A0C
:10215000C3F85025054AC3F854254FF48072C3F8DC
:102160000425704700F001403C41014000800040E0
:10217000054B4FF48072C3F808250022C3F85025A0
:10218000C3F85425704700BF00F00140074B084AD0
:10219000C3F8682500F1402000F580304FF400625C
:1021A000C3F86C05C3F80425704700BF00F0014078
:1021B00068110040054B4FF40062C3F80825002267
:1021C000C3F86825C3F86C25704700BF00F00140D4
:1021D000074A00231360074A1370074B18B9187099
:1021E000064B1870704702781A704078F8E700BF05
:1021F000B8510020246B0020236B0020226B0020AC
:10220000014B186001487047B8510020256B002031
:10221000034B1A68034B002A18BF1846704700BFCB
:10222000B8510020256B002038B504460D4609B989
:102230000DF0A1FD0E4A0F4B10780F4A1B78126863
:102240002B70687092B10D490A780132D2B240B158
:1022500023B12046BDE8384012F0FEBB084B1A7887
:10226000F7E71BB1064B1B78D21AF2E738BD00BF67
:10227000226B0020236B0020B8510020256B00202A
:10228000246B0020014B01221A707047236B002041
:10229000014B01221A707047226B0020014B18700D
:1022A000704700BF246B002010B586B0044618228A
:1022B0000021684612F0F8FB054B1B88ADF8003092
:1022C000044B6A46186821460EF07EF806B010BD31
:1022D000A96B0020BC51002030B589B0FCF70CF987
:1022E000204B1C78012505FA04F4013C04404FF40E
:1022F000A07320220021E4B268465C4312F0D4FBB4
:102300000FF02FFB022300198DF81130164B0593A7
:1023100041F100016FF00203CDE900010693FEF7E1
:102320009DFC022817D004D8A84209D00DF023FD47
:1023300009E00338C0B20128F8D88DF8105002E047
:1023400004238DF81030684604F0EEFB08B90DF058
:1023500012FD09B030BD054B1B78002B14BF0423C0
:102360000123EEE7AB6B002029240100AC6B0020B9
:1023700010B5012104466FF002000FF087FA54B93E
:10238000FEF77EFC044B1B78834204D3BDE810406B
:102390000120FFF789BF10BDAC6B0020BFF35F8F3A
:1023A000084AD2E84F3FDBB2834203D0BFF32F8FFE
:1023B00000207047C2E8431F002BF2D1BFF35F8FAC
:1023C00001207047A56B002010B501210220FFF706
:1023D000E5FF08B9012010BD104C237801332370AC
:1023E000FEF748FC0E4A1378984284BF01331370FD
:1023F000FEF746FC237883424FF000040AD9094BCC
:10240000214601201C60FFF7C9FF0028E2D10DF032
:10241000B2FCDFE7FFF760FF2046DCE7AC6B002093
:10242000AB6B0020BC5100201FB5C31C044601D07B
:102430000DF0A1FC02210120FFF7B0FF68B31A4B99
:102440001C78FEF70BFC4CB9022807D104216FF071
:1024500002000FF039FA08B90DF08DFC134B144A45
:102460001B88ADF80830134B1B88ADF80A30124BAF
:102470001B788DF80C3001238DF80D300F4B009335
:1024800000201268ADF80E0002AB03210EF074F8C4
:1024900008B9FFF799FF04B010BD0121204604B030
:1024A000BDE810400FF0F2B9AC6B0020A96B002022
:1024B000BC510020A76B0020A66B002071230100F7
:1024C00070B506460C460FF04CFA02460B46EFF389
:1024D000108172B61648C0E9082381F310880121E3
:1024E0000020FFF75BFF08B90DF045FC2379D3B15D
:1024F0006579104B22881E600F4B1A800F4B00220B
:102500001A70FEF7B1FB0E4BE17818700D4B0E4AB6
:102510001D70A378284643EA01210EF005FAFFF763
:10252000DBFE012070BDFEF72DFB0546E1E700BF95
:1025300010200020BC510020A96B0020AC6B0020B3
:10254000AB6B0020A66B0020A76B0020012908B50B
:1025500001D9012008BDBFF35F8F0A4B1A78BFF382
:102560005F8F002AF5D00028F4D0BFF35F8F0322DD
:102570001A70BFF35F8F00216FF002000FF086F931
:10258000E7E700BFA56B002070B5124AA1F1080370
:10259000012B166804460D460BD8B04207D1002324
:1025A0001360BFF35F8F0C4A1370BFF35F8F01207E
:1025B00070BD00210320FFF7F1FE28B1B442F6D030
:1025C0002846FFF771FEF2E7B442F0D1BDE8704053
:1025D000FFF7FABEBC510020A56B0020064A136825
:1025E000834207D100231360BFF35F8F034A137048
:1025F000BFF35F8F01207047BC510020A56B002006
:1026000008B5024607484368C16D9A4205D18A421F
:1026100001D10DF0B0FB034803E058308A4218BFE7
:10262000002008BDB820002030B50C4C636804338E
:1026300087B0054602D00DF09EFB002465B9182234
:102640002946684612F030FAA38A2069ADF80030B6
:102650006A4607210DF0B8FE07B030BD60200020AB
:1026600013B5184C6368984202D00DF084FB002427
:102670000422022120460EF079F908B90DF07BFB07
:10268000114B00930521226904F1140301200DF080
:1026900073FF606801210FF0F9F860B90DF06BFB72
:1026A0000122042120460EF061F940B902B0BDE8D4
:1026B00010400DF060BB4FF0FF336360F0E702B0F5
:1026C00010BD00BF602000202926010070B50F4C0E
:1026D00000254FF0FF3604F1100004F0C1FB024664
:1026E00078B961680A200DF05EFE08B90DF043FB71
:1026F00066600122042120460EF038F908B90DF079
:102700003AFB583405B170BD0125E4E7B82000203C
:1027100070B50546EFF3108672B61B480DF0AEFE9D
:10272000044619480DF0B0FE86F3108824681CB9E1
:10273000BDE870400DF01FBBEDB1FFF7C7FF0FF014
:1027400010F90B46A16BA4620246891843F10005FB
:102750000020C4E908150121C4E9102384F82C10D5
:1027600084F8480084F8490004F1100004F040FBAC
:102770000028DDD170BD61682A4607200DF013FEE8
:102780000028F7D1D4E700BFC851002073B5054633
:10279000FFF736FF0446002843D0042202210EF042
:1027A000E5F8A0B9012128460FF070F808B90DF03E
:1027B000E2FA4FF0FF3363600122042120460EF05D
:1027C000D5F870BB02B0BDE870400DF0D4BAEFF39D
:1027D000108672B619480DF060FE08B10DF0CBFA04
:1027E00016480DF03CFE046014480DF03EFE86F3E2
:1027F0001088FEF7C7F994F85030984213D16368F7
:102800000093012305210E4A18460DF086FE012192
:10281000064628460FF03AF808B90DF0ACFA002E3B
:10282000C7D002B070BD1846FEF7B2F905200DF012
:102830004DFF0028E3D1FFF76BFFB3E7C85100203D
:102840001127010070B50D4C0D490E4804230822D4
:102850000DF0E7FD01264FF0FF3504F11000267062
:1028600065600FF085F804F1680084F85860E5654C
:102870000FF07EF8044B1E705D6070BDB820002024
:10288000C0510020C8510020602000202DE9F041F7
:1028900088B08046012125480E9D16461F460EF041
:1028A0007FF8044600283FD0AB78002B39D1B6F52D
:1028B0009B764FF000032372C4F810802B88A3820C
:1028C0002B796979E87843EA012104F1160247F18E
:1028D000FF370EF029F8AB7863760123A376AA7947
:1028E000E276EA7822766FF0030262604FF4877135
:1028F0008DF808308DF812300D4B03916846042195
:10290000CDE90067CDE90532ADF8101004F00CF9FF
:10291000054610B920460EF097F8284608B0BDE8E5
:10292000F081B6F5E576C4E70546F6E760200020BD
:10293000612601002DE9F04389B00546DDF84080AD
:1029400040460E4617469946FFF75AFE20B100252D
:10295000284609B0BDE8F083174802210EF020F8A0
:1029600004460028F3D0154B036301224FF487730C
:102970000272C0F80480039340F20113B5F59B7511
:10298000ADF8103007F59B770D4B876380F85090BA
:1029900046F1FF366846CDE90056CDE905388DF899
:1029A00008208DF8122004F0BFF805460028CFD18A
:1029B00020460EF049F8CBE7B8200020C9090200F4
:1029C0008D27010010B5094C002160680EF05EFFF4
:1029D00050B14FF0FF3301220221204663600DF019
:1029E000C5FF10B90DF0C7F9002010BD6020002010
:1029F00008B5064B1A78042A03D093F85830042BF4
:102A000002D110B1FFF762FE012008BDB8200020FE
:102A100030B5154B01781A78042A08BF1C4613F804
:102A2000582F87B018BF00240131042A08BF1C4664
:102A3000C9B26B46012205460EF069F890B18CB11F
:102A40000EF08FFFC4E910012B7884F84830009B0A
:102A50005B7803F00702052A14BFC3F34013002379
:102A600084F8493007B030BDB82000202DE9F3418B
:102A70004FF0FF320023CDE900230027134D064617
:102A80004FF0FF3838462B78022B16D1686869461C
:102A90000EF027FF009B019A13F59B7342F1000291
:102AA000CDE9003248B14345AC6B72F1000238BF4A
:102AB0009846A4F59B7408EB5404583527B100B12F
:102AC000346002B0BDE8F0810127DCE7B8200020C7
:102AD0002DE9F34103680446C8075D789E7893F8B2
:102AE00000800F462FD523790BB90DF044F9A8F1DA
:102AF0000508B8F17A0F00F28F8005F00705052D63
:102B000006F0300614D01ED8042D13D0302E11D06C
:102B1000202E30D00ED823689B78190703F00C02C2
:102B200011D43AB9FEF71EF840B93DB1032002E0D6
:102B3000002EF0D0012002B0BDE8F081236893F9A7
:102B40000230002BF6DABB0753D52379012B01D8CD
:102B50000DF011F92668A2797778E579FF2A07F058
:102B600007070CD1FF2D2FD1FDF7FCFF002840D126
:102B7000002F3ED0DAE7E37CFF2BE4D1DAE7FF2D2C
:102B80002DD035441644FEF717F802220146304690
:102B900011F052FFB0B1214B0222B3F80080ADF822
:102BA000048001A9304611F047FF58B1002FBDD174
:102BB000FEF702F802226946ADF8008011F03CFFF2
:102BC0000028B3D10DB9CFE73544647C022C08D07E
:102BD000082C1CD0002CC7D00DF0CDF8AAE700259A
:102BE000D0E7FEF703F822460146284611F024FFFD
:102BF00008B900209FE7094B1B88ADF80430224636
